:080000009C170400020000003F
:04000C00164A000090
:10001000A64900006E490000DE490000164A0000B3
:10002000164A0000164A0000164A0000164A000050
:10003000164A0000164A0000164A0000164A000040
:10004000164A0000164A0000E84B0000164A00005D
:10005000164A00004A4A0000164A0000164A0000EC
:10006000164A0000164A0000164A0000164A000010
:10007000164A0000164A0000164A0000164A000000
:10008000164A0000164A0000164A0000164A0000F0
:10009000164A0000164A0000164A0000164A0000E0
:1000A0007C4B0000164A0000164A0000164A000069
:1000B000164A0000164A0000164A0000164A0000C0
:1000C000164A0000164A0000164A0000164A0000B0
:1000D000164A0000164A0000164A0000164A0000A0
:1000E000164A0000164A0000164A0000164A000090
:1000F000164A000036570000164A0000164A000053
:10010000164A0000164A0000164A0000164A00006F
:10011000164A0000164A0000164A0000164A00005F
:10012000164A0000164A0000164A0000FE48000069
:1001300036490000164A0000164A0000164A000020
:10014000164A0000164A0000164A0000164A00002F
:10015000164A0000164A0000164A0000164A00001F
:10016000164A0000164A0000164A0000164A00000F
:10017000164A0000164A0000164A0000164A0000FF
:10018000164A0000164A0000164A0000164A0000EF
:10019000164A0000164A0000164A0000164A0000DF
:1001A000164A0000164A0000164A0000164A0000CF
:1001B000164A0000164A0000164A0000164A0000BF
:1001C000164A0000164A0000164A0000164A0000AF
:1001D000164A0000164A0000164A0000164A00009F
:1001E000164A0000164A0000164A0000164A00008F
:1001F000164A0000164A0000164A0000164A00007F
:100400003220EF00C3202000008041001040BA00DD
:100410000160EF00000006000A0D000052650000B8
:1004200061640000436F00006E66000069670000B1
:1004300045450000507200006F6D0000204500002F
:10044000727200006F72000028730000293A0000E9
:100450000A0D0000000000003220EF00832320007E
:10046000008041001040BA000160EF00000006006B
:10047000254C0000583A000020250000327800008A
:10048000202100003D20000025320000780A0000F5
:100490000D0000003220EF006325200000804100A5
:1004A0001040BA000160EF00000006004368000041
:1004B000656300006B730000756D00002052000042
:1004C000656100006420000025320000782C0000E7
:1004D00020430000616C0000637500006C61000047
:1004E000746500006420000025320000780A0000D6
:1004F0000D0000003220EF00632820000080410042
:100500001040BA000160EF0000000600202000004B
:10051000204300006F6E0000666900006720000045
:100520005361000076650000642000002020000078
:10053000000000003220EF00632A2000008041000C
:100540001040BA000160EF0000000600436F000099
:100550006E660000696700002053000061760000AD
:10056000656400000A0D0000000000003220EF006A
:10057000232C2000008041001040BA000160EF00F1
:1005800000000600537400006F7200006520000038
:1005900046610000637400006F7200007920000063
:1005A000446500006661000075740000732000005F
:1005B00046610000696C0000656400000A0D0000DF
:1005C000000000003220EF00E32E200000804100F8
:1005D0001040BA000160EF00000006005265000004
:1005E000616400002045000045500000726F00006B
:1005F0006D20000046610000696C00006564000029
:100600000A0D0000000000003220EF00033120003E
:10061000008041001040BA000160EF0000000600B9
:10062000537400006F7200006520000044650000F4
:1006300066610000757400007320000046610000D0
:10064000696C0000656400000A0D000000000000F5
:100650003220EF0023032000830150000500310009
:1006600043342000008041001040BA000160EF00D8
:100670000000060040342000838141008081410059
:100680001380BA00000006000A0D5800446F2000D5
:100690004C6F250061644C00507258006573200057
:1006A0006574250020204C00253258007820200059
:1006B0002532630078206800254C650058206300CF
:1006C000254C6B0058207300254C750058206D0098
:1006D000254C3D0058202500254C3200582058005C
:1006E000254C000058200000254C00003220EF006F
:1006F000230320008301500005003100233920002E
:10070000008041001040BA000160EF0000000600C8
:100710002039200083814100808141001380BA008C
:1007200000000600446F25004C6F320061647800C1
:10073000507220006573210065743D003A2020004E
:1007400043204100256463002C2074005020690080
:10075000256476002C2865006B3D2000254C430065
:100760005829610020426D0061642000202D250081
:10077000205032007265640073650A0074200D0019
:10078000436100006D2000003220EF0023022000B2
:100790008301500005003100033E2000008041002D
:1007A0001040BA000160EF0000000600003E20008B
:1007B00083814100808141001380BA00000006005F
:1007C000446F6F004C6F20006164500050727200E3
:1007D00065736500657473003A20650043207400FA
:1007E000256420002C20660050206F0025647500D1
:1007F0002C286E006B3D6400254C0A0058290D0022
:10080000204E00003220EF0023032000830150001F
:1008100005003100E3412000008041001040BA0093
:100820000160EF0000000600E041200083814100EC
:10083000808141001380BA0000000600446F6B0005
:100840004C6F73006164750050726D006573200019
:10085000657425003A2032004320580025642000AA
:100860002C20210050203D00256420002C2843002E
:100870006B3D6100254C6C0058296300204220002C
:1008800061642500202D32002050580072650A0056
:1008900073650D007420000063680000656300004C
:1008A0003220EF00230320008301500005003100B7
:1008B000C3462000008041001040BA000160EF00F4
:1008C00000000600C0462000838141008081410075
:1008D0001380BA0000000600446F25005265320004
:1008E00061647800507220006573210065743D00DA
:1008F0003A20200043204100256463002C2074002E
:1009000050206900256476002C2865006B3D20008E
:10091000254C43005829610020426D00616420008D
:10092000202D2500205032007265640073650A0096
:1009300074200D00436100006D2000003220EF00A4
:10094000230220008301500005003100A34B20004A
:10095000008041001040BA000160EF000000060076
:10096000A04B200083814100808141001380BA00A8
:1009700000000600446F6F00526520006164500063
:100980005072720065736500657473003A206500EB
:1009900043207400256420002C20660050206F0046
:1009A000256475002C286E006B3D6400254C0A0000
:1009B00058290D00204E00003220EF0023032000B4
:1009C0008301500005003100834F2000008041006A
:1009D0001040BA000160EF0000000600804F2000C8
:1009E00083814100808141001380BA00000006002D
:1009F000446F6B00526573006164750050726D0046
:100A000065732000657425003A20320043205800A9
:100A1000256420002C20210050203D00256420006A
:100A20002C2843006B3D6100254C6C005829630065
:100A30002042200061642500202D32002050580003
:100A400072650A0073650D00742000006368000081
:100A5000656300003220EF00030220008301500094
:100A60000500310063542000008041001040BA00AE
:100A70000160EF0000000600605420008381410007
:100A8000808141001380BA00000006004C6F6500B1
:100A900063206E0025327400782C20002050430023
:100AA0006F72610074206D00256465002C50720027
:100AB000726561007365250074203200256464004E
:100AC0002C200A0043750D00727200003220EF00E6
:100AD000C30220008301500005003100235820008C
:100AE000008041001040BA000160EF0000000600E5
:100AF0002058200083814100808141001380BA008A
:100B000000000600536120007665250020254C007A
:100B100032785800202520003278630020256800B4
:100B20004C586500202563004C586B00202573004D
:100B30004C58750020256D004C583D00202525009F
:100B40004C583200202558004C580A0020250D0032
:100B50004C580000202500004C5800003220EF00C7
:100B6000A35B2000008041001040BA000160EF004C
:100B700000000600536F00006E7900002045000061
:100B8000564900002D4400003330000020200000B2
:100B90002020000020200000200000003220EF0074
:100BA000A35D2000008041001040BA000160EF000A
:100BB00000000600536F00006E7900002045000021
:100BC000564900002D440000333000002F4400003F
:100BD0003331000020200000200000003220EF0010
:100BE000A35F2000008041001040BA000160EF00C8
:100BF000000006005661000064640000696F000098
:100C000020410000646400002D6100002D430000BD
:100C1000616D000020200000200000003220EF0065
:100C2000A3612000008041001040BA000160EF0085
:100C300000000600536F00006E79000020450000A0
:100C4000564900002D4400003130000030200000E3
:100C50002020000020200000200000003220EF00B3
:100C6000A3632000008041001040BA000160EF0043
:100C7000000006005641000044440000494F0000B7
:100C800020480000442D00003138000020200000E2
:100C90002020000020200000200000003220EF0073
:100CA000A3652000008041001040BA000160EF0001
:100CB00000000600536F00006E7900002045000020
:100CC000564900002D44000037300000202000006D
:100CD0002020000020200000200000003220EF0033
:100CE000A3672000008041001040BA000160EF00BF
:100CF00000000600536F00006E79000020420000E3
:100D0000524300002D33000030300000202000004E
:100D10002020000020200000200000003220EF00F2
:100D2000A3692000008041001040BA000160EF007C
:100D300000000600536F00006E79000020420000A2
:100D4000524300002D4800003730000030200000E2
:100D50002020000020200000200000003220EF00B2
:100D6000A36B2000008041001040BA000160EF003A
:100D700000000600536F00006E7900002042000062
:100D8000524300002D5A0000373000003020000090
:100D90002020000020200000200000003220EF0072
:100DA000A36D2000008041001040BA000160EF00F8
:100DB00000000600536F00006E7900002042000022
:100DC000524300002D5A0000333300003020000051
:100DD0002020000020200000200000003220EF0032
:100DE000A36F2000008041001040BA000160EF00B6
:100DF00000000600536F00006E79000020450000DF
:100E0000564900002D480000443100002020000019
:100E10002020000020200000200000003220EF00F1
:100E2000A3712000008041001040BA000160EF0073
:100E300000000600506100006E610000736F00004A
:100E40006E69000063200000415700002D4800003B
:100E50004531000030300000200000003220EF005B
:100E6000A3732000008041001040BA000160EF0031
:100E70000000060043650000696C0000696E000018
:100E80006756000049450000572000002020000060
:100E90002020000020200000200000003220EF0071
:100EA000A3752000008041001040BA000160EF00EF
:100EB00000000600436100006E6E00006F6E0000CF
:100EC00020560000432D000043350000306900002B
:100ED0002F72000020200000200000003220EF00D0
:100EE000A3772000008041001040BA000160EF00AD
:100EF00000000600436100006E6E00006F6E00008F
:100F000020420000552D000034350000482000002C
:100F10002020000020200000200000003220EF00F0
:100F2000A3792000008041001040BA000160EF006A
:100F300000000600436100006E6E00006F6E00004E
:100F400020420000552D00003530000048200000F0
:100F50002020000020200000200000003220EF00B0
:100F6000A37B2000008041001040BA000160EF0028
:100F700000000600556E00006B6E00006F770000E9
:100F80006E200000436100006D650000726100008A
:100F90002020000020200000200000003220EF0070
:100FA000A37D2000008041001040BA000160EF00E6
:100FB0000000060045560000492D000044330000A3
:100FC0003020000020200000202000000000000051
:100FD0003220EF00437F2000008041001040BA0023
:100FE0000160EF000000060045560000492D00009A
:100FF00044330000302F0000443300003120000053
:10100000000000003220EF00E3802000008041005B
:101010001040BA000160EF000000060041640000CB
:10102000642D0000612D0000436100006D20000070
:1010300020200000000000003220EF00838220000A
:10104000008041001040BA000160EF00000006007F
:1010500045560000492D00004431000030300000AA
:101060002020000020200000000000003220EF00BF
:1010700023842000008041001040BA000160EF008E
:1010800000000600484400002D3100003820000018
:101090002020000020200000202000000000000090
:1010A0003220EF00C3852000008041001040BA00CC
:1010B0000160EF000000060045560000492D0000C9
:1010C00044370000302000002020000020200000D5
:1010D000000000003220EF00638720000080410004
:1010E0001040BA000160EF0000000600425200000C
:1010F000432D00003330000030200000202000008D
:1011000020200000000000003220EF0003892000B2
:10111000008041001040BA000160EF0000000600AE
:1011200042520000432D00004837000030300000DC
:101130002020000020200000000000003220EF00EE
:10114000A38A2000008041001040BA000160EF0037
:101150000000060042520000432D00005A370000F4
:10116000303000002020000020200000000000009F
:101170003220EF00438C2000008041001040BA0074
:101180000160EF000000060042520000432D000005
:101190005A330000333000002020000020200000DF
:1011A000000000003220EF00E38D200000804100AD
:1011B0001040BA000160EF00000006004556000034
:1011C000492D00004844000031200000202000008C
:1011D00020200000000000003220EF00838F20005C
:1011E000008041001040BA000160EF0000000600DE
:1011F000415700002D48000045310000303000000C
:101200002020000020200000000000003220EF001D
:1012100023912000008041001040BA000160EF00DF
:101220000000060043650000696C0000696E000064
:1012300067560000494500005720000000000000EC
:101240003220EF00C3922000008041001040BA001D
:101250000160EF0000000600564300002D4300002F
:1012600035300000692F00007220000020200000AF
:10127000000000003220EF00639420000080410055
:101280001040BA000160EF00000006004255000067
:101290002D340000354800002020000020200000F0
:1012A00020200000000000003220EF000396200004
:1012B000008041001040BA000160EF00000006000D
:1012C000425500002D35000030480000202000006D
:1012D0002020000020200000000000003220EF004D
:1012E000A3972000008041001040BA000160EF0089
:1012F00000000600556E00006B6E00006F77000066
:101300006E200000202000002020000000000000CF
:101310003220EF0043992000008041001040BA00C5
:101320000160EF0000000600000000003220EF0026
:10133000239A2000008041001040BA000160EF00B5
:10134000000006005379000073740000656D000012
:1013500020430000616D0000204900006E6900001C
:10136000742000003A200000557300006520000042
:101370005072000065730000657400003134000095
:10138000000000003220EF00E39C200000804100BC
:101390001040BA000160EF00000006005379000021
:1013A00073740000656D000020430000616D000053
:1013B000204900006E690000742000003A200000FF
:1013C000486F00006D65000020430000616D000063
:1013D0006572000061200000000000003220EF0074
:1013E000A39F2000008041001040BA000160EF0080
:1013F0000000060050720000657300006574000074
:10140000204C00006F63000061740000696F0000F1
:101410006E3A0000203100002D3600002049000007
:101420006E430000616D00002C3700002D3100007C
:10143000342000004C6F0000636100006C0000006D
:101440003220EF00C3A22000008041001040BA000B
:101450000160EF000000060050720000657300009C
:1014600065740000204C00006F6300006174000090
:10147000696F00006E3A0000203100002D3100003D
:10148000342000004C6F0000636100006C0000001D
:101490003220EF0043A52000008041001040BA0038
:1014A0000160EF0000000600486F00007374000048
:1014B0002053000065720000696100006C2000008C
:1014C000496E000070750000743A0000204500006D
:1014D0006E610000626C00006564000000000000A6
:1014E0003220EF00C3A72000008041001040BA0066
:1014F0000160EF0000000600486F000073740000F8
:101500002053000065720000696100006C2000003B
:10151000496E000070750000743A0000204400001D
:1015200069730000616200006C65000064000000E7
:101530003220EF0043AA2000008041001040BA0092
:101540000160EF00000006005365000072690000B2
:10155000616C000020450000636800006F3A0000E5
:10156000204500006E610000626C000065640000B0
:10157000000000003220EF0063AC2000008041003A
:101580001040BA000160EF00000006005365000043
:1015900072690000616C0000204500006368000073
:1015A0006F3A00002044000069730000616200008F
:1015B0006C650000640000003220EF0083AE200064
:1015C000008041001040BA000160EF0000000600FA
:1015D0005365000072690000616C00002049000042
:1015E0006E6600006F3A0000204F00006E000000A1
:1015F0003220EF0043B02000008041001040BA00CC
:101600000160EF00000006005365000072690000F1
:10161000616C0000204900006E6600006F3A000017
:10162000204F000066660000000000003220EF003E
:1016300023B22000008041001040BA000160EF009A
:1016400000000600546100006C6C0000792000006E
:101650004C650000766500006C3A000020410000F7
:10166000637400006976000065200000486900008E
:1016700067680000000000003220EF0083B4200003
:10168000008041001040BA000160EF000000060039
:10169000546100006C6C0000792000004C65000073
:1016A000766500006C3A0000204100006374000081
:1016B00069760000652000004C6F00007700000094
:1016C0003220EF00C3B62000008041001040BA0075
:1016D0000160EF0000000600486F00006D6500002B
:1016E0002042000075740000746F00006E3A000024
:1016F0002044000069730000616200006C65000016
:10170000640000003220EF00E3B8200000804100B8
:101710001040BA000160EF0000000600486F0000B2
:101720006D6500002042000075740000746F0000B9
:101730006E3A0000204500006E610000626C0000FF
:1017400065640000000000003220EF0003BB2000B1
:10175000008041001040BA000160EF000000060068
:1017600044690000616700006E6F00007374000040
:1017700069630000204D00006F640000653A0000BE
:10178000204F00006E0000003220EF0003BD20005B
:10179000008041001040BA000160EF000000060028
:1017A00044690000616700006E6F00007374000000
:1017B00069630000204D00006F640000653A00007E
:1017C000204F000066660000000000003220EF009D
:1017D00023BF2000008041001040BA000160EF00EC
:1017E000000006005365000072690000616C000093
:1017F0002044000069610000672000004D6F000078
:10180000646500003A2000004F6E000000000000F8
:101810003220EF0043C12000008041001040BA0098
:101820000160EF00000006005365000072690000CF
:10183000616C000020440000696100006720000026
:101840004D6F0000646500003A2000004F66000004
:10185000660000003220EF0063C3200000804100DA
:101860001040BA000160EF00000006004361000074
:101870006D6500007261000020530000656C00007F
:1018800065630000742000006F6E0000203A0000C5
:10189000204300006F6E0000747200006F6C000047
:1018A00020410000000000003220EF0003C62000AD
:1018B000008041001040BA000160EF000000060007
:1018C000436100006D65000072610000205300005C
:1018D000656C000065630000742000006F6E0000FE
:1018E000203A0000204300006F6E00007472000078
:1018F0006F6C000020420000000000003220EF006A
:10190000A3C82000008041001040BA000160EF0031
:1019100000000600436100006D6500007261000078
:1019200020530000656C0000656300007420000017
:101930006F6E00003A2000004469000073610000EF
:10194000626C000065640000000000003220EF00BF
:1019500023CB2000008041001040BA000160EF005E
:1019600000000600526500006D6F00007465000005
:10197000204C0000696E00006B2000004D6F0000DD
:10198000646500003A20000044750000616C0000AE
:10199000204D0000617300007465000072000000BB
:1019A0003220EF00C3CD2000008041001040BA007B
:1019B0000160EF0000000600526500006D6F00003E
:1019C00074650000204C0000696E00006B20000070
:1019D0004D6F0000646500003A2000004D6100007A
:1019E0007374000065720000203C00002D3E000072
:1019F000205300006C6100007665000000000000CC
:101A00003220EF00C3D02000008041001040BA0017
:101A10000160EF00000006004461000074610000F6
:101A20002053000077690000746300006820000004
:101A30004D6F0000646500003A200000456400001E
:101A4000697200006F6C0000000000003220EF009F
:101A500023D32000008041001040BA000160EF0055
:101A60000000060044610000746100002053000083
:101A70007769000074630000682000004D6F00006B
:101A8000646500003A2000004953000049530000FB
:101A9000000000003220EF0063D5200000804100EC
:101AA0001040BA000160EF00000006004461000031
:101AB0007461000020530000776900007463000027
:101AC000682000004D6F0000646500003A200000AF
:101AD000416E0000616C00006F67000057610000FC
:101AE000790000003220EF00E3D7200000804100A1
:101AF0001040BA000160EF000000060044610000E1
:101B000074610000205300007769000074630000D6
:101B1000682000004D6F0000646500003A2000005E
:101B200045780000747200006F6E00000000000035
:101B30003220EF0043DA2000008041001040BA005C
:101B40000160EF00000006004461000074610000C5
:101B500020530000776900007463000068200000D3
:101B60004D6F0000646500003A20000055730000CE
:101B7000657200002044000065660000696E000088
:101B800065640000000000003220EF0003DD20004B
:101B9000008041001040BA000160EF000000060024
:101BA0004461000074610000205300007769000068
:101BB00074630000682000004D6F00006465000041
:101BC0003A2000004469000073610000626C00006C
:101BD00065640000000000003220EF0083DF200079
:101BE000008041001040BA000160EF0000000600D4
:101BF0005061000073730000204F00006E20000051
:101C00005374000061740000757300003A200000F6
:101C10004163000074690000766500000000000068
:101C20003220EF00C3E12000008041001040BA00E4
:101C30000160EF00000006005061000073730000B7
:101C4000204F00006E2000005374000061740000FB
:101C5000757300003A200000496E000061630000C7
:101C60007469000076650000000000003220EF007B
:101C700023E42000008041001040BA000160EF0022
:101C80000000060050610000737300002052000045
:101C900065730000706F00006E7300006520000027
:101CA0005374000061740000757300003A20000056
:101CB000506500006E640000696E0000670000005F
:101CC0003220EF00C3E62000008041001040BA003F
:101CD0000160EF0000000600506100007373000017
:101CE0002052000065730000706F00006E730000EA
:101CF00065200000537400006174000075730000DB
:101D00003A200000496400006C65000000000000FB
:101D10003220EF0043E92000008041001040BA006B
:101D20000160EF00000006005061000073730000C6
:101D3000204D00006F640000652000005374000017
:101D40006172000074650000640000003220EF0042
:101D500023EB2000008041001040BA000160EF003A
:101D6000000006005061000073730000204D000069
:101D70006F640000652000006E6F0000742000009A
:101D8000537400006172000074650000640000007C
:101D90003220EF0043ED2000008041001040BA00E7
:101DA0000160EF0000000600506100006E2F00008F
:101DB000546900006C74000020530000746100003E
:101DC00074750000733A0000204100006374000045
:101DD00069760000650000003220EF0083EF2000EC
:101DE000008041001040BA000160EF0000000600D2
:101DF000506100006E2F0000546900006C740000F8
:101E0000205300007461000074750000733A0000F4
:101E100020490000646C0000650000003220EF00E3
:101E2000A3F12000008041001040BA000160EF00E3
:101E3000000006005A6F00006F6D00002053000084
:101E40007461000074750000733A000020410000C6
:101E50006374000069760000650000003220EF0026
:101E6000A3F32000008041001040BA000160EF00A1
:101E7000000006005A6F00006F6D00002053000044
:101E80007461000074750000733A0000204900007E
:101E9000646C0000650000003220EF0083F5200034
:101EA000008041001040BA000160EF000000060011
:101EB0004C6F0000636100006C2000006361000053
:101EC0006D6500007261000073200000666F000005
:101ED000756E0000643A0000204E00006F000000A4
:101EE0003220EF00C3F72000008041001040BA000C
:101EF0000160EF00000006004C6F0000636100000D
:101F00006C200000636100006D65000072610000DC
:101F100073200000666F0000756E0000643A0000D8
:101F20002059000065730000000000003220EF001F
:101F300023FA2000008041001040BA000160EF0049
:101F400000000600436100006D6500007261000042
:101F5000204300006F6E0000747200006F6C000080
:101F60003A2000004C6F0000636100006C0000002C
:101F70003220EF0043FC2000008041001040BA00F6
:101F80000160EF0000000600436100006D65000085
:101F900072610000204300006F6E00007472000048
:101FA0006F6C00003A200000526500006D6F000069
:101FB00074650000000000003220EF0083FE200066
:101FC000008041001040BA000160EF0000000600F0
:101FD000526500006D6F000074650000284D000020
:101FE000617300007465000072290000204C00003D
:101FF000696E00006B2000004163000074690000FE
:1020000076650000000000003220EF00030121008F
:10201000008041001040BA000160EF00000006009F
:10202000526500006D6F000074650000284D0000CF
:10203000617300007465000072290000204C0000EC
:10204000696E00006B2000006E6F000074200000BD
:102050004163000074690000766500000000000024
:102060003220EF00C3032100008041001040BA007D
:102070000160EF0000000600526500006D6F000077
:1020800074650000285300006C6100007665000054
:10209000292000004C6900006E6B00002041000008
:1020A0006374000069760000650000003220EF00D4
:1020B00023062100008041001040BA000160EF00BB
:1020C00000000600526500006D6F0000746500009E
:1020D000285300006C610000766500002920000094
:1020E0004C6900006E6B0000206E00006F740000F1
:1020F0002041000063740000697600006500000064
:102100003220EF00C3082100008041001040BA00D7
:102110000160EF0000000600436F00006E740000D5
:10212000726F00006C6C00006572000020530000AC
:102130007461000074750000733A000020520000C2
:10214000656D00006F740000650000003220EF0034
:10215000230B2100008041001040BA000160EF0015
:1021600000000600436F00006E740000726F0000F4
:102170006C6C000065720000205300007461000068
:1021800074750000733A0000204C00006F6300007B
:10219000616C0000000000003220EF00830D210080
:1021A000008041001040BA000160EF00000006000E
:1021B000507200006F670000726100006D20000027
:1021C0004D6F0000646500003A200000416300008C
:1021D0007469000076650000000000003220EF0006
:1021E000A30F2100008041001040BA000160EF0001
:1021F00000000600507200006F670000726100006E
:102200006D2000004D6F0000646500003A20000062
:10221000496400006C650000000000003220EF00FF
:10222000A3112100008041001040BA000160EF00BE
:1022300000000600525800002053000074610000A6
:10224000746500003A200000584F00004646000028
:10225000000000003220EF006313210000804100E5
:102260001040BA000160EF00000006005258000064
:102270002053000074610000746500003A200000E3
:10228000584F00004E0000003220EF0003152100DF
:10229000008041001040BA000160EF00000006001D
:1022A0005458000020530000746100007465000061
:1022B0003A200000584F0000464600000000000091
:1022C0003220EF00C3162100008041001040BA0008
:1022D0000160EF0000000600545800002053000089
:1022E00074610000746500003A200000584F00003F
:1022F0004E0000003220EF006318210000804100F2
:102300001040BA000160EF000000060050540000C9
:102310005A200000536500006E6400002053000046
:1023200074610000746500003A20000050650000F0
:102330006E640000696E0000670000003220EF004C
:10234000A31A2100008041001040BA000160EF0094
:1023500000000600505400005A20000053650000A1
:102360006E6400002053000074610000746500007A
:102370003A200000496400006C6500000000000085
:102380003220EF00C31C2100008041001040BA0041
:102390000160EF0000000600446F00004669000085
:1023A0006E640000416300007469000076650000FF
:1023B0005072000065730000657400007320000017
:1023C000506F00007274000020250000642000009F
:1023D00062610000640A00000D0000003220EF007E
:1023E000030220008301500005003100A3202100DA
:1023F000008041001040BA000160EF0000000600BC
:10240000A020210083814100808141001380BA0017
:10241000000006000A0D7200446F650046697300F3
:102420006E64650041637400746920007665310054
:10243000507220006573250065744C0073205800AD
:1024400043613A006D202000256420003A202000DE
:102450002D5000003220EF00632321000080410056
:102460001040BA000160EF00000006000A0D0000F5
:10247000553400005F490000535200002025000041
:1024800032580000202500003258000020250000AE
:10249000325800002025000032580000202500009E
:1024A00032580000000000003220EF000326210017
:1024B000008041001040BA000160EF0000000600FB
:1024C0002043000043550000204D00006F640000D1
:1024D000652000004163000074690000766500001B
:1024E000200000003220EF00E3272100008041009F
:1024F0001040BA000160EF000000060055340000F3
:102500005F4200003020000049530000522D0000BF
:1025100045720000722000002532000058200000A3
:10252000253200005820000025320000582000000D
:1025300025320000582000005B25000032580000C2
:102540005D0A00000D0000003220EF00032B210087
:10255000008041001040BA000160EF00000006005A
:10256000553400005F420000312000004953000054
:10257000522D00004572000072200000253200003C
:1025800058200000253200005820000025320000AD
:10259000582000005B250000325800005D2000003C
:1025A00025320000580A00000D0000003220EF0024
:1025B000232E2100008041001040BA000160EF008E
:1025C00000000600553800005F4200003220000085
:1025D00049530000522D0000457200007220000097
:1025E000253200005820000025320000582000004D
:1025F0005B250000325800005D20000025320000FD
:102600005820000025320000580A00000D0000008C
:102610003220EF0043312100008041001040BA0019
:102620000160EF0000000600524D00005420000041
:10263000506700006D2000004D6F000064650000D1
:1026400020250000750A00000D0000003220EF0078
:1026500023332100008041001040BA000160EF00E8
:1026600000000600205200004D54000020500000E1
:10267000726F000067720000616D0000204D000065
:102680006F64000065200000000000003220EF00B1
:1026900023352100008041001040BA000160EF00A6
:1026A00000000600553400005F42000033200000A7
:1026B00049530000522D00004572000072200000B6
:1026C00025320000582000005B2500003258000031
:1026D0005D20000025320000582000002532000057
:1026E0005820000025320000582000000A0D00008C
:1026F000000000003220EF0063382100008041001C
:102700001040BA000160EF000000060055340000E0
:102710005F4200003420000049530000522D0000A9
:1027200045720000722000005B2500003258000056
:102730005D200000253200005820000025320000F6
:1027400058200000253200005820000025320000EB
:10275000582000000A0D0000000000003220EF00A9
:10276000A33B2100008041001040BA000160EF004F
:10277000000006000A0D00004E6F00004C690000CA
:102780006E6B0000000000003220EF00033D2100CE
:10279000008041001040BA000160EF000000060018
:1027A0000A0D0000576900006E6400006F7700009A
:1027B0002053000068750000746400006F7700000B
:1027C0006E2C0000204D00006178000028250000DC
:1027D000752900002043000075720000726500003A
:1027E0006E7400002825000075290000000000001C
:1027F0003220EF0043402100008041001040BA0029
:102800000160EF00000006000A0D0000282500000E
:1028100075290000536500006E640000204C000024
:10282000696E00006B2000004461000074610000CC
:1028300020250000327800002025000032780000BA
:1028400020250000327800002025000032780000AA
:10285000000000003220EF0003022000830150003E
:102860000500310063442100008041001040BA009F
:102870000160EF00000006006044210083814100F8
:10288000808141001380BA00000006000A0D780024
:102890004F7520007451250020463200756C780079
:1028A0006C2C2000206D2500657332007361780068
:1028B0006765200020642500726F32007070780018
:1028C0006564290020280000253200003220EF0036
:1028D00043032000830150000500310023482100FC
:1028E000008041001040BA000160EF0000000600C7
:1028F0002048210083814100808141001380BA007B
:10290000000006000A0D250044514C00204D7500C2
:1029100065732900736120006765480020446900E1
:10292000617467006120680028252800327825003E
:1029300020254C00327875002025290032782000AF
:10294000202557003278690029206E00496E640006
:1029500064656F00782877002575280029202500F8
:10296000436F7500756E2900742800003220EF0057
:10297000234C2100008041001040BA000160EF00AC
:10298000000006000A0D0000507200006F63000096
:1029900065730000735200006D7400004274000003
:1029A0006E28000029200000636D000064200000F4
:1029B0002532000078200000253200007820000039
:1029C0002532000078200000253200007800000049
:1029D0003220EF00434F2100008041001040BA0038
:1029E0000160EF000000060020200000204D0000E4
:1029F000616E0000756100006C200000466F0000F1
:102A0000637500007320000020200000000000001B
:102A10003220EF0043512100008041001040BA00F5
:102A20000160EF00000006002020000020200000D0
:102A300041750000746F0000204600006F630000C5
:102A4000757300002020000020200000000000001E
:102A50003220EF0043532100008041001040BA00B3
:102A60000160EF0000000600204E00006F740000BF
:102A70002073000075700000706F00007274000019
:102A800065640000202000002020000000000000FD
:102A90003220EF0043552100008041001040BA0071
:102AA0000160EF0000000600202000002020000050
:102AB0004661000073740000204600006F63000050
:102AC000757300002020000020200000000000009E
:102AD0003220EF0043572100008041001040BA002F
:102AE0000160EF000000060020200000466F00009B
:102AF0006375000073200000506F00007320000019
:102B0000256C0000750000003220EF000359210001
:102B1000008041001040BA000160EF000000060094
:102B2000204600006173000074200000466F000022
:102B30006375000073200000457800006974000090
:102B400020200000000000003220EF00035B210085
:102B5000008041001040BA000160EF000000060054
:102B60002043000043550000204D00006F6400002A
:102B70006520000041630000746900007665000074
:102B800020200000000000003220EF00035D210043
:102B9000008041001040BA000160EF000000060014
:102BA000204D0000616E0000756100006C20000087
:102BB0005768000069740000652000004261000051
:102BC0006C200000000000003220EF00035F2100B5
:102BD000008041001040BA000160EF0000000600D4
:102BE00041750000746F0000205700006869000004
:102BF0007465000020420000616C0000616E0000FE
:102C000063650000000000003220EF000361210036
:102C1000008041001040BA000160EF000000060093
:102C20004E6F000020430000616D000065720000DF
:102C300061200000536500006C65000063740000B3
:102C400065640000000000003220EF0003632100F3
:102C5000008041001040BA000160EF000000060053
:102C6000204F00006E6500002050000075730000CA
:102C700068200000574200002020000020200000B3
:102C800020200000000000003220EF00036521003A
:102C9000008041001040BA000160EF000000060013
:102CA00042610000636B00006C690000676800000F
:102CB00074200000436F00006D700000206E000063
:102CC0002F610000000000003220EF0003672100A8
:102CD000008041001040BA000160EF0000000600D3
:102CE00020200000204D0000616E00007561000092
:102CF0006C20000049720000697300002020000071
:102D000020200000000000003220EF0003692100B5
:102D1000008041001040BA000160EF000000060092
:102D20002020000020410000757400006F2000008A
:102D3000497200006973000020200000202000007C
:102D400020200000000000003220EF00036B210073
:102D5000008041001040BA000160EF000000060052
:102D600042610000636B00006C690000676800004E
:102D700074200000436F00006D700000204F0000C1
:102D800066660000000000003220EF00036D2100A5
:102D9000008041001040BA000160EF000000060012
:102DA00042610000636B00006C690000676800000E
:102DB00074200000436F00006D700000204F000081
:102DC0006E200000000000003220EF00036F2100A1
:102DD000008041001040BA000160EF0000000600D2
:102DE00020200000204800006F6D000065200000DA
:102DF000436100006D65000072610000202000004A
:102E000020200000000000003220EF0003712100AC
:102E1000008041001040BA000160EF000000060091
:102E20002020000020200000436100006D650000AC
:102E300072610000202500006420000020200000B6
:102E400020200000200000003220EF00037321004A
:102E5000008041001040BA000160EF000000060051
:102E60004E6F000020430000616D0000657200009D
:102E700061200000466F0000756E000064200000B5
:102E800020200000000000003220EF000375210028
:102E9000008041001040BA000160EF000000060011
:102EA000427400006E20000025640000206E0000C7
:102EB0006F7400002064000065660000696E000009
:102EC00065640000200000003220EF00037721003D
:102ED000008041001040BA000160EF0000000600D1
:102EE000496E0000436100006D65000072610000E2
:102EF000205000007265000073650000742000001F
:102F000025320000640000003220EF000379210028
:102F1000008041001040BA000160EF000000060090
:102F200020200000507200006573000065740000EE
:102F30002025000032640000000000003220EF0075
:102F4000A37A2100008041001040BA000160EF0028
:102F50000000060020200000426100006420000004
:102F600050720000657300006574000020250000A9
:102F70003264000020200000000000003220EF003A
:102F8000A37C2100008041001040BA000160EF00E6
:102F900000000600202000004E6F000020500000BE
:102FA0007265000073650000742000002532000087
:102FB00064200000200000003220EF00837E21000A
:102FC000008041001040BA000160EF0000000600E0
:102FD000202000004E6F0000742000006F6E000083
:102FE000205000007265000073650000742000002E
:102FF00020200000000000003220EF00838021002C
:10300000008041001040BA000160EF00000006009F
:10301000202000002049000072690000733A00007F
:1030200020250000730000003220EF000382210001
:10303000008041001040BA000160EF00000006006F
:103040002020000020490000726900007320000069
:1030500025730000000000003220EF008383210070
:10306000008041001040BA000160EF00000006003F
:103070002020000020490000726900007320000039
:10308000256C0000750000003220EF000385210050
:10309000008041001040BA000160EF00000006000F
:1030A000202000004D610000782000005A6F0000D1
:1030B0006F6D000020250000750000003220EF0039
:1030C000A3862100008041001040BA000160EF009B
:1030D00000000600202000004D6100007820000064
:1030E000506100006E200000257500000000000007
:1030F0003220EF0043882100008041001040BA00D8
:103100000160EF0000000600202000004D6100007B
:1031100078200000546900006C7400002025000035
:10312000750000003220EF00E3892100008041009B
:103130001040BA000160EF000000060020200000EF
:103140002052000065640000204700006169000013
:103150006E2000004E2F00004120000020200000C3
:10316000000000003220EF00E38B210000804100CE
:103170001040BA000160EF000000060020200000AF
:10318000526500006420000047610000696E000085
:103190003E20000025640000000000003220EF0007
:1031A000A38D2100008041001040BA000160EF00B3
:1031B000000006002020000052650000642000008E
:1031C00047610000696E00003E200000254C0000B1
:1031D000640000003220EF00638F21000080410076
:1031E0001040BA000160EF0000000600202000003F
:1031F000204200006C75000065200000476100005F
:10320000696E0000204E00002F41000020200000C9
:10321000000000003220EF00639121000080410097
:103220001040BA000160EF000000060020200000FE
:10323000426C0000756500002047000061690000D5
:103240006E3E000020250000640000003220EF00E8
:1032500023932100008041001040BA000160EF007C
:103260000000060020200000426C00007565000090
:1032700020470000616900006E3E0000202500002C
:103280004C640000000000003220EF000395210094
:10329000008041001040BA000160EF00000006000D
:1032A00020200000204400006574000061690000D7
:1032B0006C2000004E2F0000412000002020000064
:1032C00020200000000000003220EF0003972100C2
:1032D000008041001040BA000160EF0000000600CD
:1032E000202000004465000074610000696C00004B
:1032F0003E20000025640000000000003220EF00A6
:10330000A3982100008041001040BA000160EF0046
:10331000000006002020000020200000476100007F
:10332000696E0000204E00002F41000020200000A8
:103330002020000020200000000000003220EF00CC
:10334000A39A2100008041001040BA000160EF0004
:103350000000060020470000616900006E3E00008A
:1033600025730000000000003220EF00039C2100C4
:10337000008041001040BA000160EF00000006002C
:1033800020490000726900007320000047610000BE
:10339000696E00003E2500007564000042000000D8
:1033A0003220EF00C39D2100008041001040BA0090
:1033B0000160EF0000000600204700006169000086
:1033C0006E3E000020250000750000003220EF0056
:1033D000239F2100008041001040BA000160EF00EF
:1033E000000006002041000057420000204D000070
:1033F0006F640000652000004163000074690000F4
:103400007665000020200000000000003220EF0060
:1034100023A12100008041001040BA000160EF00AC
:10342000000006002020000020200000497200005B
:1034300069730000204E00002F4100002020000092
:103440002020000020200000000000003220EF00BB
:1034500023A32100008041001040BA000160EF006A
:103460000000060020200000466F00006375000089
:1034700073200000506F0000732000004E2F0000EA
:103480004120000020200000000000003220EF005A
:1034900023A52100008041001040BA000160EF0028
:1034A0000000060020200000466F00006375000049
:1034B000732000004E6500006172000020200000B3
:1034C0002020000020200000000000003220EF003B
:1034D00023A72100008041001040BA000160EF00E6
:1034E0000000060020200000466F00006375000009
:1034F00073200000466100007220000020200000C0
:103500002020000020200000000000003220EF00FA
:1035100023A92100008041001040BA000160EF00A3
:103520000000060020410000757400006F200000BC
:1035300049720000697300002041000063740000BC
:103540006976000065200000000000003220EF00D6
:1035500023AB2100008041001040BA000160EF0061
:10356000000006002057000069700000657200002E
:10357000204100006374000069760000617400005F
:103580006564000020200000000000003220EF00F1
:1035900023AD2100008041001040BA000160EF001F
:1035A0000000060020200000486F00006D6500004C
:1035B0002044000069730000616200006C65000037
:1035C0006420000020200000000000003220EF00F6
:1035D00023AF2100008041001040BA000160EF00DD
:1035E0000000060020430000616E00006F6E0000C6
:1035F000204900006D670000537400006162000004
:10360000204F00004E200000000000003220EF009C
:1036100023B12100008041001040BA000160EF009A
:103620000000060020430000616E00006F6E000085
:10363000204900006D6700005374000061620000C3
:10364000204F000046460000000000003220EF003E
:1036500023B32100008041001040BA000160EF0058
:103660000000060020200000204900006E760000C7
:10367000616C000069640000204300006F6400007A
:103680006520000020200000000000003220EF0034
:1036900023B52100008041001040BA000160EF0016
:1036A00000000600427400006E2800002532000071
:1036B000782F000025750000292D000047720000BA
:1036C00070310000200A00000D0000003220EF00E1
:1036D00023B72100008041001040BA000160EF00D4
:1036E0000000060020200000504700004D20000090
:1036F0004D6F00006465000020410000637400000D
:103700006976000065200000200000003220EF00F4
:1037100023B92100008041001040BA000160EF0091
:1037200000000600506F0000776500007220000066
:103730004F660000660A00000D0000003220EF0016
:10374000A3BA2100008041001040BA000160EF00E0
:1037500000000600506F0000776500007220000036
:103760004F6E00000A0D0000000000003220EF0044
:1037700023BC2100008041001040BA000160EF002E
:1037800000000600466F000063750000734D0000E6
:10379000616E0000756100006C0A00000D00000001
:1037A0003220EF00C3BD2100008041001040BA006C
:1037B0000160EF0000000600466F00006375000026
:1037C00073410000757400006F0A00000D000000D6
:1037D0003220EF0043BF2100008041001040BA00BA
:1037E0000160EF0000000600204E00006F74000032
:1037F0002073000075700000706F0000727400008C
:103800006564000020200000200000003220EF004E
:1038100023C12100008041001040BA000160EF0088
:10382000000006004661000073740000466F00004F
:1038300063750000732000004F6E00000A0D000049
:10384000000000003220EF00E3C2210000804100B0
:103850001040BA000160EF00000006004661000061
:1038600073740000466F0000637500007320000051
:103870004F460000460A00000D0000003220EF0015
:10388000A3C42100008041001040BA000160EF0095
:1038900000000600574200004D6100006E750000F8
:1038A000616C00000A0D0000000000003220EF00F3
:1038B00023C62100008041001040BA000160EF00E3
:1038C000000006005742000041750000746F0000C0
:1038D0000A0D0000000000003220EF0083C7210025
:1038E000008041001040BA000160EF0000000600B7
:1038F000204F00006E65000020500000757300002E
:103900006820000057420000202000002020000016
:10391000000000003220EF0063C921000080410058
:103920001040BA000160EF00000006004F6E00007A
:1039300065200000507500007368000020570000EB
:10394000420A00000D0000003220EF0003CB2100EE
:10395000008041001040BA000160EF000000060046
:103960002041000057420000204D00006F6400001D
:103970006520000041630000746900007665000066
:10398000200000003220EF00E3CC21000080410045
:103990001040BA000160EF0000000600497200000C
:1039A000697300004D6100006E0A00000D00000008
:1039B0003220EF0043CE2100008041001040BA00C9
:1039C0000160EF000000060049720000697300000A
:1039D00041750000746F00000A0D00000000000037
:1039E0003220EF00C3CF2100008041001040BA0018
:1039F0000160EF0000000600424C00004320000080
:103A00004F660000660A00000D0000003220EF0043
:103A100023D12100008041001040BA000160EF0076
:103A200000000600424C0000432000004F6E0000E2
:103A30000A0D0000000000003220EF0083D22100B8
:103A4000008041001040BA000160EF000000060055
:103A500020200000204800006F6D0000652000005D
:103A6000436100006D6500007261000020200000CD
:103A7000200000003220EF0063D4210000804100CC
:103A80001040BA000160EF0000000600486F00001F
:103A90006D650000436100006D0A00000D0000002C
:103AA0003220EF00C3D52100008041001040BA0051
:103AB0000160EF000000060020200000486F0000B9
:103AC0006D65000020440000697300006162000021
:103AD0006C65000064200000200000003220EF0030
:103AE000A3D72100008041001040BA000160EF0020
:103AF000000006000A0D0000427400006E2800005D
:103B000025320000782F000025750000292D0000C7
:103B10004772000070330000000000003220EF0008
:103B2000A3D92100008041001040BA000160EF00DD
:103B30000000060025630000494E0000503A0000D6
:103B4000256400003B25000063540000414B000049
:103B50003A250000642E0000256400003B000000B0
:103B60003220EF00C3DB2100008041001040BA008A
:103B70000160EF000000060025630000494E0000D0
:103B8000503A0000256400003B0000003220EF00A6
:103B900023DD2100008041001040BA000160EF00E9
:103BA000000006000A0D0000436100006D65000082
:103BB00072610000202500006420000053650000B1
:103BC0006C65000063740000656400000000000084
:103BD0003220EF0043DF2100008041001040BA0096
:103BE0000160EF00000006004E6F00002050000052
:103BF000726F000067720000616D000020730000AA
:103C000075700000706F000072740000000000000A
:103C10003220EF0043E12100008041001040BA0053
:103C20000160EF0000000600506700006D200000FA
:103C30004D6F00006465000020250000750A00003B
:103C40000D0000003220EF00E3E22100008041007F
:103C50001040BA000160EF00000006002050000094
:103C6000726F000067720000616D0000204D00005F
:103C70006F6400006520000020200000202000006C
:103C8000000000003220EF00E3E42100008041004A
:103C90001040BA000160EF00000006004361000020
:103CA0006D6500007261000020250000640A0000BC
:103CB0000D0000003220EF0063E62100008041008B
:103CC0001040BA000160EF0000000600496E0000DD
:103CD00043740000726C0000412000002564000065
:103CE0000A0D0000000000003220EF0003E8210070
:103CF000008041001040BA000160EF0000000600A3
:103D0000496E000043740000726C00004220000005
:103D1000256400000A0D0000000000003220EF00C2
:103D2000A3E92100008041001040BA000160EF00CB
:103D300000000600427400006E28000025320000DA
:103D4000782F000025750000292D00004772000023
:103D500070340000200A00000D0000003220EF0047
:103D6000A3EB2100008041001040BA000160EF0089
:103D700000000600496E000020430000616D000055
:103D80006572000061200000537400006F72000033
:103D90006520000025640000000000003220EF00D4
:103DA000A3ED2100008041001040BA000160EF0047
:103DB00000000600496E000020430000616D000015
:103DC0006572000061200000537400006F720000F3
:103DD00065200000256400000A0D000000000000BE
:103DE0003220EF00C3EF2100008041001040BA00F4
:103DF0000160EF0000000600202000005265000076
:103E000061640000696E00006720000043610000EB
:103E10006D650000726100002020000000000000BD
:103E20003220EF00C3F12100008041001040BA00B1
:103E30000160EF0000000600202000005374000025
:103E40006F720000696E0000672000005072000071
:103E50006573000065740000202000002000000051
:103E60003220EF00C3F32100008041001040BA006F
:103E70000160EF000000060020530000746F000096
:103E8000726500002050000072650000736500003C
:103E90007420000025320000642000002000000093
:103EA0003220EF00C3F52100008041001040BA002D
:103EB0000160EF0000000600537400006F72000004
:103EC00065200000256400000A0D000000000000CD
:103ED0003220EF0043F72100008041001040BA007B
:103EE0000160EF0000000600452D00005374000043
:103EF0006F72000065200000253200006420000081
:103F000046610000696C000065640000000000006C
:103F10003220EF0043F92100008041001040BA0038
:103F20000160EF000000060020530000746F0000E5
:103F30007265000020250000326400002046000069
:103F4000616900006C650000640000003220EF0031
:103F500023FB2100008041001040BA000160EF0007
:103F600000000600496E0000436100006D6500001E
:103F7000726100002050000072650000736500004F
:103F800074200000256400000A0D000000000000FD
:103F90003220EF0043FD2100008041001040BA00B4
:103FA0000160EF0000000600507200006573000021
:103FB0006574000020250000640A00000D00000068
:103FC0003220EF00C3FE2100008041001040BA0003
:103FD0000160EF00000006000A0D000050720000B2
:103FE0006563000069730000696F00006E430000A4
:103FF000616D0000436F00006E740000726F00007E
:104000006C6C000065720000257300000A0D000052
:10401000000000003220EF00630122000080410018
:104020001040BA000160EF000000060020200000F0
:1040300020200000436F00006D700000696C0000DC
:10404000656400003A200000257300002061000034
:1040500074200000257300000A0D0000000000001D
:104060003220EF00C3032200008041001040BA005C
:104070000160EF0000000600313200002D4A000010
:10408000616E00002D310000300000003220EF0092
:1040900023052200008041001040BA000160EF00BB
:1040A00000000600313600003A330000373A0000C5
:1040B00034370000000000003220EF0083062200A9
:1040C000008041001040BA000160EF0000000600CF
:1040D000202000002053000061760000696E00007F
:1040E00067200000436F00006E66000069670000F3
:1040F00020200000000000003220EF008308220092
:10410000008041001040BA000160EF00000006008E
:1041100020460000696E0000646900006E670000C0
:1041200020430000616D00006572000061730000B3
:10413000000000003220EF00630A220000804100EE
:104140001040BA000160EF000000060020430000AC
:104150006C65000061720000696E0000672000005D
:104160005072000065730000657400007300000069
:104170003220EF00430C2200008041001040BA00C2
:104180000160EF0000000600204300006C650000A5
:1041900061720000696E000067200000416C000041
:1041A0006C20000020200000000000003220EF0002
:1041B000230E2200008041001040BA000160EF0091
:1041C00000000600205200006573000074610000CA
:1041D00072740000205300007973000074650000C1
:1041E0006D200000000000003220EF0003102200CC
:1041F000008041001040BA000160EF00000006009E
:10420000202000004E6F0000742000006F6E000040
:1042100020500000726500007365000074200000EB
:10422000000000003220EF00E31122000080410076
:104230001040BA000160EF0000000600456E00006B
:10424000616200006C650000204800006F73000090
:10425000742000005365000072690000616C00006A
:10426000000000003220EF00E31322000080410034
:104270001040BA000160EF00000006004469000031
:1042800073610000626C000065200000536500004F
:1042900072690000616C00002020000020200000F6
:1042A000000000003220EF00E315220000804100F2
:1042B0001040BA000160EF00000006000A0D000087
:1042C000436F00006D6D0000616E0000642000000F
:1042D000436F00006D7000006C65000074650000A5
:1042E0000A0D00003E0000003220EF0003182200FB
:1042F000008041001040BA000160EF00000006009D
:10430000202000005368000075740000646F0000F6
:10431000776E0000204100006374000069760000A1
:1043200065200000000000003220EF00031A220088
:10433000008041001040BA000160EF00000006005C
:1043400020430000616D00006572000061200000E4
:10435000506F000077650000726400006F77000006
:104360006E200000000000003220EF004302200019
:104370008301500005003100031D22000080410030
:104380001040BA000160EF0000000600001D22008E
:1043900083814100808141001380BA000000060043
:1043A0000A0D6700536320006865250064753400BA
:1043B0006C654C0042757800747420006F6E430089
:1043C00028296F0020257000327879002F252000E1
:1043D0003278250020533100746178007475000034
:1043E000734600006C6100003220EF0003202200C1
:1043F000008041001040BA000160EF00000006009C
:10440000536500006172000063680000696E00007F
:1044100067200000666F00007220000041740000F9
:1044200074610000636800006564000020430000C0
:10443000616D000065720000617300000D0A0000EC
:10444000000000003220EF00E32222000080410043
:104450001040BA000160EF0000000600506F00003D
:104460007274000020250000643A00000A0D00006C
:10447000000000003220EF00632422000080410091
:104480001040BA000160EF00000006004361000028
:104490006D6500007261000073200000466F00002F
:1044A000756E000064200000256400000A0D000005
:1044B000000000003220EF0063262200008041004F
:1044C0001040BA000160EF0000000600506F0000CD
:1044D0007274000020250000643A000020430000B0
:1044E000616D00006572000061200000256400001D
:1044F0000A0D0000000000003220EF008328220097
:10450000008041001040BA000160EF00000006008A
:10451000436100006D6500007261000020530000DF
:10452000656100007263000068200000436F0000B6
:104530006D7000006C650000746500000A0D0000DD
:104540000A0000003220EF00E32A22000080410030
:104550001040BA000160EF0000000600204E00008D
:104560006F200000436100006D200000202000004B
:10457000205000006F720000742000003020000006
:10458000200000003220EF00E32C220000804100D8
:104590001040BA000160EF00000006000D0A0000A4
:1045A000506100006E610000736F00006E690000D2
:1045B00063200000415700002D48000045310000F5
:1045C000303000000D0A0000000000003220EF0033
:1045D000232F2200008041001040BA000160EF004C
:1045E0000000060020410000572D00004845000053
:1045F0003130000030200000205000006F720000B9
:104600007420000030200000200000003220EF0065
:1046100023312200008041001040BA000160EF0009
:1046200000000600204700006574000038200000EC
:10463000000000003220EF006332220000804100C1
:104640001040BA000160EF000000060020200000CA
:10465000202D00002D2000002532000058200000F1
:104660002D2D00000A0D0000000000003220EF0098
:1046700023342200008041001040BA000160EF00A6
:10468000000006000A0D0000202000002067000046
:104690006574000031360000200000003220EF0079
:1046A000A3352200008041001040BA000160EF00F5
:1046B0000000060020200000202D00002D2000001A
:1046C000254C0000582000002D2D0000200A00007D
:1046D0000D0000003220EF0063372200008041000F
:1046E0001040BA000160EF00000006000A0D000053
:1046F00020200000206700006574000033320000B5
:10470000200000003220EF00E3382200008041004A
:104710001040BA000160EF000000060020200000F9
:10472000202D00002D200000254C00005820000006
:104730002D2D00000A0D0000000000003220EF00C7
:10474000A33A2200008041001040BA000160EF004F
:10475000000006000A0D000020430000616D00000B
:10476000657200006154000079700000652000004F
:104770002D200000000000003220EF00833C2200CA
:10478000008041001040BA000160EF000000060008
:10479000536F00006E79000020450000564900006C
:1047A0002D4400003330000028720000290D000065
:1047B0000A0000003220EF00633E2200008041002A
:1047C0001040BA000160EF00000006002045000024
:1047D000564900002D4400003330000028720000CC
:1047E000295000006F72000074200000302000008B
:1047F000200000003220EF006340220000804100D2
:104800001040BA000160EF0000000600496E000091
:10481000766100006C6900006420000043610000C4
:104820006D650000726100000D0A000000000000CC
:104830003220EF0043422200008041001040BA00C5
:104840000160EF0000000600204900006E760000C5
:10485000616C00006964000020430000616D00008D
:1048600065720000610000003220EF000344220066
:10487000008041001040BA000160EF000000060017
:104880000D0A0000536F00006E7900002045000003
:10489000564900002D440000333000002F33000043
:1048A000312000000D0A0000000000003220EF005F
:1048B00023462200008041001040BA000160EF0052
:1048C0000000060020450000564900002D4400006D
:1048D000333000002F330000315000006F720000B1
:1048E0007420000030200000200000003220EF0083
:1048F00023482200008041001040BA000160EF0010
:10490000000006000D0A0000536F00006E790000E1
:1049100020450000564900002D44000033300000BF
:104920000D0A0000000000003220EF00034A2200C0
:10493000008041001040BA000160EF000000060056
:1049400020450000564900002D440000333000008F
:1049500020200000205000006F7200007420000032
:1049600030200000200000003220EF00034C220025
:10497000008041001040BA000160EF000000060016
:104980000D0A00005661000064640000696F0000B9
:1049900020410000646400002D4100002D43000010
:1049A000616D00000D0A0000000000003220EF00E1
:1049B000234E2200008041001040BA000160EF0049
:1049C0000000060020410000646400002D4100004A
:1049D0002D430000616D0000205000006F72000048
:1049E0007420000030200000200000003220EF0082
:1049F00023502200008041001040BA000160EF0007
:104A0000000006000D0A0000536F00006E790000E0
:104A100020450000564900002D44000031300000C0
:104A2000300D00000A0000003220EF000352220087
:104A3000008041001040BA000160EF000000060055
:104A400020450000564900002D4400003130000090
:104A500030200000205000006F7200007420000021
:104A600030200000200000003220EF00035422001C
:104A7000008041001040BA000160EF000000060015
:104A80000D0A0000536F00006E7900002045000001
:104A9000564900002D440000373000000D0A000088
:104AA000000000003220EF00E355220000804100AA
:104AB0001040BA000160EF00000006002045000031
:104AC000564900002D44000037300000202000002F
:104AD000205000006F7200007420000030200000A1
:104AE000200000003220EF00E35722000080410048
:104AF0001040BA000160EF00000006000D0A00003F
:104B0000536F00006E790000204200005243000005
:104B1000482D000037300000300D00000A00000072
:104B20003220EF00C3592200008041001040BA003B
:104B30000160EF0000000600204200005243000028
:104B4000482D0000373000003020000020500000C9
:104B50006F72000074200000302000002000000070
:104B60003220EF00C35B2200008041001040BA00F9
:104B70000160EF00000006000D0A0000456C000017
:104B80006D6F000020430000616D00006572000041
:104B9000610D00000A0000003220EF00835D22005A
:104BA000008041001040BA000160EF0000000600E4
:104BB000204500006C6D00006F20000020200000E8
:104BC00020200000205000006F72000074200000C0
:104BD00030200000200000003220EF00835F220020
:104BE000008041001040BA000160EF0000000600A4
:104BF0000D0A0000536F00006E7900002042000093
:104C0000524300002D330000303000000D0A000038
:104C1000000000003220EF006361220000804100AC
:104C20001040BA000160EF000000060020420000C2
:104C3000524300002D3300003030000020200000DF
:104C4000205000006F72000074200000302000002F
:104C5000200000003220EF0063632200008041004A
:104C60001040BA000160EF00000006000D0A0000CD
:104C7000536F00006E790000204200005243000094
:104C80002D5A000037300000300D00000A000000EF
:104C90003220EF0043652200008041001040BA003E
:104CA0000160EF00000006002042000052430000B7
:104CB0002D5A000037300000302000002050000046
:104CC0006F720000742000003020000020000000FF
:104CD0003220EF0043672200008041001040BA00FC
:104CE0000160EF00000006000D0A0000536F000095
:104CF0006E79000020420000524300002D5A00004F
:104D000033330000300D00000A0000003220EF00B5
:104D100023692200008041001040BA000160EF00CA
:104D20000000060020420000524300002D5A0000FF
:104D30003333000030200000205000006F7200006C
:104D40007420000030200000200000003220EF001E
:104D5000236B2200008041001040BA000160EF0088
:104D6000000006000D0A0000564100004444000007
:104D7000494F000020480000442D00003138000059
:104D80000D0A0000000000003220EF00036D220039
:104D9000008041001040BA000160EF0000000600F2
:104DA0005641000044440000494F000020480000E4
:104DB0004431000038200000506F00007274000081
:104DC00020300000000000003220EF00036F2200BE
:104DD000008041001040BA000160EF0000000600B2
:104DE0000D0A0000536F00006E790000204500009E
:104DF000564900002D480000443100000D0A000013
:104E0000000000003220EF00E3702200008041002B
:104E10001040BA000160EF000000060020450000CD
:104E2000564900002D4800004431000020200000B9
:104E3000205000006F72000074200000302000003D
:104E4000200000003220EF00E372220000804100C9
:104E50001040BA000160EF00000006000D0A0000DB
:104E60005661000064640000696F00002043000088
:104E7000656900006C6900006E670000564900001B
:104E8000455700000D0A0000000000003220EF002E
:104E900023752200008041001040BA000160EF003D
:104EA0000000060020430000562F0000435600007B
:104EB0004D50000020200000205000006F720000C4
:104EC0007420000030200000200000003220EF009D
:104ED00023772200008041001040BA000160EF00FB
:104EE00000000600556E00006B6E00006F7700003A
:104EF0006E200000436100006D65000072610000DB
:104F00000D0A0000000000003220EF0003792200AB
:104F1000008041001040BA000160EF000000060070
:104F2000205500006E6B00006E6F0000776E000071
:104F300020200000205000006F720000742000004C
:104F400030200000200000003220EF00037B220010
:104F5000008041001040BA000160EF000000060030
:104F60000A0D000020410000542F00004D440000B5
:104F70005F4D00006F640000654900006E71000025
:104F8000200000003220EF00E37C2200008041007E
:104F90001040BA000160EF00000006000D0A00009A
:104FA0005761000069740000536F00006E790000C3
:104FB000496E00007152000065730000702000000F
:104FC000000000003220EF00E37E2200008041005C
:104FD0001040BA000160EF00000006000D0A00005A
:104FE0002057000061690000745300006F6E0000DC
:104FF00079410000636B0000000000003220EF00E8
:10500000A3802200008041001040BA000160EF0040
:10501000000006000D0A0000205700006169000032
:10502000745300006F6E0000790000003220EF0022
:1050300023822200008041001040BA000160EF008E
:10504000000006002A570000616900007453000048
:105050006F6E0000790000003220EF008383220091
:10506000008041001040BA000160EF00000006001F
:105070000D0A000020570000616900007452000012
:1050800065730000705300006F6E0000790000002F
:105090003220EF0043852200008041001040BA001A
:1050A0000160EF0000000600202D000020540000E9
:1050B000696D0000656F0000757400002025000018
:1050C00075200000286D0000732900000D0A000003
:1050D000000000003220EF006387220000804100C2
:1050E0001040BA000160EF000000060043610000BC
:1050F0006E630000656C000020530000312000004A
:10510000000000003220EF00E38822000080410010
:105110001040BA000160EF0000000600436100008B
:105120006E630000656C0000205300003220000018
:10513000000000003220EF00638A2200008041005E
:105140001040BA000160EF00000006000A0D0000E8
:10515000202000002047000065740000425200003B
:1051600043500000616E0000546900006C74000040
:10517000506F000073200000000000003220EF009C
:10518000A38C2200008041001040BA000160EF00B3
:105190000000060020200000202D00002D2000002F
:1051A000503A0000254C0000582C0000543A0000F2
:1051B000254C0000582000002D2D00000A0D000095
:1051C000000000003220EF00E38E2200008041004A
:1051D0001040BA000160EF00000006000A0D000058
:1051E00020430000616D0000657200006154000002
:1051F0007970000065200000000000003220EF0000
:10520000A3902200008041001040BA000160EF002E
:10521000000006000A0D0000205000006F7700001B
:1052200065720000204F00006E20000052650000F3
:105230007472000079200000000000003220EF00AE
:10524000A3922200008041001040BA000160EF00EC
:10525000000006000A0D000020430000616D000000
:105260006572000061540000797000006520000044
:1052700056310000200000003220EF00839422000D
:10528000008041001040BA000160EF0000000600FD
:10529000436100006E6F00006E2000004255000068
:1052A0002D340000354800000D0A00000000000009
:1052B0003220EF0043962200008041001040BA00E7
:1052C0000160EF000000060020420000552D0000A4
:1052D000343500004820000020200000205000004D
:1052E0006F720000742000003020000020000000D9
:1052F0003220EF0043982200008041001040BA00A5
:105300000160EF0000000600436100006E6F0000C6
:105310006E200000425500002D350000304800008E
:105320000D0A0000000000003220EF00039A220066
:10533000008041001040BA000160EF00000006004C
:1053400020420000552D00003530000048200000AC
:1053500020200000205000006F7200007420000028
:1053600030200000200000003220EF00039C2200CB
:10537000008041001040BA000160EF00000006000C
:10538000436100006E6F00006E2000005643000075
:105390002D43000035300000490D00000A000000D8
:1053A0003220EF00C39D2200008041001040BA006F
:1053B0000160EF000000060020560000432D0000B1
:1053C000433500003069000020200000205000001C
:1053D0006F720000742000003020000020000000E8
:1053E0003220EF00C39F2200008041001040BA002D
:1053F0000160EF0000000600205D00000A0D0000C3
:10540000000000003220EF00E3A0220000804100F5
:105410001040BA000160EF00000006000D0A000015
:10542000205700006169000074430000616E0000B5
:105430006F6E0000000000003220EF0083A2220007
:10544000008041001040BA000160EF00000006003B
:105450000D0A00002057000061690000744300003D
:10546000616E00006F6E00004E6F0000744200001D
:1054700075730000790000003220EF0083A4220041
:10548000008041001040BA000160EF0000000600FB
:105490000D0A0000205700006169000074430000FD
:1054A000616E00006F6E0000505400005A530000FF
:1054B000746F0000700000003220EF0083A622000D
:1054C000008041001040BA000160EF0000000600BB
:1054D000202D000020540000696D0000656F000061
:1054E00075740000202500006C7500002028000065
:1054F0006D730000290D00000A0000003220EF004B
:10550000A3A82200008041001040BA000160EF0013
:10551000000006000D0A000020570000616900002D
:1055200074500000616E0000617300006F6E000037
:1055300069630000000000003220EF0083AA22000F
:10554000008041001040BA000160EF00000006003A
:105550000A0D00005531000028450000727200005D
:10556000292000005B4C0000535200005D25000024
:1055700032780000000000003220EF0083AC2200EF
:10558000008041001040BA000160EF0000000600FA
:105590000A0D00005532000028450000727200001C
:1055A000292000005B4C0000535200005D250000E4
:1055B00032780000000000003220EF0083AE2200AD
:1055C000008041001040BA000160EF0000000600BA
:1055D0000A0D0000584F00004E20000053650000E7
:1055E0006E740000205800004F4600004620000066
:1055F0005374000061740000652000003100000059
:105600003220EF00C3B02200008041001040BA00F9
:105610000160EF00000006000A0D0000584F000076
:105620004E200000536500006E74000020580000FA
:105630004F460000462000005374000061740000D3
:1056400065200000320000003220EF0003B322008A
:10565000008041001040BA000160EF000000060029
:105660000A0D0000536C00006176000065490000DF
:105670006E70000075740000282500006429000089
:10568000204D000061730000746500007249000045
:105690006E70000075740000282500006429000069
:1056A000000000003220EF00E3B52200008041003E
:1056B0001040BA000160EF00000006000A0D000073
:1056C000584F00004E200000536500006E7400002B
:1056D00020490000646C0000652000005374000045
:1056E00061740000650000003220EF0003B8220062
:1056F000008041001040BA000160EF000000060089
:105700000A0D0000507200006F6300006573000016
:10571000735300006C6100007665000028290000CA
:105720002062000061640000205300004F4D000023
:105730003D25000032780000000000003220EF001C
:10574000A3BA2200008041001040BA000160EF00BF
:10575000000006000A0D0000507200006F63000098
:1057600065730000734D00006173000074650000F4
:1057700072280000292000006261000064200000FF
:10578000534F00004D3D000025320000780000001E
:105790003220EF0043BD2200008041001040BA00DB
:1057A0000160EF00000006000A0D000043680000E1
:1057B0006B4600006F63000075730000456E0000CB
:1057C000636F00006465000072280000253000004F
:1057D000344C000078290000000000003220EF0067
:1057E000A3BF2200008041001040BA000160EF001A
:1057F0000000060020200000466F000063750000D6
:10580000732000004E65000061720000202500003A
:105810006C750000000000003220EF0083C1220000
:10582000008041001040BA000160EF000000060057
:1058300020200000466F0000637500007320000008
:105840004661000072200000256C00007500000019
:105850003220EF0043C32200008041001040BA0014
:105860000160EF00000006000A0D00004368000020
:105870006B49000072690000734500006E63000010
:105880006F640000657200002825000030340000BD
:105890004C780000290000003220EF0083C5220070
:1058A000008041001040BA000160EF0000000600D7
:1058B0000A0D0000436800006B5A00006F6F000083
:1058C0006D4500006E6300006F64000065720000AB
:1058D00028250000303400004C780000290000002A
:1058E0003220EF00C3C72200008041001040BA0000
:1058F0000160EF00000006000A0D00004368000090
:105900006B500000616E0000456E0000636F000088
:10591000646500007228000025300000344C00004F
:1059200078290000000000003220EF0003CA2200A6
:10593000008041001040BA000160EF000000060046
:105940000A0D0000436800006B540000696C000001
:10595000744500006E6300006F6400006572000013
:1059600028250000303400004C7800002900000099
:105970003220EF0043CC2200008041001040BA00EA
:105980000160EF00000006000A0D000043680000FF
:105990006B52000065640000456E0000636F0000FC
:1059A000646500007228000025300000344C0000BF
:1059B00078290000000000003220EF0083CE220092
:1059C000008041001040BA000160EF0000000600B6
:1059D0000A0D0000436800006B4200006C75000077
:1059E000654500006E6300006F6400006572000092
:1059F00028250000303400004C7800002900000009
:105A00003220EF00C3D02200008041001040BA00D5
:105A10000160EF00000006000A0D0000436800006E
:105A20006B44000065740000616900006C45000073
:105A30006E6300006F64000065720000282500009E
:105A4000303400004C780000290000003220EF00C4
:105A500023D32200008041001040BA000160EF0013
:105A6000000006000A0D0000436800006B470000BC
:105A7000616900006E4500006E6300006F64000005
:105A80006572000028250000303400004C780000CA
:105A9000290000003220EF0063D522000080410081
:105AA0001040BA000160EF00000006002020000056
:105AB0002020000047610000696E0000204E0000B9
:105AC0002F41000020200000200000003220EF00C5
:105AD00023D72200008041001040BA000160EF008F
:105AE000000006000A0D0000203E0000000000003B
:105AF0003220EF0043D82200008041001040BA005D
:105B00000160EF00000006003E2500007320000049
:105B10004E6F000074200000466F0000756E00009C
:105B2000640A00000D3E0000000000003220EF007B
:105B300023DA2200008041001040BA000160EF002B
:105B4000000006000A2500007325000073200000F5
:105B500020200000200000003220EF0083DB220024
:105B6000008041001040BA000160EF000000060014
:105B7000436F00006D700000696C000065640000F8
:105B80003A2000002573000020610000742000000E
:105B9000257300000A0D0000000000003220EF0015
:105BA000E30220008301500005003100A3DE220043
:105BB000008041001040BA000160EF0000000600C4
:105BC000A0DE220083814100808141001380BA0061
:105BD000000006000D0A2000537920007374440071
:105BE000656D650020536600657461007469750019
:105BF0006E676C00733A74000A0D20000A0D5000A5
:105C00004465720066616500756C73007420650000
:105C1000436174006D653A00726120003A202500EE
:105C20002564640020200A0020200D0020200000B0
:105C30003220EF0043E22200008041001040BA0011
:105C40000160EF000000060054720000616E000069
:105C500073690000746900006F6E0000205400003A
:105C6000696D0000653A000020250000640A00000C
:105C70000D0000003220EF0043032000830150009C
:105C80000500310063E52200008041001040BA00A9
:105C90000160EF000000060060E522008381410002
:105CA000808141001380BA00000006000A0D3A000E
:105CB000436120006D65200072613100205020009A
:105CC0006F72200074203200536520006172200042
:105CD000636833003A202000203120002020340067
:105CE00032202000203320002020350034202000E6
:105CF00020352000202036003620200020372000CC
:105D00002020370043430A0055200D004D6F00004E
:105D1000646500003220EF0063E92200008041004A
:105D20001040BA000160EF000000060020200000D3
:105D30002020000020200000202000002020000063
:105D40002020000020200000202000002020000053
:105D500020200000000000003220EF0083EB220032
:105D6000008041001040BA000160EF000000060012
:105D70002020000020200000202000002020000023
:105D800020200000200000003220EF00430220000D
:105D9000830150000500310003EE22000080410025
:105DA0001040BA000160EF000000060000EE220083
:105DB00083814100808141001380BA000000060009
:105DC0000A0D2000506150006E53610070656E0036
:105DD0006564650020206C002020200054694C0080
:105DE0006C74690053706700656568006420740016
:105DF000202073005A6F0A006F6D0D005370000071
:105E000065650000642000003220EF0003022000DE
:105E1000830150000500310003F2220000804100A0
:105E20001040BA000160EF000000060000F22200FE
:105E300083814100808141001380BA000000060088
:105E40002020200020252000642020002020200089
:105E500020202000202020002020200020202000C2
:105E6000256425002020640020200A0020200D0049
:105E700020200A0020200D002564000020200000C2
:105E80003220EF00C3F42200008041001040BA002D
:105E90000160EF00000006004A6F00007973000007
:105EA00074690000636B00002053000065740000FB
:105EB000757000003A0A00000D0000003220EF006B
:105EC000230320008301500005003100A3F72200C6
:105ED000008041001040BA000160EF0000000600A1
:105EE000A0F7220083814100808141001380BA0025
:105EF000000006000A0D3A0020502000616E2000CC
:105F0000205031006F72200074202000446932005C
:105F10007265200063742000696F33006E3A2000C0
:105F200020202000312034002032200020202000BA
:105F3000332035002034200020202000352036007A
:105F400020362000202020003720370020530A0070
:105F500070650D00656400003220EF0083FB2200B5
:105F6000008041001040BA000160EF000000060010
:105F70002020000020200000202000002020000021
:105F80002020000020200000202000002020000011
:105F90002020000020200000200000003220EF0020
:105FA000A3FD2200008041001040BA000160EF0014
:105FB000000006002020000020200000202000001B
:105FC00020200000000000003220EF00230320000A
:105FD00083015000050031000300230000804100D0
:105FE0001040BA000160EF0000000600000023002E
:105FF00083814100808141001380BA0000000600C7
:106000000D0A3A00546920006C74200020503100C1
:106010006F722000742020004469320072652000F5
:1060200063742000696F33006E3A20002020200046
:106030003120340020322000202020003320350081
:10604000203420002020200035203600203620007B
:10605000202020003720370020530A0070650D00F3
:10606000656400003220EF0023032000830150000C
:1060700005003100E3042300008041001040BA0015
:106080000160EF0000000600E0042300838141006E
:10609000808141001380BA00000006000D0A3A001A
:1060A0005A6F20006F6D2000205031006F72200069
:1060B000742020004469320072652000637420005F
:1060C000696F33006E3A2000202020003120340018
:1060D00020322000202020003320350020342000F2
:1060E00020202000352036002036200020202000EF
:1060F0003720370020530A0070650D0065640000EA
:106100003220EF00C3082300008041001040BA0095
:106110000160EF00000006000D0A00004E6500005F
:1061200075740000726100006C2000005A6F00005E
:106130006E6500003A200000506100006E200000F3
:10614000546900006C740000205A00006F6F00005A
:106150006D0A00000D0000003220EF00830B2300C9
:10616000008041001040BA000160EF00000006000E
:10617000202000002020000020200000202000001F
:10618000202000002020000020200000202500000A
:10619000326400002020000025320000642000004E
:1061A0002020000025320000640000003220EF00B3
:1061B000230E2300008041001040BA000160EF0070
:1061C000000006000A0D0000507200006573000018
:1061D00065740000733A00000A0D00000A0D00000B
:1061E000000000003220EF00230320008301500054
:1061F00005003100E3102300008041001040BA0088
:106200000160EF0000000600E010230083814100E0
:10621000808141001380BA000000060043617300D2
:106220006D20200050722000652047004D6F6100F6
:10623000646569006C206E00202020002020200072
:106240002020520020506500616E64002020200054
:106250002020200020542000696C420074206C0033
:10626000205A75006F6F65006D20200020464400A5
:106270006F6365007573740020492E007269000019
:106280003220EF00C3142300008041001040BA0008
:106290000160EF0000000600205B00004972000072
:1062A000697300002C4600006F63000075730000E6
:1062B0002C410000574200002C200000424C0000FE
:1062C000435D00000A0D00000A0D00000000000000
:1062D0003220EF00E302200083015000050031006E
:1062E00043182300008041001040BA000160EF0015
:1062F0000000060040182300838141008081410096
:106300001380BA0000000600202520006420200031
:106310002025250032644C00202058002531200023
:10632000327320002025250058254C0058255800A0
:1063300058202000202520004C5825002020320025
:10634000254C4C0058205800202520004C58200097
:1063500020202000254C200058200000202500008F
:106360004C5800003220EF00E31B23000080410066
:106370001040BA000160EF00000006004F6E000000
:1063800020200000200000003220EF00031D230029
:10639000008041001040BA000160EF0000000600DC
:1063A0004F66000066200000200000003220EF0051
:1063B000231E2300008041001040BA000160EF005E
:1063C000000006000A0D0000436100006D2000007F
:1063D0004D6F0000646500006C0A00000D000000B5
:1063E0003220EF00C31F2300008041001040BA009C
:1063F0000160EF000000060020250000642000007E
:10640000204E00006F200000436100006D65000019
:10641000726100000A0D0000000000003220EF0051
:10642000A3212300008041001040BA000160EF006A
:106430000000060045450000507200006F6D00002E
:1064400020440000756D0000703A00000A0D000045
:10645000000000003220EF00632323000080410091
:106460001040BA000160EF00000006004545000042
:10647000507200006F6D0000204300006F6E00003E
:106480006669000067200000447500006D70000020
:106490003A0A00000D0000003220EF00832523009F
:1064A000008041001040BA000160EF0000000600CB
:1064B00045450000507200006F6D00002050000044
:1064C00072650000736500007420000044750000D0
:1064D0006D7000003A0A00000D0000003220EF004D
:1064E000A3272300008041001040BA000160EF00A4
:1064F0000000060045450000507200006F6D00006E
:106500002048000069670000682000004475000012
:106510006D7000003A0A00000D0000003220EF000C
:10652000A3292300008041001040BA000160EF0061
:106530000000060020200000202000002020000095
:10654000000000003220EF00E32A23000080410019
:106550001040BA000160EF00000006000A0D0000C4
:106560003E20000041570000423D00004F6E0000F9
:106570000A0D00003E200000000000003220EF0065
:10658000A32C2300008041001040BA000160EF00FE
:10659000000006000A0D00003E20000041570000E8
:1065A000423D00004F660000660A00000D3E0000FC
:1065B000200000003220EF00632E23000080410005
:1065C0001040BA000160EF00000006000A0D000054
:1065D0003E200000424C0000433D00004F6E000092
:1065E0000A0D00003E200000000000003220EF00F5
:1065F00023302300008041001040BA000160EF000A
:10660000000006000A0D00003E200000424C000081
:10661000433D00004F660000660A00000D3E00008A
:10662000200000003220EF00E33123000080410011
:106630001040BA000160EF00000006000A0D0000E3
:106640000A0D0000204900006E760000616C000019
:10665000696400002049000032630000204100000E
:10666000646400007265000073730000202800005D
:1066700025730000290A00000D0000003220EF0001
:10668000A3342300008041001040BA000160EF00F5
:10669000000006000A0D00000A0D0000204900005D
:1066A0006E760000616C0000696400002049000003
:1066B000326300002052000065670000697300002B
:1066C0007465000072200000282500007329000076
:1066D0000A0D0000000000003220EF0043022000FD
:1066E0008301500005003100833823000080410001
:1066F0001040BA000160EF0000000600803823005F
:1067000083814100808141001380BA0000000600AF
:106710000A0D58000A0D20005265520061646500A0
:10672000204973003243700020416F0064646E00A2
:1067300072657300737365003D253D003258250076
:10674000205232006567580069730A0074650D00B5
:10675000723D0000253200003220EF0003022000CD
:106760008301500005003100833C2300008041007C
:106770001040BA000160EF0000000600803C2300DA
:1067800083814100808141001380BA00000006002F
:106790000A0D32000A0D580057722C00697444002B
:1067A00065206100416474006472610065733D009E
:1067B000733D250025323200582C580052652000C8
:1067C00067690A0073740D00657200003D250000C2
:1067D0003220EF00433F2300008041001040BA0008
:1067E0000160EF00000006000A0D000020450000D7
:1067F000727200006F7200002D20000043610000E3
:106800006D65000072610000204E00006F74000092
:1068100020530000656C0000656300007465000093
:10682000640D00000A3E0000200000003220EF004E
:1068300023422300008041001040BA000160EF00B5
:10684000000006000A0D000045720000726F000093
:10685000722D0000204900007269000073200000C2
:10686000696E000020410000757400006F20000078
:106870004D6F0000646500000A0D0000000000007C
:106880003220EF00C3442300008041001040BA00D2
:106890000160EF00000006002020000020490000F9
:1068A0007269000073200000436F00006D6D0000EE
:1068B000616E000064200000466F0000726D0000F1
:1068C000617400000A0D0000000000003220EF009B
:1068D00023472300008041001040BA000160EF0010
:1068E000000006002020000020490000726900001E
:1068F0007320000041750000746F000028630000E1
:10690000722900002C200000497200006973000009
:10691000204D0000616E0000756100006C280000D1
:1069200063720000290A00000D0000003220EF0011
:10693000234A2300008041001040BA000160EF00AC
:1069400000000600202000002049000072690000BD
:1069500073200000557000002C34000028630000F4
:10696000722900002C2000004972000069730000A9
:10697000204400006F7700006E2C000030340000CF
:1069800028630000722900000A0D000000000000CA
:106990003220EF00434D2300008041001040BA0038
:1069A0000160EF00000006000A0D00003E2000001C
:1069B00044690000616700003D4F00006E0A00005E
:1069C0000D3E0000200000003220EF00034F2300A6
:1069D000008041001040BA000160EF000000060096
:1069E0000A0D00003E2000004469000061670000BD
:1069F0003D4F0000666600000A0D00003E200000CA
:106A0000000000003220EF00E3502300008041002E
:106A10001040BA000160EF00000006003E200000B8
:106A2000257300002042000075740000746F0000A0
:106A30006E20000025730000204300006C650000FC
:106A400061720000656400000D0A00003E20000035
:106A5000000000003220EF004302200083015000BC
:106A60000500310063542300008041001040BA004B
:106A70000160EF00000006006054230083814100A4
:106A8000808141001380BA00000006003E206400AF
:106A90002573200020456C00727265006F726E00D5
:106AA0002C20670025737400204268007574200054
:106AB000746F25006E20750073742E0072690D00CE
:106AC0006E670A002C203E00696E2000766100008F
:106AD0006C6900003220EF00E301200083015000C8
:106AE0000500310063582300008041001040BA00C7
:106AF0000160EF0000000600605823008381410020
:106B0000808141001380BA00000006003E20700022
:106B10002573720020456F00727276006F726900F3
:106B20002C20640042756500747464006F6E0D0063
:106B300020730A0074723E00696E20006720000016
:106B40006E6F0000742000003220EF00630220000E
:106B50008301500005003100035C230000804100E8
:106B60001040BA000160EF0000000600005C230046
:106B700083814100808141001380BA00000006003B
:106B80003E2065002573650020456E00727220006E
:106B90006F7231002C2020004275610074746E0009
:106BA0006F6E6400206E2000756D310062653400E8
:106BB00072202E0025780D002C200A006E6F3E00FA
:106BC0007420200062650000747700003220EF001E
:106BD000E301200083015000050031002360230001
:106BE000008041001040BA000160EF000000060084
:106BF0002060230083814100808141001380BA001E
:106C0000000006003E2070002573720020456F00D2
:106C1000727276006F7269002C2064004275650004
:106C2000747464006F6E2E00206E0D00756D0A0086
:106C300062653E00722020006E6F0000742000002C
:106C40003220EF00C3622300008041001040BA00F0
:106C50000160EF00000006000A0D00003E20000069
:106C6000506F000077650000723D00004F6E00001D
:106C70000A0D00003E200000000000003220EF005E
:106C8000A3642300008041001040BA000160EF00BF
:106C9000000006000A0D00003E200000506F0000BA
:106CA00077650000723D00004F660000660A000034
:106CB0000D3E0000200000003220EF00836623001C
:106CC000008041001040BA000160EF0000000600A3
:106CD0000A0D00003E2000005344000069610000DE
:106CE000673D00004F6E00000A0D00003E200000CE
:106CF000000000003220EF006368230000804100A4
:106D00001040BA000160EF00000006000A0D00000C
:106D10003E2000005344000069610000673D000010
:106D20004F660000660A00000D3E000020000000D3
:106D30003220EF00230220008301500005003100C3
:106D4000436B2300008041001040BA000160EF0057
:106D500000000600406B23008381410080814100D8
:106D60001380BA00000006000A0D61003E20690091
:106D70004A53740044375400302069002D206D00C0
:106D80004A6F65007973280074692500636B75008C
:106D9000205329006C6F0A0077200D0044373E0015
:106DA000302020004F6E00002C5700003220EF00F2
:106DB000230220008301500005003100236F2300CF
:106DC000008041001040BA000160EF0000000600A2
:106DD000206F230083814100808141001380BA002D
:106DE000000006000A0D57003E2061004A5369006A
:106DF00044377400302054002D2069004A6F6D0024
:106E00007973650074692800636B25002053750051
:106E10006C6F290077200A0044370D0030203E00B7
:106E20004F662000662C00003220EF000372230022
:106E3000008041001040BA000160EF000000060031
:106E40000A0D00003E200000546100006C6C000040
:106E5000793D000041630000746900007665000020
:106E60002048000069670000680A00000D3E00002D
:106E7000200000003220EF006374230000804100F6
:106E80001040BA000160EF00000006000A0D00008B
:106E90003E200000546100006C6C0000793D000051
:106EA000416300007469000076650000204C00001A
:106EB0006F7700000A0D00003E2000000000000077
:106EC0003220EF00C3762300008041001040BA005A
:106ED0000160EF000000060045720000726F0000C4
:106EE000722D0000204600006F63000075730000E3
:106EF000206900006E20000041750000746F0000E2
:106F0000204D00006F640000650A00000D000000C5
:106F10003220EF0043792300008041001040BA0086
:106F20000160EF0000000600202000002046000065
:106F30006F63000075730000204300006F6D000058
:106F40006D6100006E640000204600006F7200005A
:106F50006D610000740A00000D0000003220EF0097
:106F6000A37B2300008041001040BA000160EF00C5
:106F70000000060020200000204600006F63000093
:106F80007573000020410000757400006F28000038
:106F900063720000292C0000202000002046000021
:106FA0006F63000075730000204D0000616E0000EB
:106FB000756100006C28000063720000290A00005F
:106FC0000D0000003220EF00E37E2300008041002E
:106FD0001040BA000160EF00000006002020000011
:106FE000204600006F63000075730000205500000C
:106FF000702C00003428000063720000292C00006F
:1070000020200000204600006F6300007573000020
:10701000204400006F7700006E2C00003428000030
:1070200063720000290A00000D0000003220EF000A
:10703000C301200083015000050031002383230099
:10704000008041001040BA000160EF00000006001F
:107050002083230083814100808141001380BA0096
:107060000000060020206F00204677006F636E004E
:1070700075732C0020553000702C61003061300099
:107080003028280063726300292C720020462900F2
:107090006F630A0075730D00204400003220EF007A
:1070A000A3852300008041001040BA000160EF007A
:1070B0000000060020200000204600006F63000052
:1070C0007573000020250000750000003220EF00DD
:1070D00023872300008041001040BA000160EF00C8
:1070E000000006000A0D00003E2000004361000081
:1070F0006D65000072610000202500006420000022
:107100004E6F00007420000061760000616900008D
:107110006C610000626C0000650A00000D3E00001A
:10712000200000003220EF00E389230000804100AE
:107130001040BA000160EF00000006000A0D0000D8
:107140003E2000004A500000616E000053700000B5
:10715000643A0000205000006F72000074200000AC
:1071600020310000202000003220000020330000E9
:1071700020200000342000002035000020200000E6
:1071800036200000203700000A0D0000000000003B
:107190003220EF000302200083015000050031007F
:1071A000438E2300008041001040BA000160EF00D0
:1071B00000000600408E2300838141008081410051
:1071C0001380BA0000000600202025002020320095
:1071D00020206400202020002020250020203200D4
:1071E0002020640020202000253225006420320069
:1071F0002532640064200A0025320D0064203E0020
:1072000025320000642000003220EF0003912300AB
:10721000008041001040BA000160EF00000006004D
:107220000D0A00003E4A0000506100006E4400005C
:1072300069720000202000004469000072650000AF
:1072400063740000696F00006E3A00002031000096
:1072500020320000203300002034000020350000E0
:1072600020360000203700000A0D0000000000005A
:107270003220EF00E30120008301500005003100BF
:1072800043952300008041001040BA000160EF00E8
:107290000000060040952300838141008081410069
:1072A0001380BA0000000600202025002020630083
:1072B0002020200020202500202063002020200006
:1072C00020202500202063002020200020202500F1
:1072D0002025630063200A0025630D0020253E0061
:1072E000632000003220EF00E3972300008041007C
:1072F0001040BA000160EF00000006000A0D000017
:107300003E200000506100006E53000070650000D8
:10731000656400003D250000640A00000D3E000089
:10732000200000003220EF00C30120008301500044
:1073300005003100E39A2300008041001040BA00AC
:107340000160EF0000000600E09A23008381410005
:10735000808141001380BA00000006000A0D200061
:107360003E2034004A5A20006F6F20006D533500D4
:10737000706420003A202000506F360072742000A4
:10738000202020003120370020320A0020200D006C
:10739000332000003220EF00030220008301500060
:1073A00005003100639E2300008041001040BA00B8
:1073B0000160EF0000000600609E23008381410011
:1073C000808141001380BA000000060020202000C8
:1073D00020202500202032002020640020202000D2
:1073E00020202500202032002020640020252000BD
:1073F00032642500202532003264640020250A0012
:1074000032640D0020253E00326400003220EF007F
:1074100023A12300008041001040BA000160EF006A
:10742000000006000D0A00003E4A00005A6F0000EE
:107430006F6D0000446900007220000020440000CD
:107440006972000065630000746900006F6E0000DF
:107450003A200000312000003220000033200000DC
:10746000342000003520000036200000370A0000DC
:107470000D0000003220EF000302200083015000C5
:107480000500310063A52300008041001040BA00D0
:107490000160EF000000060060A523008381410029
:1074A000808141001380BA000000060020206300A4
:1074B0002020200020202500202063002020200004
:1074C00020202500202063002020200020202500EF
:1074D0002020630020200A0025630D0020253E00A7
:1074E0006320000025630000202500003220EF000B
:1074F00023A82300008041001040BA000160EF0083
:10750000000006000D0A00003E4A00005469000019
:107510006C740000446900007220000020440000E8
:107520006972000065630000746900006F6E0000FE
:107530003A200000312000003220000033200000FB
:10754000342000003520000036200000370A0000FB
:107550000D0000003220EF00C30120008301500025
:107560000500310063AC2300008041001040BA00E8
:107570000160EF000000060060AC23008381410041
:10758000808141001380BA00000006000A0D20002F
:107590003E2034004A542000696C200074533500AA
:1075A000706420003A202000506F36007274200072
:1075B000202020003120370020320A0020200D003A
:1075C000332000003220EF00C3012000830150006F
:1075D00005003100E3AF2300008041001040BA00F5
:1075E0000160EF0000000600E0AF2300838141004E
:1075F000808141001380BA00000006000A0D64007B
:107600003E202C00496420006C655A005A6F6F00C0
:107610006E656F003A206D0050613D006E3D2500A3
:10762000256464002C200A0054690D006C743E002F
:107630003D2500003220EF0063B2230000804100AE
:107640001040BA000160EF00000006000A0D0000C3
:107650003E200000546900006C740000537000006C
:1076600065650000643D0000256400000A0D00000F
:107670003E200000000000003220EF0083B4230011
:10768000008041001040BA000160EF0000000600D9
:107690000A0D00003E2000005A6F00006F6D0000D0
:1076A0005370000065650000643D00002564000023
:1076B0000A0D00003E200000000000003220EF0014
:1076C000A3B62300008041001040BA000160EF0023
:1076D000000006004F6E000020430000616D0000B6
:1076E0006572000061200000496E000069740000AE
:1076F0002C200000736500006E640000204800002C
:107700006F6D000065200000636F00006D6D00006C
:10771000616E0000640A00000D3E000020000000C1
:107720003220EF00430220008301500005003100A9
:10773000C3BA2300008041001040BA000160EF008E
:1077400000000600C0BA230083814100808141000F
:107750001380BA00000006004F6E6E0020436400E4
:10776000616D20006572730061206500496E7100D3
:10777000697475002C20650073656E006E6463008B
:107780002050650072650A0073650D0074203E008C
:1077900031342000206300006F6D00006D61000037
:1077A0003220EF0063022000830150000500310009
:1077B000C3BE2300008041001040BA000160EF000A
:1077C00000000600C0BE230083814100808141008B
:1077D0001380BA00000006000A0D34003E2020008D
:1077E00050726F0065737200657420004C6F30003A
:1077F000633D2900283120002D364C00206F6F009A
:1078000072206300312D610031346C0029200A00A0
:10781000496E0D0043613E006D20200028370000B6
:107820002D3100003220EF00E3C123000080410031
:107830001040BA000160EF00000006000A0D0000D1
:107840003E20000050720000657300006574000067
:107850004C6F0000633D0000416C00006C20000094
:107860004C6F0000636100006C0A00000D3E0000D8
:10787000200000003220EF0063C42300008041009C
:107880001040BA000160EF00000006002F6E0000FB
:107890002F720000000000003220EF0083C523009B
:1078A000008041001040BA000160EF0000000600B7
:1078B0000A0D00003E53000065740000446500009E
:1078C00066610000756C00007420000025640000F3
:1078D000200A00000D3E0000200000003220EF00D2
:1078E000A3C72300008041001040BA000160EF00F0
:1078F000000006000A0D00003E440000656600001E
:10790000617500006C740000436100006D20000090
:1079100025640000200A00000D3E00002000000049
:107920003220EF00C3C92300008041001040BA009C
:107930000160EF00000006000A0D00003E2000007C
:107940005365000072690000616C0000456300002F
:10795000686F00003D4500006E610000626C000031
:10796000656400000A0D00003E20000000000000D9
:107970003220EF0043CC2300008041001040BA00C9
:107980000160EF00000006000A0D00003E2000002C
:107990005365000072690000616C000045630000DF
:1079A000686F00003D4400006973000061620000E0
:1079B0006C650000640A00000D3E0000200000001D
:1079C0003220EF00C3CE2300008041001040BA00F7
:1079D0000160EF00000006000A0D00003E200000DC
:1079E0005365000072690000616C0000496E000080
:1079F000666F00003D4500006E610000626C000093
:107A0000656400000A0D00003E2000000000000038
:107A10003220EF0043D12300008041001040BA0023
:107A20000160EF00000006000A0D00003E2000008B
:107A30005365000072690000616C0000496E00002F
:107A4000666F00003D440000697300006162000041
:107A50006C650000640A00000D3E0000200000007C
:107A60003220EF00C3D32300008041001040BA0051
:107A70000160EF00000006000A0D00003E2000003B
:107A8000486F00006D6500004275000074740000CE
:107A90006F6E00003D4400006973000061620000E9
:107AA0006C650000640A00000D3E0000200000002C
:107AB0003220EF0043D62300008041001040BA007E
:107AC0000160EF00000006000A0D00003E200000EB
:107AD000486F00006D65000042750000747400007E
:107AE0006F6E00003D4500006E610000626C00009A
:107AF000656400000A0D00003E2000000000000048
:107B00003220EF00C3D82300008041001040BA00AB
:107B10000160EF000000060020200000205300005C
:107B200059530000544500004D2000004D45000011
:107B30004E55000020200000202000000000000022
:107B40003220EF00C3DA2300008041001040BA0069
:107B50000160EF000000060020200000205300001C
:107B600065720000696100006C200000496E000031
:107B7000707500007420000020200000000000004C
:107B80003220EF00C3DC2300008041001040BA0027
:107B90000160EF00000006002020000020530000DC
:107BA00065720000696100006C2000004563000000
:107BB000686F00002020000020200000000000006E
:107BC0003220EF00C3DE2300008041001040BA00E5
:107BD0000160EF000000060020200000205300009C
:107BE00065720000696100006C200000496E0000B1
:107BF000666F000020200000202000000000000030
:107C00003220EF00C3E02300008041001040BA00A2
:107C10000160EF000000060020200000205000005E
:107C2000616E0000656C0000204C00006967000078
:107C30006874000073200000202000000000000095
:107C40003220EF00C3E22300008041001040BA0060
:107C50000160EF000000060020200000204300002B
:107C60006C65000061720000204D0000656D000031
:107C70006F7200007920000020200000000000004A
:107C80003220EF00C3E42300008041001040BA001E
:107C90000160EF00000006002020000020430000EB
:107CA0006C650000617200002050000072650000E9
:107CB00073650000747300002020000000000000C5
:107CC0003220EF00C3E62300008041001040BA00DC
:107CD0000160EF000000060020200000506F00004F
:107CE00077650000722000005570000020500000F1
:107CF0007265000073650000742000000000000041
:107D00003220EF00C3E82300008041001040BA0099
:107D10000160EF000000060020200000507200000B
:107D20006573000065740000204C00006F63000064
:107D300061740000696F00006E2000000000000008
:107D40003220EF00C3EA2300008041001040BA0057
:107D50000160EF0000000600202000002044000029
:107D6000756100006C2000004C6900006E6B000023
:107D7000204D00006F64000065200000000000003E
:107D80003220EF00C3EC2300008041001040BA0015
:107D90000160EF000000060020200000566900008E
:107DA000646500006F2000005377000069740000D4
:107DB00063680000657200002020000000000000E1
:107DC0003220EF00C3EE2300008041001040BA00D3
:107DD0000160EF0000000600202000005472000047
:107DE000616E000073690000746900006F6E00002E
:107DF00020540000696D00006520000000000000B4
:107E00003220EF00C3F02300008041001040BA0090
:107E10000160EF0000000600202000002054000058
:107E2000616C00006C790000204F00007574000048
:107E30007075000074730000202000000000000036
:107E40003220EF00C3F22300008041001040BA004E
:107E50000160EF0000000600202000002048000024
:107E60006F6D000065200000427500007474000012
:107E70006F6E0000202000002020000000000000A5
:107E80003220EF00C3F42300008041001040BA000C
:107E90000160EF00000006002020000020500000DC
:107EA000414E00002044000049520000204D0000D7
:107EB000454E00005520000020200000000000007A
:107EC0003220EF00C3F62300008041001040BA00CA
:107ED0000160EF0000000600202000002054000098
:107EE000494C00005420000044490000522000008A
:107EF0004D4500004E55000020200000000000000D
:107F00003220EF00C3F82300008041001040BA0087
:107F10000160EF000000060020200000205A000051
:107F20004F4F00004D200000444900005220000047
:107F30004D4500004E5500002020000000000000CC
:107F40003220EF00C3FA2300008041001040BA0045
:107F50000160EF0000000600202000004341000007
:107F60004D200000534500004152000043480000EE
:107F7000204D0000454E000055200000000000008C
:107F80003220EF00C3FC2300008041001040BA0003
:107F90000160EF00000006002020000043430000C5
:107FA000552000004D4F000044450000204D0000CA
:107FB000454E000055200000202000000000000079
:107FC0003220EF00C3FE2300008041001040BA00C1
:107FD0000160EF00000006002020000020200000CB
:107FE000204100006C6C0000205000006F72000007
:107FF000747300002020000020200000000000001A
:108000003220EF00C3002400008041001040BA007D
:108010000160EF000000060020200000202000008A
:1080200020200000506F000072740000203000001B
:10803000312000002020000020200000000000006F
:108040003220EF00C3022400008041001040BA003B
:108050000160EF000000060020200000202000004A
:1080600020200000506F00007274000020300000DB
:10807000322000002020000020200000000000002E
:108080003220EF00C3042400008041001040BA00F9
:108090000160EF000000060020200000202000000A
:1080A00020200000506F000072740000203000009B
:1080B00033200000202000002020000000000000ED
:1080C0003220EF00C3062400008041001040BA00B7
:1080D0000160EF00000006002020000020200000CA
:1080E00020200000506F000072740000203000005B
:1080F00034200000202000002020000000000000AC
:108100003220EF00C3082400008041001040BA0074
:108110000160EF0000000600202000002020000089
:1081200020200000506F000072740000203000001A
:10813000352000002020000020200000000000006A
:108140003220EF00C30A2400008041001040BA0032
:108150000160EF0000000600202000002020000049
:1081600020200000506F00007274000020300000DA
:108170003620000020200000202000000000000029
:108180003220EF00C30C2400008041001040BA00F0
:108190000160EF0000000600202000002020000009
:1081A00020200000506F000072740000203000009A
:1081B00037200000202000002020000000000000E8
:1081C0003220EF00C30E2400008041001040BA00AE
:1081D0000160EF00000006002020000020200000C9
:1081E000204D0000414900004E2000004D45000098
:1081F0004E5500002020000020200000000000005C
:108200003220EF00C3102400008041001040BA006B
:108210000160EF0000000600202000005265000011
:1082200073630000616E000020430000616D000078
:108230006572000061730000202000000000000053
:108240003220EF00C3122400008041001040BA0029
:108250000160EF00000006002020000043610000E4
:108260006D2000005365000061720000636800002B
:10827000204D0000656E0000752000000000000029
:108280003220EF00C3142400008041001040BA00E7
:108290000160EF0000000600204400006566000059
:1082A000617500006C74000020430000616D0000E7
:1082B00065720000612000004E6F000000000000A9
:1082C0003220EF00C3162400008041001040BA00A5
:1082D0000160EF0000000600204400006566000019
:1082E000617500006C740000205000007265000091
:1082F00073650000742000004E6F00000000000055
:108300003220EF00C3182400008041001040BA0062
:108310000160EF0000000600202000002043000064
:1083200043550000204D00006F64000065200000F0
:108330004D6500006E750000202000000000000068
:108340003220EF00C31A2400008041001040BA0020
:108350000160EF0000000600202000002050000017
:10836000616E00002044000069720000204D000092
:10837000656E000075200000202000000000000055
:108380003220EF00C31C2400008041001040BA00DE
:108390000160EF00000006002020000020540000D3
:1083A000696C000074200000446900007220000025
:1083B0004D6500006E7500002020000000000000E8
:1083C0003220EF00C31E2400008041001040BA009C
:1083D0000160EF000000060020200000205A00008D
:1083E0006F6F00006D2000004469000072200000E3
:1083F0004D6500006E7500002020000000000000A8
:108400003220EF00C3202400008041001040BA0059
:108410000160EF000000060020430000616D0000D5
:108420006572000061200000536500006C6500006B
:10843000637400002042000075730000000000001B
:108440003220EF00C3222400008041001040BA0017
:108450000160EF000000060020500000726500007F
:108460007365000074200000506100006E20000061
:1084700053700000656500006420000000000000EB
:108480003220EF00C3242400008041001040BA00D5
:108490000160EF000000060020500000726500003F
:1084A0007365000074200000546900006C740000C3
:1084B00020530000706500006564000000000000AB
:1084C0003220EF00C3262400008041001040BA0093
:1084D0000160EF00000006002050000072650000FF
:1084E00073650000742000005A6F00006F6D00007B
:1084F000205300007065000065640000000000006B
:108500003220EF00C3282400008041001040BA0050
:108510000160EF0000000600202000002020000085
:108520005379000073740000656D0000204D000059
:10853000656E000075200000202000000000000093
:108540003220EF00C32A2400008041001040BA000E
:108550000160EF0000000600202000002020000045
:10856000202000005374000061720000742000009D
:10857000202000002020000020200000000000003B
:108580003220EF00C32C2400008041001040BA00CC
:108590000160EF0000000600202000002020000005
:1085A000204300006F6E0000747200006F6C0000CA
:1085B00020410000202000002020000000000000DA
:1085C0003220EF00C32E2400008041001040BA008A
:1085D0000160EF00000006002020000020200000C5
:1085E000204300006F6E0000747200006F6C00008A
:1085F0002042000020200000202000000000000099
:108600003220EF00C3302400008041001040BA0047
:108610000160EF0000000600202000002020000084
:1086200020200000202000004F4E000020200000ED
:10863000202000002020000020200000000000007A
:108640003220EF00C3322400008041001040BA0005
:108650000160EF0000000600202000002020000044
:1086600020200000204F000046460000202000008F
:10867000202000002020000020200000000000003A
:108680003220EF00C3342400008041001040BA00C3
:108690000160EF0000000600202000002020000004
:1086A000204800006F6D000065200000436100005D
:1086B0006D650000726100002020000000000000D5
:1086C0003220EF00C3362400008041001040BA0081
:1086D0000160EF00000006002020000020200000C4
:1086E00020500000726500007365000074200000D7
:1086F0003134000020200000202000000000000095
:108700003220EF00C3382400008041001040BA003E
:108710000160EF0000000600202000002020000083
:10872000204100006C6C0000204C00006F630000D2
:10873000616C0000202000002020000000000000EC
:108740003220EF00C33A2400008041001040BA00FC
:108750000160EF000000060020200000362000002D
:10876000496E0000436100006D20000038200000C9
:108770004C6F0000636100006C20000000000000EE
:108780003220EF00C33C2400008041001040BA00BA
:108790000160EF000000060020200000204E0000D5
:1087A0006F7200006D6100006C6C000079200000A9
:1087B0004F700000656E00002020000000000000E7
:1087C0003220EF00C33E2400008041001040BA0078
:1087D0000160EF000000060020200000204E000095
:1087E0006F7200006D6100006C6C00007920000069
:1087F000436C00006F73000065640000000000001F
:108800003220EF00C3402400008041001040BA0035
:108810000160EF0000000600202000002020000082
:1088200020200000202000004E6F00006E65000038
:108830002020000020200000202000000000000078
:108840003220EF00C3422400008041001040BA00F3
:108850000160EF000000060020200000204500001D
:1088600064690000726F00006C2000003448000052
:108870002C200000335300002020000000000000E6
:108880003220EF00C3442400008041001040BA00B1
:108890000160EF0000000600204900006E6F00003C
:1088A00076610000746900006F6E000020620000B5
:1088B00079200000495300004953000000000000E7
:1088C0003220EF00C3462400008041001040BA006F
:1088D0000160EF000000060020200000205500008D
:1088E00073650000722000004465000066690000A6
:1088F0006E650000642000002020000000000000E1
:108900003220EF00C3482400008041001040BA002C
:108910000160EF0000000600202000002020000081
:10892000202000004E6F0000726D0000616C00009E
:108930002020000020200000202000000000000077
:108940003220EF00C34A2400008041001040BA00EA
:108950000160EF0000000600202000002020000041
:1089600020200000496E000076650000727400004F
:108970002020000020200000202000000000000037
:108980003220EF00C34C2400008041001040BA00A8
:108990000160EF0000000600204100007574000037
:1089A0006F200000536500006172000063680000E2
:1089B000204D00006F6400006520000000000000F2
:1089C0003220EF00C34E2400008041001040BA0066
:1089D0000160EF00000006002020000020200000C1
:1089E000205300006F6E0000792000004F6E0000E1
:1089F0006C79000020200000202000000000000012
:108A00003220EF00C3502400008041001040BA0023
:108A10000160EF0000000600202000002020000080
:108A2000436100006E6F00006E2000004F6E00007A
:108A30006C790000202000002020000000000000D1
:108A40003220EF00C3522400008041001040BA00E1
:108A50000160EF000000060020430000616E00008E
:108A60006F6E0000204F00006E6C00007920000047
:108A700049530000204F00006E200000000000005D
:108A80003220EF00C3542400008041001040BA009F
:108A90000160EF000000060020200000506100008F
:108AA0006E610000736F00006E69000063200000BB
:108AB0004F6E00006C7900002020000000000000D4
:108AC0003220EF00C3562400008041001040BA005D
:108AD0000160EF00000006002020000020200000C0
:108AE000204E00006F200000436100006D65000013
:108AF0007261000020200000202000000000000023
:108B00003220EF00C3582400008041001040BA001A
:108B10000160EF0000000600202000004469000012
:108B2000726500006374000020430000616D000066
:108B300020430000747200006C2000000000000060
:108B40003220EF00C35A2400008041001040BA00D8
:108B50000160EF00000006002020000043430000F9
:108B600055200000436100006D200000436F0000AD
:108B70006E740000726F00006C20000000000000A6
:108B80003220EF00C35C2400008041001040BA0096
:108B90000160EF0000000600205300007973000020
:108BA000746500006D200000496E00002053000035
:108BB000746100006E640000627900000000000033
:108BC0003220EF00C35E2400008041001040BA0054
:108BD0000160EF0000000600556E0000657800009F
:108BE000706500006374000065640000205500009B
:108BF0004152000054310000204500007272000014
:108C00006F7200000A0D0000000000003220EF002B
:108C100023612400008041001040BA000160EF0091
:108C200000000600556E00006578000070650000C9
:108C3000637400006564000020550000415200008C
:108C40005432000020450000727200006F72000074
:108C50000A0D0000000000003220EF0083632400B2
:108C6000008041001040BA000160EF0000000600E3
:108C7000556E0000657800007065000063740000A8
:108C8000656400002053000054410000434B000085
:108C9000455200005220000045720000726F000033
:108CA000720A00000D0000003220EF00036624006D
:108CB000008041001040BA000160EF000000060093
:108CC000556E000065780000706500006374000058
:108CD000656400002041000044440000524500004B
:108CE0005252000020450000727200006F720000B6
:108CF0000A0D0000000000003220EF00836824000D
:108D0000008041001040BA000160EF000000060042
:108D1000556E000065780000706500006374000007
:108D200065640000204D00004154000048450000EB
:108D30005252000020450000727200006F72000065
:108D40000A0D0000000000003220EF00036B240039
:108D5000008041001040BA000160EF0000000600F2
:108D6000556E0000657800007065000063740000B7
:108D70006564000020640000656600006175000005
:108D80006C74000020450000727200006F720000D9
:108D90000A0D0000000000003220EF00836D240067
:108DA000008041001040BA000160EF0000000600A2
:108DB0005365000072690000616C000020420000F1
:108DC0006F6F0000742000004C6F000061640000B1
:108DD000203F0000000000003220EF00836F2400DD
:108DE000008041001040BA000160EF000000060062
:108DF000204800006F6C0000642000004D610000FE
:108E00007374000065720000506F00007765000009
:108E100072200000000000003220EF008371240067
:108E2000008041001040BA000160EF000000060021
:108E3000666F00007220000034200000736500009F
:108E400063200000746F0000205300007461000074
:108E500072740000000000003220EF0083732400D1
:108E6000008041001040BA000160EF0000000600E1
:108E700020200000204200006F6F000074200000DE
:108E80006C6F00006164000065720000202000002B
:108E900020200000000000003220EF008375240035
:108EA000008041001040BA000160EF0000000600A1
:108EB0002020000020200000256600002073000014
:108EC000656300002020000020200000202000001A
:108ED000200000003220EF00637724000080410072
:108EE0001040BA000160EF000000060020200000E2
:108EF00020520000656C0000656100007365000091
:108F0000207400006F2000002020000020200000BE
:108F1000000000003220EF0063792400008041004F
:108F20001040BA000160EF000000060020200000A1
:108F300020200000436F00006E740000696E000086
:108F40007565000020200000202000002020000087
:108F5000000000003220EF00637B2400008041000D
:108F60001040BA000160EF00000006002020000061
:108F700020200000202000002020000020200000F1
:108F800020200000202000002020000020200000E1
:108F9000000000003220EF00637D240000804100CB
:108FA0001040BA000160EF0000000600426F0000B0
:108FB0006F7400006C6F0000616400006572000057
:108FC00020530000746100007274000065640000AA
:108FD000000000003220EF00637F24000080410089
:108FE0001040BA000160EF0000000600746F00003E
:108FF000204300006F6E000066690000726D000083
:109000002052000065710000756500007374000057
:10901000000000003220EF00638124000080410046
:109020001040BA000160EF000000060020200000A0
:10903000204200006F6F00007420000052650000A5
:10904000717500006573000074200000202000008E
:10905000000000003220EF00638324000080410004
:109060001040BA000160EF0000000600204300003D
:109070006F6E0000746900006E75000065200000CE
:10908000486F00006C640000696E000067200000FB
:10909000000000003220EF006385240000804100C2
:1090A0001040BA000160EF000000060020420000FE
:1090B0006F6F0000746C00006F610000642000009E
:1090C00053740000617200007465000064200000A9
:1090D000000000003220EF00638724000080410080
:1090E0001040BA000160EF000000060020200000E0
:1090F0002020000020250000730000003220EF0037
:10910000A3882400008041001040BA000160EF00F5
:1091100000000600204900006E690000746900002C
:10912000616C00007A650000204500004550000099
:10913000726F00006D200000000000003220EF0080
:10914000A38A2400008041001040BA000160EF00B3
:10915000000006002045000045500000726F00002E
:109160006D200000496E0000697400006961000014
:109170006C7A000065640000200000003220EF00DF
:10918000A38C2400008041001040BA000160EF0071
:1091900000000600204C00006F61000064690000C0
:1091A0006E670000204400006566000061750000E5
:1091B0006C74000073200000000000003220EF00FB
:1091C000A38E2400008041001040BA000160EF002F
:1091D00000000600202000002020000020200000C9
:1091E000202000002020000020200000202000007F
:1091F0002020000020200000200000004200F80095
:109200003600F800801F7800200020000C000900C4
:10921000B01F78000100200001007800E045020046
:10922000000000008100E800811F78002322AF00C9
:10923000FEFF370020118800CF0078007001200069
:109240000008E600F4FF37008C20A9008C20A9005C
:10925000A00120000C0009004F1078004F0078009A
:109260003600F9004200F900004006004200F80014
:109270003600F800801F7800200020000C00090054
:10928000B01F7800010020000100780006460200AF
:10929000000000008100E800811F78002322AF0059
:1092A000FEFF370020118800CF00780070012000F9
:1092B0000008E600F4FF37008C40A9008C40A900AC
:1092C000A00120000C0009004F1078004F0078002A
:1092D0003600F9004200F900004006004200F800A4
:1092E0003600F800801F7800200020000C000900E4
:1092F000B01F780001002000010078002C46020019
:10930000000000008100E800811F78002322AF00E8
:10931000FEFF370020118800CF007800A001200058
:109320000008E600F4FF37008040A9008040A90053
:10933000A00120000C0009004F1078004F007800B9
:109340003600F9004200F900004006004200F80033
:109350003600F800801F7800200020000C00090073
:10936000B01F780001002000010078005446020080
:10937000000000008100E800811F78002322AF0078
:10938000FEFF370020118800CF00780090012000F8
:109390000008E600F4FF37008060A9008060A900A3
:1093A000A00120000C0009004F1078004F00780049
:1093B0003600F9004200F900004006004200F800C3
:1093C0003600F800801F7800200020000C00090003
:1093D000B01F780001002000010078007C460200E8
:1093E000000000008100E800811F78002322AF0008
:1093F000FEFF370020118800CF0078009001200088
:109400000008E600F4FF37008080A9008080A900F2
:10941000A00120000C0009004F1078004F007800D8
:109420003600F9004200F900004006004200F80052
:109430003600F800801F7800200020000C00090092
:10944000B01F78000100200001007800A44602004F
:10945000000000008100E800811F78002322AF0097
:10946000FEFF370020118800CF0078009001200017
:109470000008E600F4FF3700A00120000C000900FE
:109480004F1078004F0078003600F9004200F900D4
:10949000004006004200F8003600F800801F780007
:1094A000200020000C000900B01F7800503F810010
:1094B00000C0B300503F8900503F81000160EF00C1
:1094C000503F89002202AE00FEFF370030118000BD
:1094D000EA27F800F0FF9F00EA27F900944B80008C
:1094E0004822DE00C399200083024200EA27F800E8
:1094F0004F0078004800DE00804A780073C9BF0042
:10950000EA27F800E0FF9F00EA27F900944B80006B
:109510004822DE00614242000440780000E0B700CB
:10952000F40F20000024E10004003A00000037009E
:109530007369EF00A04A0400000000007369EC00AA
:1095400073C9BF008B49E30003003A0000003700F5
:10955000503F810073E9B700503F81004800DE00B2
:109560006D04E10002003A00000037009B69EC0046
:109570004148A80040C9BF007F4060000004E000EF
:1095800050003A00000037008C08AE0001003700A0
:109590004C0037003E69AF0001003700490037003A
:1095A000503F81004800DE00140220000024E1004A
:1095B00001003A000C003700503F81004800DE00F7
:1095C000240220000024E10001003A0006003700D8
:1095D000503F81004800DE00040320000024E10029
:1095E00010003A0000003700444380004822DE00AB
:1095F00013082000041CE1000A003E0000003700B0
:10960000444380004822DE0093082000041CE1004F
:109610000400390000003700503F81000160EF0076
:10962000503F8900503F81004800DE007F04E10088
:109630000700360000003700503F81004800DE0080
:10964000F40720000024E100010036000500370087
:10965000503F81004800DE006804E10019003A0034
:1096600000003700EA27F8004F0078004800DE00CD
:109670002322AF00FEFF370024E2B7002562EF008F
:10968000503F81004800DE006804E1000D003A0010
:109690000000370000C2B3002322AF00FEFF3700F6
:1096A00024E2B7002562EF00EA27F8004F007800B7
:1096B0004800DE002322AF00FEFF370024E2B7009F
:1096C0002562EF00EA27F8004F0078004800DE002E
:1096D00069E8B7009560A8008560A900A001200096
:1096E0000C0009004F1078004F0078003600F90098
:1096F0004200F900004006004200F8003600F80081
:10970000801F7800200020000C000900B01F7800A6
:10971000503F810000C0B300503F89003202AE00CC
:10972000FEFF3700B0118000EA27F800E0FF9F003D
:10973000EA27F9008C28AF00010037000700370046
:10974000503F81002322AF00FEFF370024E2B70024
:109750002562EF00D64B040000000000D4548000C6
:109760004822DE00C3A9200083024200503F81004E
:10977000804298004168A800D45480004822DE004E
:10978000614242000440780000E0B700F407200086
:109790000024E10004003E00000037009B6AEF0057
:1097A000D64B0400000000009B6AEC0097C0A800A4
:1097B00087C0A900A00120000C0009004F1078000C
:1097C0004F0078003600F9004200F9000040060022
:1097D0004200F8003600F800801F780020002000CA
:1097E0000C000900B01F780004002000543F8900DD
:1097F00004002000643F890004002000743F8900B9
:1098000004002000843F890004002000943F890068
:1098100004002000A43F890004002000B43F890018
:10982000C03F810000C0B300C03F8900C03F81003D
:109830000160EF00C03F8900D03F810000C0B3004D
:10984000D03F8900D03F81000160EF00D03F890008
:10985000E03F810000C0B300E03F8900E03F8100AD
:109860000160EF00E03F89009500A900F4F72F00A8
:1098700094168800D402F800EA27F900503F8100CE
:1098800000027800F0F7270004006000703F8900B4
:10989000703F81007288B600903F8900141828003C
:1098A00024178800E602F800EC27F900603F8100E9
:1098B000000278001018280004006000803F890032
:1098C000803F81007488B600A03F8900903F8100EE
:1098D0000000E0000100320004003700A03F8100DA
:1098E0000000E0009E00320000003700903F810041
:1098F0000000E0005100320000003700903F81007E
:10990000FA27F800E0FF9F00FA27F900F227F80095
:109910004F0078004800DE00FA27F800F0FF9F00B3
:10992000FA27F900D03F8100D43F81004822DE00B1
:109930002E08F800F4FF9F002E08F9002FE8B6006B
:1099400072C8BF00FC27F800E0FF9F00FC27F90069
:1099500073C8BF00FC27F800F0FF9F00FC27F90048
:10996000D03F81004800DE00E43F810004406800F1
:10997000F827F800E0FF9F00F827F900703F81000A
:10998000FA27F800E0FF9F00FA27F900D03F810096
:10999000E43F81004822DE001C08F800F4FF9F002D
:1099A0001C08F9001DE8B60004002000B43F89003F
:1099B000B03F81006700E1001E0031000000370069
:1099C0002FC8BF0080007800B03F81000100A500D3
:1099D00001003100120037001DC8BF008000780070
:1099E000B03F81000100A5000100390007003700E9
:1099F000B03F81004100DD008487200084024000E8
:109A0000950AE900104D040000000000B03F8100FD
:109A10004100DD008487200084024000950AE800B0
:109A2000B03F81000000E800B03F8900D84C04003E
:109A300000000000EE27F8007208F900A03F810046
:109A40000000E0004200320000003700A03F81002B
:109A5000FA27F800E0FF9F00FA27F900F427F80042
:109A60004F0078004800DE00FA27F800F0FF9F0062
:109A7000FA27F900D03F8100D43F81004822DE0060
:109A80002E08F800F4FF9F002E08F9002FE8B6001A
:109A900074C8BF00FC27F800E0FF9F00FC27F90016
:109AA00075C8BF00FC27F800F0FF9F00FC27F900F5
:109AB000D03F81004800DE00E43F810004406800A0
:109AC000F827F800E0FF9F00F827F900803F8100A9
:109AD000FA27F800E0FF9F00FA27F900D03F810045
:109AE000E43F81004822DE001C08F800F4FF9F00DC
:109AF0001C08F9001DE8B6002F08AF000100370070
:109B0000070037001D08AE000100370003003700D2
:109B10008628ED00904D0400000000008628EC002F
:109B20002FE8AF0001003700070037001DE8AE0046
:109B300001003700030037008828ED00A44D040021
:109B4000000000008828EC00F027F8007408F900F5
:109B50004108A8007628EF00B24D04000000000084
:109B60007628EC002003A9002023A8002003AE00E3
:109B7000FEFF3700001880004200DE00F827F800E2
:109B8000F0FF9F00F827F900B4A180006D4052005B
:109B90000080FB008443210084024000F827F80085
:109BA0004F0078004800DE00804A78003674EC00F0
:109BB000B4A180006F24E1000300360000003700EC
:109BC000D0C0B30036F4B70036D4BF0028E3B700E6
:109BD0002963EF008500A9009500A8008500A90071
:109BE000A00120000C0009004F1078004F00780001
:109BF0003600F9004200F900004006008200200013
:109C00001E00090000000000C4E2A900C0E2A90093
:109C10001F0009000000000081C0D200C4C2A900DA
:109C20004200AF00C0C2A8004200AE00C0C2A900FE
:109C3000C0E2A800C2E2AE00FEFF37000201E90068
:109C4000EFFF3A001E00090000000000C4E2A90076
:109C5000C0E2A90000000000C0C2A8001F00090067
:109C6000000000001F00090000000000C0E2A80082
:109C7000C2E2AE00FEFF37001F0009000000000036
:109C800000002000C2C2AF000000A000C4E2A90092
:109C9000C0E2A900C4C2A900C0C2A9000000060019
:109CA000C0C2A8001E00090000000000C0E2A80019
:109CB0001F00090000000000C2E2AE00FEFF3700F6
:109CC000C4C2A900C0C2A9001E0009000000000013
:109CD000C4E2A900C0E2A9009E0009000000000043
:109CE00061C4B300FE4D0200000000009E000900A8
:109CF00000000000E13F8100FE4D02000000000076
:109D00009E00090000000000FC27F800CF0078004A
:109D1000C808DE00FE4D0200000000009E000900A1
:109D200000000000C0C2A90000000000C0E2A800BE
:109D3000C2E2AE00FEFF37001E0009000000000076
:109D40000100090000000000C0C2A8001E000900B8
:109D500000000000BE000900000000000000060036
:109D6000A03F81000160EF001080B2004D00320082
:109D70007080B200570032005080B20055003200AF
:109D80007080B200530032003080B20051003200C7
:109D9000F080B2004F003200D080B2004D0032009F
:109DA0009081B200AC0032001080B200AA003200F4
:109DB0003080B200A80032001080B200A60032004D
:109DC000F083B200A40032001080B200A200320082
:109DD0003080B200A00032001080B20013013200C7
:109DE0007080B200110132001080B2000F01320009
:109DF0003080B2000D0132001080B2000B01320041
:109E0000F080B200090132001080B2000701320078
:109E1000D083B200820132007080B2008001320033
:109E20001080B2007E0132003080B2007C0132002E
:109E30001080B2007A013200F081B2007801320065
:109E40001080B200760132005081B200E30132008E
:109E50001080B200E10132003080B200DF01320038
:109E60001080B200DD013200F080B200DB01320070
:109E70001080B200D90132003080B200D701320028
:109E8000C085B200440232003080B2004F0232007E
:109E90001080B2005A0232007080B20070023200AC
:109EA000A8023700A03F81004800DE000004E00067
:109EB00004003A00DCC2A800D8C2A900664F040022
:109EC00000000000DCC2A900D8C2A900A25404000E
:109ED00000000000A03F81004800DE000004E00018
:109EE0002A003A00A03F81006604E10004003A0025
:109EF000E41221001400A100C24F04000000000081
:109F0000A03F81006304E10004003A00E412210054
:109F10001410A100C24F040000000000A03F810007
:109F20006404E10004003A00E41221001420A100BE
:109F3000C24F040000000000A03F81006704E10060
:109F400004003A00E41221001430A100C24F0400C2
:109F500000000000A03F81006804E10004003A0016
:109F6000E41221001440A100C24F040000000000D0
:109F7000A03F81006504E10002003A00E4122100E4
:109F80001450A1001650040000000000A03F810002
:109F90006604E10004003A00E41221001400A0006D
:109FA0001650040000000000A03F81006304E1009F
:109FB00004003A00E41221001410A000165004001E
:109FC00000000000A03F81006404E10004003A00AA
:109FD000E41221001420A00016500400000000002C
:109FE000A03F81006704E10004003A00E412210070
:109FF0001430A0001650040000000000A03F8100B3
:10A000006804E10004003A00E41221001440A000BA
:10A010001650040000000000A03F81006504E1002C
:10A0200002003A00E41221001450A000E03F810039
:10A0300080C0B300E03F89002ED1BF00FC27F800AC
:10A04000F0FF9F00FC27F900504E020000000000C6
:10A05000A254040000000000A03F81004800DE0080
:10A060000004E00034003A00A03F81007C04E100DD
:10A0700004003A00041321001410A10098500400B9
:10A0800000000000A03F81007D04E10004003A00D0
:10A09000041321001420A1009850040000000000C7
:10A0A000A03F81007E04E10004003A000413210077
:10A0B0001430A1009850040000000000A03F81006F
:10A0C0007F04E10004003A00041321001440A100C1
:10A0D0009850040000000000A03F8100040220000E
:10A0E0000024E10004003A00041321001450A100F0
:10A0F0009850040000000000A03F810014022000DE
:10A100000024E10004003A00041321001460A100BF
:10A110009850040000000000A03F810024022000AD
:10A120000024E10002003A00041321001470A10091
:10A130000051040000000000A03F81007C04E10009
:10A1400004003A00041321001410A0000051040080
:10A1500000000000A03F81007D04E10004003A00FF
:10A16000041321001420A00000510400000000008E
:10A17000A03F81007E04E10004003A0004132100A6
:10A180001430A0000051040000000000A03F810036
:10A190007F04E10004003A00041321001440A000F1
:10A1A0000051040000000000A03F810004022000D4
:10A1B0000024E10004003A00041321001450A00020
:10A1C0000051040000000000A03F810014022000A4
:10A1D0000024E10004003A00041321001460A000F0
:10A1E0000051040000000000A03F81002402200074
:10A1F0000024E10002003A00041321001470A000C2
:10A20000E03F810090C0B300E03F890030D1BF0043
:10A21000FC27F800F0FF9F00FC27F900504E0200D9
:10A2200000000000A254040000000000A03F8100D4
:10A230004800DE000004E00038003A00A03F810042
:10A24000340220000024E10004003A00241321001D
:10A250001410A1008A51040000000000A03F8100FA
:10A26000440220000024E10004003A0024132100ED
:10A270001420A1008A51040000000000A03F8100CA
:10A28000540220000024E10004003A0024132100BD
:10A290001430A1008A51040000000000A03F81009A
:10A2A000640220000024E10004003A00241321008D
:10A2B0001440A1008A51040000000000A03F81006A
:10A2C000740220000024E10004003A00241321005D
:10A2D0001450A1008A51040000000000A03F81003A
:10A2E000840220000024E10004003A00241321002D
:10A2F0001460A1008A51040000000000A03F81000A
:10A30000940220000024E10002003A0024132100FE
:10A310001470A100FA51040000000000A03F810069
:10A32000340220000024E10004003A00241321003C
:10A330001410A000FA51040000000000A03F8100AA
:10A34000440220000024E10004003A00241321000C
:10A350001420A000FA51040000000000A03F81007A
:10A36000540220000024E10004003A0024132100DC
:10A370001430A000FA51040000000000A03F81004A
:10A38000640220000024E10004003A0024132100AC
:10A390001440A000FA51040000000000A03F81001A
:10A3A000740220000024E10004003A00241321007C
:10A3B0001450A000FA51040000000000A03F8100EA
:10A3C000840220000024E10004003A00241321004C
:10A3D0001460A000FA51040000000000A03F8100BA
:10A3E000940220000024E10002003A00241321001E
:10A3F0001470A000E03F8100A0C0B300E03F8900DE
:10A4000032D1BF00FC27F800F0FF9F00FC27F900C5
:10A41000504E020000000000A254040000000000A2
:10A42000A03F81004800DE000004E00031003A0057
:10A43000A03F81007404E10004003A0044132100AD
:10A440001410A1007652040000000000A03F81001B
:10A450007304E10004003A00441321001420A10019
:10A460007652040000000000A03F81007204E10069
:10A4700004003A00441321001430A1007652040075
:10A4800000000000A03F81007104E10004003A00D8
:10A49000441321001440A100765204000000000083
:10A4A000A03F81007004E10004003A004413210041
:10A4B0001450A1007652040000000000A03F81006B
:10A4C0006F04E10004003A00441321001460A1006D
:10A4D0007652040000000000A03F81006E04E100FD
:10A4E00002003A00441321001470A100D852040065
:10A4F00000000000A03F81007404E10004003A0065
:10A50000441321001410A000D852040000000000E1
:10A51000A03F81007304E10004003A0044132100CD
:10A520001420A000D852040000000000A03F8100C9
:10A530007204E10004003A00441321001430A0002A
:10A54000D852040000000000A03F81007104E10027
:10A5500004003A00441321001440A000D852040023
:10A5600000000000A03F81007004E10004003A00F8
:10A57000441321001450A000D85204000000000031
:10A58000A03F81006F04E10004003A004413210061
:10A590001460A000D852040000000000A03F810019
:10A5A0006E04E10002003A00441321001470A00080
:10A5B000E03F8100B0C0B300E03F890034D1BF006C
:10A5C000FC27F800F0FF9F00FC27F900504E020026
:10A5D00000000000A254040000000000A03F810021
:10A5E0004800DE000004E00031003A00A03F810096
:10A5F0007B04E10004003A00641321001410A10060
:10A600005453040000000000A03F81007A04E100E0
:10A6100004003A00641321001420A10054530400E4
:10A6200000000000A03F81007904E10004003A002E
:10A63000641321001430A1005453040000000000F2
:10A64000A03F81007804E10004003A006413210077
:10A650001440A1005453040000000000A03F8100FA
:10A660007704E10004003A00641321001450A100B3
:10A670005453040000000000A03F81007604E10074
:10A6800004003A00641321001460A1005453040034
:10A6900000000000A03F81007504E10002003A00C4
:10A6A000641321001470A100B653040000000000E0
:10A6B000A03F81007B04E10004003A006413210004
:10A6C0001410A000B653040000000000A03F810059
:10A6D0007A04E10004003A00641321001420A00071
:10A6E000B653040000000000A03F81007904E1009F
:10A6F00004003A00641321001430A000B653040093
:10A7000000000000A03F81007804E10004003A004E
:10A71000641321001440A000B653040000000000A0
:10A72000A03F81007704E10004003A006413210097
:10A730001450A000B653040000000000A03F8100A8
:10A740007604E10004003A00641321001460A000C4
:10A75000B653040000000000A03F81007504E10032
:10A7600002003A00641321001470A000E03F810051
:10A77000C0C0B300E03F890036D1BF00FC27F8001D
:10A78000F0FF9F00FC27F900504E0200000000007F
:10A79000A254040000000000F40F2000A4898800E7
:10A7A000E03F8100B0C0B300E03F890034D1BF007A
:10A7B000FC27F800F0FF9F00FC27F900504E020034
:10A7C00000000000A254040000000000F40F20006C
:10A7D000B4898800E03F8100C0C0B300E03F890039
:10A7E00036D1BF00FC27F800F0FF9F00FC27F900DE
:10A7F000504E020000000000A254040000000000BF
:10A80000F40F200084898800E03F810090C0B300ED
:10A81000E03F890030D1BF00FC27F800F0FF9F0027
:10A82000FC27F900504E020000000000F40F200049
:10A8300094898800E03F8100A0C0B300E03F890018
:10A8400032D1BF00FC27F800F0FF9F00FC27F90081
:10A85000504E020000000000A2540400000000005E
:10A86000F40F200074898800E03F810080C0B300AD
:10A87000E03F89002ED1BF00FC27F800F0FF9F00C9
:10A88000FC27F900504E020000000000F40F2000E9
:10A8900084898800E03F810090C0B300E03F8900D8
:10A8A00030D1BF00FC27F800F0FF9F00FC27F90023
:10A8B000504E020000000000F40F20009489880030
:10A8C000E03F8100A0C0B300E03F890032D1BF006B
:10A8D000FC27F800F0FF9F00FC27F900504E020013
:10A8E00000000000F40F2000A4898800E03F8100F0
:10A8F000B0C0B300E03F890034D1BF00FC27F800AE
:10A90000F0FF9F00FC27F900504E020000000000FD
:10A91000F40F2000B4898800E03F8100C0C0B3007C
:10A92000E03F890036D1BF00FC27F800F0FF9F0010
:10A93000FC27F900504E020000000000A254040061
:10A940000000000000000600C03F81000160EF0031
:10A95000C03F8900C03F81000160EF009082B200DB
:10A960001B0032001080B2001F003200F080B200E5
:10A97000230032001080B200270032003080B20085
:10A980002B0032001080B2002F0032007080B20025
:10A99000330032001080B200370032003080B20045
:10A9A0003B0032001080B2003F003200F083B20062
:10A9B000430032001080B200470032003080B20005
:10A9C0004B0032001080B2004F0032004E003700C2
:10A9D000C03F81004800DE000040E800F827F80092
:10A9E000F0FF9F00F827F900C03F81004800DE001B
:10A9F0000040E800F827F800F0FF9F00F827F90072
:10AA0000C03F81004800DE000040E800F827F80061
:10AA1000F0FF9F00F827F900C03F81004800DE00EA
:10AA20000040E800F827F800F0FF9F00F827F90041
:10AA3000C03F81004800DE000040E800F827F80031
:10AA4000F0FF9F00F827F900C03F81004800DE00BA
:10AA50000040E800F827F800F0FF9F00F827F90011
:10AA6000C03F81004800DE000040E800F827F80001
:10AA7000F0FF9F00F827F900C03F81004800DE008A
:10AA80000040E800F827F800F0FF9F00F827F900E1
:10AA9000C03F81004800DE000040E800F827F800D1
:10AAA000F0FF9F00F827F900C03F81004800DE005A
:10AAB0000040E800F827F800F0FF9F00F827F900B1
:10AAC000C03F81004800DE000040E800F827F800A1
:10AAD000F0FF9F00F827F900C03F81004800DE002A
:10AAE0000040E800F827F800F0FF9F00F827F90081
:10AAF000C03F81004800DE000040E800F827F80071
:10AB0000F0FF9F00F827F900C03F81004800DE00F9
:10AB10000040E800F827F800F0FF9F00F827F90050
:10AB2000F827F8004F0078004800DE00000006001B
:10AB3000D03F81000160EF00D03F8900D03F81000D
:10AB40000160EF002080B2001B0032001080B200D4
:10AB5000200032007080B200250032001080B20068
:10AB60002A0032003080B2002F0032001080B20084
:10AB700034003200F080B200390032001080B200A0
:10AB80003E0032003080B200430032001080B2003C
:10AB9000480032007080B2004D0032001080B200D8
:10ABA000520032003080B20057003200F080B20014
:10ABB0005C0032005B003700D03F81000080FD0068
:10ABC000D0C1B3000080FD00D03F8900A056040032
:10ABD00000000000D03F81000080FD00E0C1B30014
:10ABE0000080FD00D03F8900A05604000000000056
:10ABF000D03F81000080FD00F0C1B3000080FD0067
:10AC0000D03F8900A056040000000000D03F810022
:10AC10000080FD0000C2B3000080FD00D03F89002D
:10AC2000A056040000000000D03F81000080FD001D
:10AC300010C2B3000080FD00D03F8900A056040080
:10AC400000000000D03F81000080FD0020C2B30062
:10AC50000080FD00D03F8900A056040000000000E5
:10AC6000D03F81000080FD0030C2B3000080FD00B5
:10AC7000D03F8900A056040000000000D03F8100B2
:10AC80000080FD0040C2B3000080FD00D03F89007D
:10AC9000A056040000000000D03F81000080FD00AD
:10ACA00050C2B3000080FD00D03F8900A0560400D0
:10ACB00000000000D03F81000080FD0060C2B300B2
:10ACC0000080FD00D03F8900A05604000000000075
:10ACD000D03F81000080FD0070C2B3000080FD0005
:10ACE000D03F8900A056040000000000D03F810042
:10ACF0000080FD0080C2B3000080FD00D03F8900CD
:10AD0000A056040000000000D03F81000080FD003C
:10AD100090C2B3000080FD00D03F8900A05604001F
:10AD200000000000D03F81000080FD00C0C1B300E2
:10AD30000080FD00D03F8900A05604000000000004
:10AD4000FA27F8004F0078004800DE0000000600F7
:10AD5000851F780004002000843F89000400200043
:10AD6000943F8900703F81007C04E10005003100C0
:10AD7000703F8100C0C1B300703F8900D05604000D
:10AD800000000000703F8100940220000024E100D8
:10AD900003003100703F810090C2B300703F890012
:10ADA000703F8100F827F800E0FF9F00F827F900C6
:10ADB000A454020000000000F027F800E0FF9F000C
:10ADC000F027F900803F81000160EF00803F89009B
:10ADD000803F81000000E0002100320004002000DC
:10ADE000943F8900903F81006E00E1001C0031001B
:10ADF000803F810061004000803F8900803F8100EA
:10AE00006E00E1000200360014002000843F89003B
:10AE1000843F81000960EF00C398200003004200D6
:10AE20001004E00009003A00803F8100FA27F80092
:10AE3000E0FF9F00FA27F90098550200000000008B
:10AE4000080037003057040000000000903F8100E8
:10AE50000000E800903F8900F25604000000000066
:10AE60000060EF00CF027800000006004200F8000A
:10AE70003600F800801F7800200020000C00090038
:10AE8000B01F780004002000543F8900603F81001B
:10AE900000C0B300603F89009A60A9006E28EC00F2
:10AEA0007008E20002003200000037007028ED0058
:10AEB0000A28EC00544080006A20E1005800390064
:10AEC000000037000A28EF0004002000543F8900EA
:10AED000503F81007100E100510031000000370057
:10AEE000503F810004832000040040001004E00073
:10AEF0004600320000003700503F8100C48020002F
:10AF0000040040001004E000380032000000370068
:10AF1000503F81000483200004004000104278006C
:10AF200004CEB2000F003A0000003700503F81000D
:10AF3000C48020000400400090427800F427F8000C
:10AF4000E5FF9F00F427F900A03F81000160EF00BA
:10AF5000A03F8900B04E020000000000F657040038
:10AF600000000000503F81000483200004004000E6
:10AF70001042780004CFB20011003A000000370000
:10AF8000503F8100C48020000400400090427800BF
:10AF9000F427F800E5FF9F00F427F900A03F8100A7
:10AFA0000080FD0010C0B3000080FD00A03F8900BC
:10AFB000B04E020000000000F65704000000000040
:10AFC000503F8100048320000400400010427800BC
:10AFD00004CDB20005003A0000003700503F810068
:10AFE000C480200084024000804AEB00503F810072
:10AFF000C480200084024000804AEB00503F810062
:10B000000483200084024000804AEB00503F81000E
:10B010000000E800503F890068570400000000006D
:10B020000828EC0044408000C30320000418E1001D
:10B0300071003E00000037000828EF0004002000E7
:10B04000543F8900503F81007100E1006A003100E7
:10B0500000003700503F8100C48020000400400001
:10B060001004E0005F00320000003700503F810014
:10B070006600E1002400320000003700503F8100EC
:10B08000C48020000400400090427800503F8100BE
:10B09000E48120000400400010437800F427F80009
:10B0A000E5FF9F00F427F900F427F800F6FF9F0062
:10B0B000F427F900B04E020000000000503F81006C
:10B0C000E4812000040040001004E000070032008A
:10B0D00000003700503F8100E481200084024000DE
:10B0E000804AEB008058040000000000503F8100BF
:10B0F000E48120008402400010C0B300804A780040
:10B10000F2580400000000001548E20035003A0043
:10B11000000037001248E200320032000000370021
:10B1200012C8BF00F427F800E0FF9F00F427F900E1
:10B13000A03F81000080FD0010C0B3000080FD0032
:10B14000A03F8900B04E02000000000012C8BF00FE
:10B15000EC27F800E0FF9F00EC27F900603F81003A
:10B16000EE27F800E0FF9F00EE27F900A856020046
:10B170000000000012E8B7001248E2001900320097
:10B1800000003700603F810012C8B6000004E000F4
:10B190000B003A00000037002448E20007003A00A4
:10B1A0000000370010C0B30024E8B7009A60A80080
:10B1B00013003700E0580400000000002468EF008E
:10B1C00012C8BF00F427F800E0FF9F00F427F90041
:10B1D000A03F81000160EF00A03F8900B04E020057
:10B1E00000000000503F81000000E800503F89004F
:10B1F00022580400000000008A60A9009A60A8009C
:10B200008A60A900A00120000C0009004F107800FE
:10B210004F0078003600F9004200F90000400600B7
:10B220000000E0004220AF0004003700793E090032
:10B23000000000000000E900F9FF370000000600F0
:10B24000C4F080006124E10004003A00D842A90063
:10B25000DC42A9003259040000000000D842A900D5
:10B26000DC42A800D802A900DC02A800DC22A90068
:10B27000D822A9001E0009000000000019DEBF004E
:10B28000C8E2B7001E00090000000000DC22A80090
:10B29000D822A9001E0009000000000000000600DE
:10B2A00000CBB30011FEB700121EA80084F080008E
:10B2B0006924E1000300360080C0B30010FEB7002F
:10B2C000121EA90011DEBF00105EB40011FEB7000F
:10B2D00010C0B30018FEB70011DEBF0019FEB700A2
:10B2E00020590200000000000040EB00121EAF00D9
:10B2F0000000E80000000600851F7800117EEF00C6
:10B30000127EEF00131EA80084F080003308200096
:10B31000041CE1000300310030C8B30010FEB70088
:10B32000131EA90010DEBF0011FEB70010DEBF0023
:10B330000160EF004400DE007040700012FEB700B4
:10B3400010C0B30018FEB70012DEBF0019FEB70030
:10B350002059020000000000A00020001059020047
:10B360000000000010DEBF00EF42600010C0B3001C
:10B3700018FEB7000540780019FEB70020590200FA
:10B3800000000000A0002000105902000000000092
:10B390000040EB00131EAF000000E800CF02780071
:10B3A00000000600F17BEF00F27BEF0084DF8000FD
:10B3B0006824E1000400360080C0B300F1FBB70050
:10B3C000E859040000000000F0DBBF00F1FBB7000B
:10B3D000F0DBBF0010FEB700505902000000000073
:10B3E000107EEF007C59020000000000F27BEF00AD
:10B3F00094DF800043082000041CE10007003600B1
:10B40000187EEF00197EEF002059020000000000B6
:10B41000F27BEC00F85904000000000010C0B300FB
:10B4200000E0B70000000600BE7BEF00BE7BEF002F
:10B43000F4DD80006924E10007003100BEDBBF00BD
:10B44000F0FBB700D259020000000000BE7BEC0008
:10B45000185A04000000000000000600BC3BEF008A
:10B4600010C0B30018FEB700E0CAB30019FEB70061
:10B470002059020000000000D862A900DC62A90087
:10B480003E01090000000000D862A900DC62A800AB
:10B49000803E20001059020000000000C602F800A3
:10B4A000BC1BF90000F02F00BC3BB600BC1BF80031
:10B4B000C602F9001E0009000000000010C0B30021
:10B4C00018FEB70080C2B30019FEB7002059020071
:10B4D0000000000010C0B30018FEB70020CEB3007B
:10B4E00019FEB700205902000000000010C0B30090
:10B4F00018FEB70000C1B30019FEB70020590200C2
:10B500000000000010C0B30018FEB700197EEF0065
:10B51000205902000000000010C0B30018FEB70060
:10B5200000CBB30019FEB700205902000000000054
:10B5300010C0B30018FEB70000C4B30019FEB70076
:10B54000205902000000000010C0B30018FEB70030
:10B5500010CAB30019FEB700205902000000000015
:10B5600010C0B30018FEB70000CCB30019FEB7003E
:10B57000205902000000000010C0B30018FEB70000
:10B58000F0CAB30019FEB700205902000000000005
:10B5900040062000105902000000000010C0B30057
:10B5A00018FEB70070CEB30019FEB7002059020094
:10B5B00000000000145A02000000000020032000D8
:10B5C000105902000000000000000600851F7800EE
:10B5D000137EEF00147EEF0094F080000302200041
:10B5E000041CE10020003E0094F08000F3032000E2
:10B5F000041CE1001C00390094F080000442B100FA
:10B600000440780013FEB700147EEF00A4F0800021
:10B610006524E1001200310094F080004822DE0031
:10B620006520B80080027800A4F080000960EF0077
:10B63000048042006425210004004000904278000C
:10B64000187EEF000540780019FEB700205902006F
:10B6500000000000147EEC00065B04000000000007
:10B66000F25B04000000000094F08000030420005E
:10B67000041CE10020003E0094F08000F30520004F
:10B68000041CE1001C00390094F080000444B10067
:10B690000440780013FEB700147EEF00A4F0800091
:10B6A0006524E1001200310094F080004822DE00A1
:10B6B0006520B80080027800A4F080000960EF00E7
:10B6C00004804200642F2100040040009042780072
:10B6D000187EEF000540780019FEB70020590200DF
:10B6E00000000000147EEC004E5B0400000000002F
:10B6F000F25B04000000000094F0800003062000CC
:10B70000041CE10020003E0094F08000F3072000BC
:10B71000041CE1001C00390094F080000446B100D4
:10B720000440780013FEB700147EEF00A4F0800000
:10B730006524E1001200310094F080004822DE0010
:10B740006520B80080027800A4F080000960EF0056
:10B7500004804200643921000400400090427800D7
:10B76000187EEF000540780019FEB700205902004E
:10B7700000000000147EEC00965B04000000000056
:10B78000F25B040000000000137EEF00147EEF0067
:10B79000A4F080006524E1001200310094F08000E4
:10B7A0004822DE006520B80080027800A4F0800006
:10B7B0000960EF000480420064252100040040007D
:10B7C00090427800187EEF000540780019FEB7001F
:10B7D0002059020000000000147EEC00C85B040049
:10B7E0000000000010C0B30000E0B700CF027800F6
:10B7F00000000600851F7800097EEF0004DEBF0010
:10B8000010FEB700505902000000000005DEBF0026
:10B8100010FEB7007C59020000000000097EEF0016
:10B8200009DEBF0044F080000024E1001500340070
:10B8300044F080004822DE0004007800061EB400B8
:10B8400090427800121EF800E5FF9F00121EF900DA
:10B85000E65A020000000000187EEF00197EEF009B
:10B860002059020000000000187EEF00197EEF0052
:10B870002059020000000000097EEC00105C04006A
:10B8800000000000CF02780000000600851F78004D
:10B89000C500200003000900B51F780000027800F1
:10B8A0008102780002037800830378000000EB0037
:10B8B0008000EB000001EB008001EB000800A1001C
:10B8C00007F0A600050037000800A0000402EA0007
:10B8D0008582EA000683EA008783EA008504720015
:10B8E00002003A0087047300150032003947200037
:10B8F0000340A7000B0037004200A9000482D200D9
:10B900008582D2000683D2008783D2000080D200D5
:10B910008180D2000281D2008381D2008904E900B3
:10B92000F3FF3A00C44CDD004200A90009F0A10079
:10B930000340A10083816C000800A70003F0A00071
:10B940002501200003000900CF127800CF02780003
:10B9500000000600881F780028012000040009006C
:10B96000B81F78008005EB006066B800030478001B
:10B9700087047800FA7F20004200A9004220A90035
:10B9800044C4DE00080465000800E00070003200D6
:10B990004200A9004220A900C4CCDE008904650051
:10B9A0000900E0006A0032000884440009B0A700E2
:10B9B00004003700F83FB100650032006400390030
:10B9C000030037001A402000854245006000310026
:10B9D000878669004200A9004220A900F300B20056
:10B9E0000340A000F700B2000740A000881F7800C5
:10B9F0000124B800002DB8000A0544008B854C00D6
:10BA00000C80B0000224B8008B0544000C864C006A
:10BA1000012CB8008B0544000C864C000034B800A3
:10BA20000005EB008B0544000C864C000A80B0003A
:10BA30008005EB000324B8000C0644000A854C0086
:10BA40000B80B000022CB8000C0644000A854C00A4
:10BA50000B80B0000134B8000C0644000A854C008D
:10BA60000B80B000003CB8000C0644000A854C0076
:10BA70000B80B0000C0078000006EB00032CB8002F
:10BA80000A0544008B854C000C80B0000234B800DD
:10BA90000A0544008B854C000C80B0000334B800CC
:10BAA0008B0544000C864C00013CB8000A0544009C
:10BAB0008B854C000C80B000023CB8008B05440024
:10BAC0000C864C00033CB8000C0644008A00780049
:10BAD0000B0178008C017800540020004200A9007E
:10BAE0008381D3000281D3008180D3000080D30002
:10BAF0000402E900F9FF3A004F0478000804E80066
:10BB000001037000010032000200370003037100DE
:10BB1000080032000340A700060037004200A900D9
:10BB20000080D2008180D2000281D2008381D200C5
:10BB30000804E9004444DD0003F0A1000DF0A70073
:10BB400003F0A0000340A10083016C000300370054
:10BB50006000B8006001B80000003700A8012000B4
:10BB6000040009004F1478004F047800000006001C
:10BB7000881F78002801200004000900B81F780001
:10BB8000878669000304780087047800FA7F200024
:10BB90004200A9004220A90044C4DE000804650058
:10BBA0000800E0006C0032004200A9004220A90019
:10BBB000C4CCDE00890465000900E00066003200A4
:10BBC0000005EB000906540003003900FC3FB000FB
:10BBD00061003100040037001B4020000B065600B6
:10BBE0005D0039005C0032000004EB008004EB00D3
:10BBF0000005EB008005EB00F301B2000340A0005C
:10BC0000F701B2000740A0008C1F78006C032000F1
:10BC100004005000858058000601590087815900B2
:10BC2000020033000600310006003A000400400024
:10BC300085804800060149008781490001003700DE
:10BC40000800A0000C06E9000B0032004200A90029
:10BC50000080D2008180D2000281D2008381D20094
:10BC60004200A9000884D2008984D2000A85D2004B
:10BC70008B85D200E6FF37004F0678000B50A700F7
:10BC800001003700060037004200A9008B85D30071
:10BC90000A85D3008984D3000884D30003003700C9
:10BCA0000C06E9004200A9002B0032004200AF0060
:10BCB000090037000080D2008180D2000281D200CA
:10BCC0008381D20004025000858258000603590087
:10BCD00087835900150039000804E80013003A0072
:10BCE0008904E80011003A000A05E8000F003A0054
:10BCF0008B05E8000D003A000C06E8001600320043
:10BD00000A0037000C06E900130032000B40A700C0
:10BD1000060037004200A9000884D2008984D200BE
:10BD20000A85D2008B85D200F8FF37004466DD001B
:10BD30004200A9000CF0A1000DF0A7000CF0A0003B
:10BD40000B40A1008B016E000A0178008900780089
:10BD500008007800050037000000200001002000E6
:10BD6000020020000300200000003700A80120008E
:10BD7000040009004F1478004F047800000006000A
:10BD8000851F7800861F780003027800030378007F
:10BD90004200A90044A2DE00F57F20000482620078
:10BDA00003003A006000B8000001EB001300370008
:10BDB0000438B100F300B200370020004200A900AF
:10BDC0000080D2008180D2000281D2008381D20023
:10BDD0008703E900F9FF3A0001007800820078004B
:10BDE0000370A1000480FD004200A9000482D3007A
:10BDF00006F0A70004F0A00003016A004F037800DA
:10BE0000CF02780000000600811F780091DB8000DF
:10BE1000805878008048EB00CF007800723BEC003F
:10BE200000000600851F78008201780082027800F9
:10BE30004200A9008381D2000380FD00F30FB2000D
:10BE400003003A006000B8006011B8001600370027
:10BE50000338B000F207B200360020000002EB0009
:10BE60004200A9000281D3008180D3000080D3006A
:10BE70004200AF000402E8000603E900F8FF3A00C0
:10BE80000270A100C419DD0003F0A10005F0A700B5
:10BE900003F0A000830169000101780080007800B0
:10BEA000810042000000EB00CF0278000000060095
:10BEB000851F7800C500200005000900B51F780027
:10BEC0000304780082037800010378008002780080
:10BED000830478003B472000C499DE00FA7F2000ED
:10BEE0008301650083855500F801B2000840A00079
:10BEF0000000EB008000EB000001EB008001EB0094
:10BF00004200A9000884D3008783D3000683D300AE
:10BF10008582D3008381D3000281D3008180D30046
:10BF20000080D3008B05E900F5FF3A0009F0A60078
:10BF3000050037000000EA008180EA000281EA0083
:10BF40008381EA0000003700650120000500090038
:10BF5000CF127800CF027800000006008C1F780016
:10BF60008D1F78000004EB008004EB000005EB005F
:10BF70008005EB000006EB008006EB00E8002000E7
:10BF8000090020001000FA000C377C000884E9004A
:10BF9000FDFF3B0005046A0002003A0007046B0045
:10BFA0002F0032000004EB000D0420000D042000DF
:10BFB0004200A9000080D2008180D2000281D2001C
:10BFC0008381D2000884D2008984D2000A85D200FD
:10BFD0008B85D2000758E10005003A0006D0E10049
:10BFE00003003A0005C8E10001003A0004C0E10086
:10BFF000050039000404540085845C0006055D00DA
:10C0000087855D004200A800080F78001907980096
:10C010002A0798003B0798004E049000DE04900029
:10C020006E059000FE0590000884D2008984D2003D
:10C030000A85D2008B85D2004807980059079800DE
:10C040006A0798007B0798001E0478009E04900001
:10C050002E059000BE0590008D06E900D4FF3A0041
:10C060004E009000DE0090006E019000FE019000F6
:10C070000080FA0000003700CF0678004F067800F5
:10C0800000000600851F7800C50020000700090099
:10C09000B51F78002A00FA00880220000006EB0095
:10C0A0000C377C000884E900FDFF3B000900E0003C
:10C0B0000E003200391798004A17980047022400F2
:10C0C0000003EB006022B800291798004702240003
:10C0D0000003EB006022B800AA5C02000000000030
:10C0E000AE1490008904E900F7FF3A00BE149000F6
:10C0F0004001200020179800D71C240056D62C00A1
:10C100006022B800000F9800110F9800220F9800CD
:10C11000330F980048012000081798000400200001
:10C12000859E28004630220077AC2800440F9800F6
:10C13000550F9800660F9800770F980003F0A6003F
:10C14000040037004E1490000804E90008D0A00055
:10C150004817980003F0A100585F0200000000009B
:10C160004E149000BE1490000900E0004220AF0081
:10C170000844E800481798009E1490008004EB00E3
:10C18000191798004E0A9000DE0A90006E0B90007E
:10C19000FE0B9000AE5F0200000000009E169000B3
:10C1A0000D00A70060003700080F9800190F9800D5
:10C1B0002A0F98003B0F98009E1690000D00A200D9
:10C1C0001D1798000000E00012003A00BE14900015
:10C1D0008904E8002E159000090455000D00320076
:10C1E000CE1590000B00E0000E0032007F84650049
:10C1F00008045500010032003F0031000BF0A70099
:10C200003D0037000BE0A7000600370000022000C9
:10C2100034003700CE1590000C0022008B0566001C
:10C220004B179800CE1590000BD0A6000E003700DB
:10C230000BD0A100BE1490000900E0004220AE0027
:10C240008B05E9008005EB004B179800000578008E
:10C25000D0C2B300045F0200000000000A007800B2
:10C260008005EB004B179800BE1490002E1590002F
:10C27000090455000B003A008005EB004B179800AD
:10C2800000057800E0C2B300045F02000000000077
:10C29000CE1590000C0022008B0566004B1798000D
:10C2A0000A00780001032000CE1590000BD0A600F4
:10C2B0000C0037000BD0A100BE1490000900E00074
:10C2C0004220AE008B05E9008005EB004B1798007B
:10C2D000D0C2B300045F0200000000000000EB00C9
:10C2E0000103200000804000801F78004F0078008C
:10C2F000045F020000000000AE1690008D06E90009
:10C30000190032002D1798004E089000DE089000AA
:10C310006E099000FE099000A40020008002EB004E
:10C320006033B8009BFF3700400F9800510F980012
:10C33000620F9800730F9800000278008102780065
:10C3400002037800830378000E0890009E08900096
:10C350002E099000BE0990009E1690000D00A200CC
:10C360001D1798008BFF37000080FA00A501200000
:10C3700007000900CF127800CF0278000000060005
:10C38000F0FF2F000862AE000500370009C2AF00C1
:10C39000FEFF37001110880009C2AF00FEFF370012
:10C3A0000000200009E2AF000000E80000000600E5
:10C3B0000862AE00040037000622A8000622AF0083
:10C3C000FEFF3700030037000602A8000602AF0098
:10C3D000FEFF37009E0009000000000081EA800097
:10C3E000C0610200000000009E0009000000000083
:10C3F00051DDBF0080007800C06102000000000035
:10C400009E0009000000000091EA8000C061020067
:10C41000000000009E00090000000000F001200064
:10C420000602B600FDFF3A000642A8000642AF0031
:10C43000FEFF3700BE0009000000000000000600FB
:10C44000F0FF2F000862AE001100370032108000AC
:10C450007F016100FDFF3A000662A8000100A7000D
:10C4600006A2A9000100A60006A2A80032108000C2
:10C470007F016100FDFF3A000682A8000822AE009D
:10C48000FEFF37000010800008C2AF0008C2A900FC
:10C4900000000600851F7800527DEF000862AE00A4
:10C4A000040037000622A8000622AF00FEFF370076
:10C4B000030037000602A8000602AF00FEFF3700A7
:10C4C000BE0009000000000081EA8000C061020097
:10C4D00000000000BE0009000000000051DDBF00A8
:10C4E00080007800C061020000000000BE0009006A
:10C4F000000000000862AE00040037000622A80019
:10C500000622AF00FEFF3700030037000602A80036
:10C510000602AF00FEFF3700BE0009000000000069
:10C5200050DDBF00E142700085407800C06102002C
:10C5300000000000BE000900000000000100200013
:10C54000811F7800CF007800206202000000000008
:10C5500052FDB700BE00090000000000F0012000FD
:10C560000602B600FDFF3A000642A8000642AF00F0
:10C57000FEFF3700DE0009000000000052DDBF00B2
:10C5800000E0B700CF02780000000600BC7BEF009F
:10C5900040C4B30050FDB70080C1B30051FDB700E7
:10C5A00052FDEF00D86102000000000040C4B3005B
:10C5B00050FDB70090C1B30051FDB70052FDEF0030
:10C5C000D86102000000000040C4B30050FDB70075
:10C5D000A0C1B30051FDB70052FDEF00D8610200C9
:10C5E0000000000040C4B30050FDB700B0C1B3006C
:10C5F00051FDB70052FDEF00D861020000000000BD
:10C6000040C4B30050FDB700C0C1B30051FDB70036
:10C6100052FDEF00D86102000000000040C4B300EA
:10C6200050FDB70000C2B30051FDB700527DEF00CE
:10C63000D86102000000000040C4B30050FDB70004
:10C6400010C2B30051FDB700527DEF00D861020067
:10C650000000000040C4B30050FDB70020C2B3008A
:10C6600051FDB700527DEF00D861020000000000CC
:10C6700040C4B30050FDB70030C2B30051FDB70055
:10C68000527DEF00D86102000000000040C4B300FA
:10C6900050FDB70040C2B30051FDB700527DEF001E
:10C6A000D86102000000000040C4B30050FDB70094
:10C6B000517DEF004A62020000000000BCFBB700A1
:10C6C00040C4B30050FDB70010C0B30051FDB70027
:10C6D0004A62020000000000BCFBB70040C4B30087
:10C6E00050FDB70020C0B30051FDB7004A62020000
:10C6F00000000000BCFBB70040C4B30050FDB70011
:10C7000030C0B30051FDB7004A62020000000000D3
:10C71000BCFBB70040C4B30050FDB70040C0B3003D
:10C7200051FDB7004A62020000000000BCFBB700E8
:10C730004200F80042E0EF00E03F810080C1B3001A
:10C74000E03F8900E03F81000160EF00E03F8900A9
:10C75000504E0200000000004200F9004200F800C4
:10C7600042E0EF00E03F810090C1B300E03F89006C
:10C77000E03F81000160EF00E03F8900504E020081
:10C78000000000004200F9004200F80042E0EF0023
:10C79000E03F8100A0C1B300E03F8900E03F81009D
:10C7A0000160EF00E03F8900504E020000000000F1
:10C7B0004200F9004200F80042E0EF00E03F810053
:10C7C000B0C1B300E03F8900E03F81000160EF00AD
:10C7D000E03F8900504E0200000000004200F900D6
:10C7E0004200F80042E0EF00E03F8100C0C1B3002A
:10C7F000E03F8900E03F81000160EF00E03F8900F9
:10C80000504E0200000000004200F9004200F80013
:10C8100042E0EF00E03F810000C2B300E03F89004A
:10C82000E03F810001E0EF00E03F8900504E020050
:10C83000000000004200F9004200F80042E0EF0072
:10C84000E03F810010C2B300E03F8900E03F81007B
:10C8500001E0EF00E03F8900504E020000000000C0
:10C860004200F9004200F80042E0EF00E03F8100A2
:10C8700020C2B300E03F8900E03F810001E0EF000B
:10C88000E03F8900504E0200000000004200F90025
:10C890004200F80042E0EF00E03F810030C2B30008
:10C8A000E03F8900E03F810001E0EF00E03F8900C8
:10C8B000504E0200000000004200F9004200F80063
:10C8C00042E0EF00E03F810040C2B300E03F89005A
:10C8D000E03F810001E0EF00E03F8900504E0200A0
:10C8E000000000004200F900F40F20007489880065
:10C8F0004200F80042E0EF00E03F810080C0B3005A
:10C90000E03F89002ED1BF00FC27F800F0FF9F0018
:10C91000FC27F900504E0200000000004200F90020
:10C92000F40F2000848988004200F80042E0EF0004
:10C93000E03F810090C0B300E03F890030D1BF00EC
:10C94000FC27F800F0FF9F00FC27F900504E020082
:10C95000000000004200F900F40F200094898800D4
:10C960004200F80042E0EF00E03F8100A0C0B300C9
:10C97000E03F890032D1BF00FC27F800F0FF9F00A4
:10C98000FC27F900504E0200000000004200F900B0
:10C99000F40F2000A48988004200F80042E0EF0074
:10C9A000E03F8100B0C0B300E03F890034D1BF0058
:10C9B000FC27F800F0FF9F00FC27F900504E020012
:10C9C000000000004200F900F40F2000B489880044
:10C9D0004200F80042E0EF00E03F8100C0C0B30039
:10C9E000E03F890036D1BF00FC27F800F0FF9F0030
:10C9F000FC27F900504E0200000000004200F90040
:10CA000000C4B30050FDB70040C0B30051FDB700F3
:10CA1000527DEF00D86102000000000000C4B300A6
:10CA200050FDB70050C0B30051FDB700527DEF007C
:10CA3000D86102000000000000C4B30050FDB70040
:10CA400060C0B30051FDB700527DEF00D861020015
:10CA50000000000000C4B30050FDB70070C0B30078
:10CA600051FDB700527DEF00D861020000000000C8
:10CA700000C4B30050FDB70020C0B30051FDB700A3
:10CA800052FDEF00D86102000000000000C4B300B6
:10CA900050FDB70030C0B30051FDB70052FDEF00AC
:10CAA000D86102000000000000000600851F780029
:10CAB000F03BEF00C0C0B3003EE9B70040C0B30098
:10CAC0003FE9B7004069EF004169EF0010C0B300D3
:10CAD00045E9B70010C0B30046E9B70020C1B30074
:10CAE00048E9B700F0C0B30047E9B70040C0B30061
:10CAF00049E9B70040C0B3004AE9B70040C0B300FD
:10CB00004BE9B70090C1B3004CE9B700E0C1B300F6
:10CB100068E9B700E0C1B30069E9B700E0C1B3005C
:10CB20006AE9B7004D69EF004E69EF004F69EF0009
:10CB300080C1B30050E9B70080C1B30051E9B7002C
:10CB400080C1B30052E9B70080C1B30053E9B70018
:10CB500080C1B30054E9B70080C1B30055E9B70004
:10CB600080C1B30056E9B70080C1B30057E9B700F0
:10CB700040C1B30058E9B70040C1B30059E9B7005C
:10CB800040C1B3005AE9B70040C1B3005BE9B70048
:10CB900040C1B3005CE9B70040C1B3005DE9B70034
:10CBA00040C1B3005EE9B70040C1B3005FE9B70020
:10CBB00070C0B30060E9B70070C0B30061E9B700AE
:10CBC00070C0B30062E9B70070C0B30063E9B7009A
:10CBD00070C0B30064E9B70070C0B30065E9B70086
:10CBE00070C0B30066E9B70070C0B30067E9B70072
:10CBF0006B69EF006C69EF006D69EF006E69EF0023
:10CC00006F69EF007069EF007169EF007269EF0002
:10CC1000A0C0B30092E8B700F03BEF0084DF8000D3
:10CC20006F20E10007003100C498200083DF8000FE
:10CC300084824100804AEB00F03BEC000E66040069
:10CC400000000000CF02780000000600851F780079
:10CC5000EF7DEF000862AE00040037000622A80056
:10CC60000622AF00FEFF3700030037000602A800CF
:10CC70000602AF00FEFF3700BE0009000000000002
:10CC800001CAB300C061020000000000BE0009003C
:10CC900000000000F1DDBF008002780085407800D0
:10CCA000C06102000000000085EF80008540780030
:10CCB000C061020000000000BE000900000000008A
:10CCC0000862AE00040037000622A8000622AF006A
:10CCD000FEFF3700030037000602A8000602AF007F
:10CCE000FEFF370011CAB300C0610200000000005F
:10CCF000BE0009000000000001002000811F780034
:10CD0000CF0078002062020000000000EFFDB700B5
:10CD1000F00120000602B600FDFF3A000642A8001E
:10CD20000642AF00FEFF3700DE00090000000000F1
:10CD3000EFDDBF00CF02780000000600851F7800FD
:10CD4000D85BE20021003200A0DE80009042780033
:10CD5000B0DE80000002780014407800002CE10072
:10CD60000E003200A0DE800090427800B0DE80002D
:10CD70000002780014407800002CE100030031002C
:10CD800000C0EB00C86604000000000010C0B30043
:10CD90000F003700D866040000000000A0DE80000D
:10CDA0001004E00002003A000060EF0008003700C5
:10CDB000A0DE8000D43BEC00B0DE8000D63BEC006F
:10CDC000D87BED00A0660400000000000060EF00CA
:10CDD000CF02780000000600851F7800BC3BEF0002
:10CDE000BE7BEF00BF7BEF000402220004DE880060
:10CDF0000402220014DE88000402220024DE8800DF
:10CE00000402220034DE88000402220044DE88008E
:10CE10000402220054DE88000402220064DE88003E
:10CE20000402220074DE88000402220084DE8800EE
:10CE3000D27BEF00F4FC2100E4DD8800BE7BEF0034
:10CE4000F4DD80007224E1001600310000CAB30056
:10CE5000EEFDB700BC1BF800F01DF90026660200CD
:10CE600000000000BFFBB700500020001059020076
:10CE700000000000F4DD80000960EF0003BC210029
:10CE800083024200BFDBBF00804A7800E4DD8000FF
:10CE900061024200E4DD8800BE7BEC0020670400F4
:10CEA00000000000D27BEF0020C1B300D8FBB70028
:10CEB00004BC2100A4DE880064852000B4DE880064
:10CEC0009E660200000000000004E00005003A0039
:10CED00010C0B30000E0B70004003700766704001C
:10CEE0000000000000E0EF0000003700CF027800F3
:10CEF00000000600851F7800041EF8000A1EF900D5
:10CF0000085EE2000C00320030F080001004E00007
:10CF10000900320050F080000A3EEC0080027800E8
:10CF200030F08000063EEC00904A7800087EED006C
:10CF30008067040000000000085EE2000700320085
:10CF400050F080000A3EEC0080027800804AEB003E
:10CF5000087EED009C67040000000000041EF8003D
:10CF60000000F900CF0278000000060001DF210078
:10CF700002002000120009008058EB0020C1B3001D
:10CF800008FEB70004DF210024F08800EE1DF80041
:10CF9000061EF9007A6702000000000070C0B300AE
:10CFA00004FEB700057EEF0020C1B30008FEB70005
:10CFB00004DF210034F08800FA5B0200000000006A
:10CFC00000000600851F78000862AE0004003700EC
:10CFD0000622A8000622AF00FEFF3700030037003C
:10CFE0000602A8000602AF00FEFF3700BE000900DF
:10CFF0000000000001CAB300C06102000000000090
:10D00000BE00090000000000F3DDBF0080027800D0
:10D0100085407800C06102000000000095EF8000AC
:10D0200085407800C0610200000000009E000900F9
:10D0300000000000F1DDBF0080007800C061020048
:10D04000000000009E00090000000000F001200028
:10D050000602B600FDFF3A000642A8000642AF00F5
:10D06000FEFF3700BE00090000000000CF0278007C
:10D0700000000600F23DEF00F17DEF00F23DEF0011
:10D0800090EF800084EF80000960EF000020E10055
:10D090000B00360090EF8000EE1DB4000002780017
:10D0A00014407800F17DB4005000200010590200B7
:10D0B00000000000F23DEC004068040000000000A9
:10D0C00084EF80004822DE00F4CFB20004407800F4
:10D0D000F1FDB70084EF80004822DE00614242008B
:10D0E00004407800F1FDB700F1DDBF00000006004C
:10D0F000851F7800D23DEF00D17DEF00E87DEF0085
:10D10000E91DA900D23DEF0090EE800084EE800082
:10D110000960EF000020E1002200360000CAB300E1
:10D12000EEFDB700D21DF800F01DF90026660200E2
:10D1300000000000E8FDB70090EE8000CE1DB400B6
:10D140000002780014407800E85DE300120032002D
:10D15000A0002000105902000000000090EE8000A6
:10D16000CE1DB4009042780000CAB300F0FDB700B5
:10D1700005407800F1FDB700D21DF800F21DF9005E
:10D18000E267020000000000A00020001059020029
:10D1900000000000E91DA800D23DEC0084680400F6
:10D1A00000000000E91DAE003E0037000200200034
:10D1B00041DD2100020078007A0202000000000038
:10D1C000805878000201E8000004E0004220AE0030
:10D1D000F8FF370044DD210074EF8800B6670200D5
:10D1E000000000003F09AE000D00370001002000E4
:10D1F000010078009A020200000000008100E800AF
:10D20000811F78002322AF00FEFF37002011880025
:10D21000CF007800D00020000008E600F4FF3700BF
:10D22000D0DDBF00F0FDB700CE1DF800EE1DF90007
:10D230003A68020000000000D1FDB70000CAB30048
:10D24000EEFDB700D0DDBF00F0FDB700F17DEF00CF
:10D250002666020000000000E8FDB700E8DDBF0020
:10D26000D15DE3000F003200A00020001059020041
:10D270000000000000CAB300F0FDB700D0DDBF0021
:10D28000F2FDB700F37DEF00D1DDBF00F1FDB70087
:10D29000E267020000000000A00020001059020018
:10D2A00000000000CF02780000000600851F780013
:10D2B000861F78000001EB000103780064C11000B4
:10D2C0004211DD000200DD00800278000C60EC00FD
:10D2D0000C60ED000D00320005007800C42ADD006E
:10D2E0004C00DE00F000B2000003B000A2032000FA
:10D2F0000200E100010039000D40B4002322AF001C
:10D30000FEFF370020118800F1FF37004F0378003F
:10D31000CF02780000000600851F7800D23DEF00A4
:10D32000D43DEF00D17DEF00D67DEF00D77DEF003B
:10D33000D87DEF00D91DA90000CAB300EEFDB700EB
:10D340001400200084EF8800266602000000000020
:10D35000D8FDB700B4EE80004822DE00F4CFB20062
:10D3600002003200D75DE20002003A00D0C0B300F4
:10D37000D8FDB700D43DEF00A4EE80006220E100AC
:10D38000A5003100D23DEF0090EE800084EE8000D9
:10D390000960EF000020E1005C00360090EE8000A4
:10D3A000CE1DB4008002780000CAB300EEFDB700C5
:10D3B000D21DF800F01DF9002666020000000000F2
:10D3C000804A7800D81DAE004A00370000CAB3007A
:10D3D000EEFDB700D21DF800F01DF9002666020030
:10D3E00000000000D7FDB70090EE8000CE1DB40015
:10D3F00010407800D75DE3003E003200D91DAF0039
:10D400000E003700D91DA80001002000010078009F
:10D4100000020200000000008100E800811F780087
:10D420002322AF00FEFF370020118800CF007800D4
:10D43000D00120000008E600F4FF370090EE8000E5
:10D44000CE1DB4009042780090EE80004170200024
:10D4500056690200000000002322AF00FEFF3700E3
:10D46000A4032000241188002322AF00FEFF370010
:10D470000402200024118800054078000160EF00BC
:10D480002170220056690200000000008100200087
:10D49000010078002C020200000000008100E8007A
:10D4A000811F78002322AF00FEFF37002011880083
:10D4B000CF007800B00020000008E600F4FF37003D
:10D4C000D7DDBF000160EF00217022005669020025
:10D4D000000000002322AF00FEFF3700A400200060
:10D4E000241188002322AF00FEFF3700D400200063
:10D4F0002411880050002000105902000000000094
:10D50000D23DEC00C46904000000000000CAB30072
:10D51000EEFDB700D0DDBF00F0FDB700F17DEF00FC
:10D520002666020000000000D6FDB700D0DDBF0077
:10D53000F0FDB700CE1DF800EE1DF9003A680200BC
:10D5400000000000D1FDB700D6DDBF00D15DE300D3
:10D550002E00320001002000010078004A02020083
:10D56000000000008100E800811F78002322AF0046
:10D57000FEFF370020118800CF007800D000200087
:10D580000008E600F4FF3700D6DDBF000160EF00C1
:10D5900021702200566902000000000011012000E5
:10D5A000010078004A020200000000008100E8004B
:10D5B000811F78002322AF00FEFF37002011880072
:10D5C000CF007800D00120000008E600F4FF37000B
:10D5D000D1DDBF000160EF0021702200566902001A
:10D5E000000000002322AF00FEFF3700A40020004F
:10D5F000241188002322AF00FEFF3700D400200052
:10D60000241188000060EF0005003700D43DEC00D5
:10D61000BC6904000000000010C0B30000E0B700C7
:10D62000CF02780000000600851F7800023CEF0062
:10D63000047CEF00057CEF00067CEF000404200072
:10D6400014E08800047CEF0024E080006724E100FF
:10D650001E003100057CEF0024E080004822DE003F
:10D660006E24E10016003100067CEF0034E08000FB
:10D670007624E1000F00310010E08000023CEC0055
:10D680008002780000CAB300F0FDB700F17DEF0022
:10D6900095EF8800E26702000000000050002000C3
:10D6A0001059020000000000067CEC00366B0400FC
:10D6B00000000000057CEC002C6B04000000000062
:10D6C000047CEC00246B040000000000047CEF00EC
:10D6D00024E080006F24E1000800310024E0800095
:10D6E0000960EF00C398200083024200804AEB00EB
:10D6F000047CEC00686B040000000000CF0278009E
:10D7000000000600851F7800023CEF00047CEF005B
:10D71000057CEF00C48A200014E08800047CEF0040
:10D7200024E080006E24E10015003100057CEF004C
:10D7300024E080004822DE0003022000041CE100F7
:10D740000C00360010E08000023CEC008002780003
:10D7500000CAB300F0FDB700F17DEF0095EF88003F
:10D76000E267020000000000057CEC00986B0400FA
:10D7700000000000047CEC00906B0400000000003E
:10D78000CF02780000000600851F7800BE3BEF0046
:10D79000C03BEF00F67BEF00F77BEF001423230084
:10D7A000C4DF8800D4A22400D4DF880014E6260059
:10D7B000E4DF8800D4122300F4DF88000403200093
:10D7C00004E08800C0C0B300C2FBB70040C0B30093
:10D7D000C3FBB700C47BEF00C57BEF0040C1B300C3
:10D7E000C6FBB70010C0B300C7FBB70010C0B30042
:10D7F000C8FBB70020C1B300C9FBB700F0C0B3003D
:10D80000CAFBB70040C0B300CBFBB70040C0B300B9
:10D81000CCFBB70040C0B300CDFBB70090C1B30054
:10D82000CEFBB700E0C1B300CFFBB700E0C1B3004F
:10D83000D0FBB700E0C1B300D1FBB700D27BEF0053
:10D84000D37BEF00D47BEF0080C1B300D5FBB700E2
:10D8500080C1B300D6FBB70080C1B300D7FBB700CF
:10D8600080C1B300D8FBB70080C1B300D9FBB700BB
:10D8700080C1B300DAFBB70080C1B300DBFBB700A7
:10D8800080C1B300DCFBB70040C1B300DDFBB700D3
:10D8900040C1B300DEFBB70040C1B300DFFBB700FF
:10D8A00040C1B300E0FBB70040C1B300E1FBB700EB
:10D8B00040C1B300E2FBB70040C1B300E3FBB700D7
:10D8C00040C1B300E4FBB70070C0B300E5FBB70094
:10D8D00070C0B300E6FBB70070C0B300E7FBB70051
:10D8E00070C0B300E8FBB70070C0B300E9FBB7003D
:10D8F00070C0B300EAFBB70070C0B300EBFBB70029
:10D9000070C0B300ECFBB700ED7BEF00EE7BEF00E7
:10D91000EF7BEF00F07BEF00F17BEF00F27BEF009D
:10D92000F37BEF00F47BEF00A0C0B300F5FBB70082
:10D9300040C3B300D0FDB70024BC210074EE8800C2
:10D94000786802000000000040C3B300D0FDB700BB
:10D9500024BC210074EE88008C69020000000000E5
:10D960006104E1001B00320040C3B300D0FDB700EA
:10D9700024BC210074EE88007868020000000000DA
:10D9800040C3B300D0FDB70024BC210074EE880072
:10D990008C690200000000006104E1000D0032000B
:10D9A0000100200001007800B60202000000000023
:10D9B0008100E800811F78002322AF00FEFF3700BE
:10D9C00020118800CF007800D00120000008E60078
:10D9D000F4FF3700146B020000000000826B0200AD
:10D9E00000000000F4FC2100F4DD8800F67BEF006D
:10D9F000B4DF80007324E1001B003100B4DF80003D
:10DA00000960EF00638520000300420010407800A9
:10DA1000F7FBB70000CAB300F0FDB700F7DBBF00AB
:10DA2000F1FDB700BE1BF800F21DF900E26702002D
:10DA30000000000000CAB300EEFDB700BE1BF800F6
:10DA4000F01DF9002666020000000000F7FBB70099
:10DA5000F4DD800061024200F4DD8800F67BEC001A
:10DA6000F86C04000000000014FE2100F4DD8800C2
:10DA7000C03BEF00F67BEF00B4DF80007324E100D1
:10DA800037003100B4DF80000960EF0023842000FC
:10DA90000300420090427800040320000524E100C6
:10DAA00004003E00940320000524E1000100390039
:10DAB000030037000040EB00626D0400000000002E
:10DAC00010C0B3006104E10022003A0004DE8000CF
:10DAD0006520E1001F003E00B4DF80000960EF0018
:10DAE000238420000300420010407800F7FBB700B9
:10DAF00000CAB300F0FDB700F7DBBF00F1FDB700CF
:10DB0000BE1BF800F21DF900E267020000000000F1
:10DB100050002000105902000000000000CAB300AD
:10DB2000EEFDB700BE1BF800F01DF90026660200EE
:10DB300000000000F7FBB700500020001059020061
:10DB400000000000C03BEC00F4DD800061024200F8
:10DB5000F4DD8800F67BEC003C6D04000000000062
:10DB600074FE2100F4DD8800F67BEF00B4DF800056
:10DB70006924E1001B003100B4DF80000960EF0080
:10DB800083BF21000300420010407800F7FBB7007C
:10DB900000CAB300F0FDB700F7DBBF00F1FDB7002E
:10DBA000BE1BF800F21DF900E26702000000000051
:10DBB00000CAB300EEFDB700BE1BF800F01DF9006F
:10DBC0002666020000000000F7FBB700F4DD8000CD
:10DBD00061024200F4DD8800F67BEC00B66D0400C3
:10DBE00000000000CF02780000000600851F7800CA
:10DBF00040C3B300D0FDB700C4BB210074EE880061
:10DC00008C690200000000000004E0001A003A00E5
:10DC100040C3B300D0FDB700C4BB210074EE880040
:10DC20008C690200000000000004E00012003A00CD
:10DC30003F09AE001000370001002000010078000D
:10DC4000E2020200000000008100E800811F78006D
:10DC50002322AF00FEFF370020118800CF0078009C
:10DC6000300120000008E600F4FF3700566502008E
:10DC7000000000006F003700BCDBBF003EE9B700CA
:10DC8000BDDBBF003FE9B700BEDBBF0040E9B70026
:10DC9000BFDBBF0041E9B700C0DBBF0042E9B7000E
:10DCA000144A800023032000041CE100020031001C
:10DCB00040C1B30042E9B700C1DBBF0045E9B7008E
:10DCC000C2DBBF0046E9B700C3DBBF0048E9B700CD
:10DCD000C4DBBF0047E9B700C5DBBF0049E9B700B7
:10DCE000C6DBBF004AE9B700C7DBBF004BE9B7009E
:10DCF000C8DBBF004CE9B700C9DBBF0068E9B7006B
:10DD0000CADBBF0069E9B700CBDBBF006AE9B70037
:10DD1000CCDBBF004DE9B700CDDBBF004EE9B7005B
:10DD2000CEDBBF004FE9B700CFDBBF0050E9B70043
:10DD3000D0DBBF0051E9B700D1DBBF0052E9B7002B
:10DD4000D2DBBF0053E9B700D3DBBF0054E9B70013
:10DD5000D4DBBF0055E9B700D5DBBF0056E9B700FB
:10DD6000D6DBBF0057E9B700D7DBBF0058E9B700E3
:10DD7000D8DBBF0059E9B700D9DBBF005AE9B700CB
:10DD8000DADBBF005BE9B700DBDBBF005CE9B700B3
:10DD9000DCDBBF005DE9B700DDDBBF005EE9B7009B
:10DDA000DEDBBF005FE9B700DFDBBF0060E9B70083
:10DDB000E0DBBF0061E9B700E1DBBF0062E9B7006B
:10DDC000E2DBBF0063E9B700E3DBBF0064E9B70053
:10DDD000E4DBBF0065E9B700E5DBBF0066E9B7003B
:10DDE000E6DBBF0067E9B700E7DBBF006BE9B70020
:10DDF000E8DBBF006CE9B700E9DBBF006DE9B70005
:10DE0000EADBBF006EE9B700EBDBBF006FE9B700EC
:10DE1000ECDBBF0070E9B700EDDBBF0071E9B700D4
:10DE2000EEDBBF0072E9B700EFDBBF0092E8B7009E
:10DE30008C28EF00CF027800000006003C32EF0093
:10DE40003C12F8003E12F900E1132100020020000C
:10DE5000FD0009008058EB0041C8A9000000060041
:10DE6000851F7800544C80004822DE00C3992000B2
:10DE700003004200B4E8800000429000B4E888004B
:10DE8000544C80004822DE00614242000440780089
:10DE900000E0B7000160EF00F40F2000110009005E
:10DEA0000480D800014078008BE9B7008BC9BF001F
:10DEB0007349E30001003A004148A90016DDBF00A4
:10DEC00000E0B700CF02780000000600851F780050
:10DED000127CEF004148AE0005003700306F0200B1
:10DEE0000000000012FCB7006A6F04000000000090
:10DEF0009B69EF00CF02780000000600851F7800C4
:10DF000080C5B30040FFB700D45880004822DE002F
:10DF1000C3A920000300420004FA800000429000E0
:10DF200004FA8800D45880004822DE006142420092
:10DF30000440780000E0B7000160EF00F407200023
:10DF4000110009000480D800014078001BEBB700E5
:10DF50001BCBBF009B4AE30001003A004168A900C7
:10DF600040DFBF0000E0B700CF02780000000600ED
:10DF7000851F7800347FEF004168AE00080037004D
:10DF80007E6F02000000000034FFB700A0002000F8
:10DF90001059020000000000BC6F040000000000E7
:10DFA0001C6BEF00CF02780000000600851F780090
:10DFB000C500200003000900B51F780000F0A6008E
:10DFC0000C0037000000EA000480A00004F0A60066
:10DFD00008003700801F7800D00220002322AF0005
:10DFE000FEFF3700201188004F0078000480A10058
:10DFF0000860ED008002EB00800378008404780064
:10E0000004F0A1000404E00006003A0009F0A700B3
:10E0100002003700050020000F0037000500200037
:10E020000D003700E64252000A00390000032000CC
:10E0300009F0A600000220002322AF00FEFF3700F7
:10E04000201188008502E900FBFF3B0055002000FD
:10E050000100370084027800640020000580A700DA
:10E060000402E80005E0A00009F0A70005F0A00008
:10E0700008712200110009008883D8008270020014
:10E080000000000081037800883E20001100090094
:10E090008883D800827002000000000081037800AD
:10E0A00048062000110009008883D8008270020011
:10E0B0000000000081037800A80020001100090082
:10E0C0008883D80082700200000000000980A6004A
:10E0D00005003700D00220002322AF00FEFF3700EA
:10E0E000201188000980A1000003200000C040002A
:10E0F000500188002322AF00FEFF37002011880066
:10E1000022003700060320000000E0000E003A0065
:10E1100005E0A600160037000402E9000524E1002E
:10E12000020032004200AF00000006000000E000E4
:10E1300005003A0005E0A6000D00370005F0A60036
:10E14000060220000A00370005E0A1000980A600B1
:10E150000700370000057800D00220002322AF001E
:10E16000FEFF3700201188000980A1000A00780016
:10E1700000404300811F78002322AF00FEFF3700DC
:10E1800020118800CF007800000006002501200043
:10E1900003000900CF127800CF02780000000600CB
:10E1A000851F7800367FEF00377FEF0000002000EA
:10E1B000341FB4001040780037FFB700375FE2002B
:10E1C000320032003F29AE00080037002322AF00A2
:10E1D000FEFF3700D4002000241188002322AF0066
:10E1E000FEFF3700A40020002411880010C0B300F7
:10E1F00036FFB70036DFBF00B4F980004822DE00EA
:10E200000024E100210035003F29AE001000370056
:10E2100036DFBF000000FB00A4F9800004004000CE
:10E22000904278000B60EF0005007800217022001A
:10E2300056690200000000002322AF00FEFF3700F5
:10E2400004022000241188002C710400000000004A
:10E250007E3E09000000000036DFBF000000FB002A
:10E26000A4F9800004004000904278000540780046
:10E270003322AF00FEFF370034E2B7003562EF0013
:10E28000367FEC00FA70040000000000CF02780036
:10E2900000000600851F7800C5002000030009006B
:10E2A000B51F7800800378008404780004F0A10092
:10E2B0000400E00006003A0009F0A7000200370061
:10E2C000050020000F003700050020000D0037007A
:10E2D000E64252000A0039000003200009F0A600BF
:10E2E000000220002322AF00FEFF3700201188002B
:10E2F0008502E900FBFF3B005500200001003700CC
:10E30000840278006400200005E0A00009F0A70066
:10E3100005F0A00008712200110009008883D800D0
:10E32000C47102000000000081037800883E2000D4
:10E33000110009008883D800C471020000000000A9
:10E340008103780048062000110009008883D80066
:10E35000C47102000000000081037800A8002000C2
:10E36000110009008883D800C47102000000000079
:10E370000003200000C040002322AF00FEFF370052
:10E380002011880019003700060320000000E0007B
:10E390000E003A0005E0A6000D0037000402E90077
:10E3A0000524E100020032004200AF000000060038
:10E3B0000000E00005003A0005E0A6000400370078
:10E3C00005F0A600060220000100370005E0A100CC
:10E3D00000404300811F78002322AF00FEFF37007A
:10E3E00020118800CF0078000000060025012000E1
:10E3F00003000900CF127800CF0278000000060069
:10E40000851F7800861F78006E3EEF00703EEF009B
:10E410006B1EA9003F29AE000D003700010020004F
:10E42000010078002C280200000000008100E800B4
:10E43000811F78002322AF00FEFF370020118800E3
:10E44000CF007800E00020000008E600F4FF37006D
:10E450004168AF002F00370074F3800023032000D1
:10E460000320B8008002780064F380000520E100FA
:10E4700022003E003F29AE001E00370001002000B0
:10E480000100780048280200000000008100E80038
:10E49000811F78002322AF00FEFF37002011880083
:10E4A000CF007800A00020000008E600F4FF37004D
:10E4B00060F38000040020004A71020000000000A8
:10E4C000D100200001007800482802000000000070
:10E4D0008100E800811F78002322AF00FEFF370093
:10E4E00020118800CF007800300120000008E600ED
:10E4F000F4FF37000060EF00D90037002003200050
:10E5000010590200000000006E3EEC00287204006A
:10E510000000000041F38000020020006ADEBF001E
:10E520000160EF000000E900008009008058EB0066
:10E530003F29AE000C0037002322AF00FEFF37005A
:10E5400004022000241188002322AF00FEFF3700C0
:10E55000D4022000241188002322AF00FEFF3700E0
:10E5600004022000241188004168AF000700370032
:10E5700074F38000230320000320B8000003780018
:10E5800064F380000620E100940036004168AE008C
:10E590005F00370080F38000681EB40080027800BE
:10E5A0007E6F020000000000804A78006B1EAF0002
:10E5B0002B00370080F38000681EB4001042780002
:10E5C00004C9B2000500320080F38000681EB40068
:10E5D0001042780084C8B2001F003A0000002000FA
:10E5E000681EB4008002780080F38000681EB400CA
:10E5F000904A78001400200084F388003F29AE0080
:10E600001400370000002000681EB400904278001B
:10E610002322AF00FEFF3700B4052000241188003C
:10E620002322AF00FEFF37000402200024118800DF
:10E63000054078000160EF0021702000566902005B
:10E64000000000002322AF00FEFF3700040220007C
:10E65000241188006B1EA8008873040000000000CD
:10E660003F29AE000C00370080F38000681EB40024
:10E6700090427800054078000160EF002170200092
:10E6800056690200000000002322AF00FEFF3700A1
:10E69000040220002411880080F38000681EB4006A
:10E6A00010427800F4CFB20011003A003F29AE00CA
:10E6B0000C0037002322AF00FEFF3700D4052000F6
:10E6C000241188002322AF00FEFF3700A4002000A1
:10E6D000241188002322AF00FEFF3700D400200061
:10E6E0002411880010C0B30000E0B7005C003700C0
:10E6F000703EEC006ADEBF000160EF0084F3800032
:10E700000020E1000200390000E0EF005400370073
:10E710004168AF002F00370074F38000230320000E
:10E720000320B8008002780064F380000520E10037
:10E7300022003E003F29AE001E00370001002000ED
:10E740000100780048280200000000008100E80075
:10E75000811F78002322AF00FEFF370020118800C0
:10E76000CF007800A00020000008E600F4FF37008A
:10E7700060F38000040020004A71020000000000E5
:10E78000D1002000010078004828020000000000AD
:10E790008100E800811F78002322AF00FEFF3700D0
:10E7A00020118800CF007800300120000008E6002A
:10E7B000F4FF37000060EF0029003700200320003D
:10E7C00010590200000000006E3EEC008873040047
:10E7D00000000000B4720400000000003F29AE00F9
:10E7E0001E003700010020000100780048280200C8
:10E7F000000000008100E800811F78002322AF00A4
:10E80000FEFF370020118800CF007800A000200014
:10E810000008E600F4FF370060F3800004002000E9
:10E820004A71020000000000D100200001007800C1
:10E8300048280200000000008100E800811F7800E5
:10E840002322AF00FEFF370020118800CF007800A0
:10E85000300120000008E600F4FF37000060EF0000
:10E860004F037800CF02780000000600851F780073
:10E870003F29AE000D0037000100200001007800A4
:10E88000E2270200000000008100E800811F7800FC
:10E890002322AF00FEFF370020118800CF00780050
:10E8A000D00020000008E600F4FF3700D0C0B3001D
:10E8B0006AFEB70084E5210044F38800561EF80084
:10E8C0006C1EF90000720200000000000004E0006D
:10E8D0002200320059DEBF000160EF001084B20058
:10E8E000110032003080B2000F0032002082B200EE
:10E8F000120032008085B200140032008086B2001F
:10E90000120032001080B200100032003080B200DD
:10E910000E0032003083B2000C0032003080B200B2
:10E920000A0032000B00370010C0B30000E0B7004F
:10E930000B003700AA7404000000000000E0EF00A4
:10E9400007003700AA74040000000000AA74040045
:10E950000000000056740400000000000060EF009A
:10E96000CF02780000000600851F780064102800A0
:10E97000F4F188001440200004F2880074002000A4
:10E9800014F2880044FEEF009410280034F288004E
:10E990001460200044F288001400200054F2880023
:10E9A0000430200064F2880034F02F0074F28800F4
:10E9B000517EEF00D4F18000F447B20004407800AB
:10E9C0003DFEB700D4F180004822DE00F447B200DB
:10E9D0000440780045FEB700E4F18000F447B2003F
:10E9E0000440780050FEB700444980006E24E100E6
:10E9F0000C003A00505EE2000A00320084448000BD
:10EA00000960EF00430D200004804100C48820000D
:10EA10000400400010407800F047B20068407000E9
:10EA200050FEB7003D5EE20006003A0010C0B300A1
:10EA30003DFEB70030C0B3004DFEB700387504008E
:10EA4000000000003ADEBF000048B20004082000C9
:10EA50000024E10004003A0010C0B3004DFEB700EE
:10EA6000387504000000000020C0B3004DFEB70060
:10EA70003DDEBF004BFEB700455EE20006003A00F7
:10EA800030C0B3004EFEB70010C0B30045FEB70063
:10EA900062750400000000003BDEBF000048B200C9
:10EAA000040820000024E10004003A0010C0B30074
:10EAB0004EFEB700627504000000000020C0B300E5
:10EAC0004EFEB70045DEBF004CFEB7004449800053
:10EAD0006A24E1003A00320064F280004822DE003D
:10EAE0006324E10003003A0074F280006324E10033
:10EAF000240032008C88A800B86F020000000000DB
:10EB000064E42100A4F98800D07002000000000035
:10EB1000444980006124E100030032004449800040
:10EB20006524E10006003A00843E2000B4F288002B
:10EB30003674020000000000BE75040000000000F2
:10EB4000444980006324E1000C003A003FA9AE0074
:10EB50000A003700A40F2000B4F2880036740200C7
:10EB60000000000042C9BF0051FEB70051DEBF00E7
:10EB70000160EF001059020000000000DC75040085
:10EB8000000000008C88AE000B0037008C88A900C4
:10EB9000B86F02000000000064E42100A4F98800BE
:10EBA000D070020000000000843E2000B4F2880013
:10EBB0003674020000000000B86F02000000000080
:10EBC000505EE20003003A00437EEF000E76040040
:10EBD0000000000050DEBF006740600050FEB7003C
:10EBE0003CDEBF000048B200040820000024E10021
:10EBF00006003A0084F280000442B300044078002A
:10EC000043FEB7000E7604000000000084F280008E
:10EC10000443B3000440780043FEB700435EE200C3
:10EC20002D003200444980006E24E10003003A00C8
:10EC30008CA8AE000100370036003700B86F020024
:10EC400000000000E4E32100A4F98800D070020075
:10EC5000000000008CA8A800444980006124E10065
:10EC600006003200444980006524E10003003200C0
:10EC7000444980006A24E10006003A00843E2000F6
:10EC8000B4F28800367402000000000068760400C8
:10EC900000000000444980006324E1000C003A00B9
:10ECA0003FA9AE000A003700A40F2000B4F288008C
:10ECB000367402000000000042C9BF0051FEB700D8
:10ECC00051DEBF000160EF0010590200000000009B
:10ECD00086760400000000008CA8AE000B00370010
:10ECE0008CA8A900B86F020000000000E4E3210036
:10ECF000A4F98800D070020000000000843E2000CB
:10ED0000B4F288003674020000000000B86F020000
:10ED100000000000CF02780000000600851F780088
:10ED2000C83EEF00C57EEF00CA1EA9004168AF00D3
:10ED30002F00370044F68000230320000320B80092
:10ED40008002780034F680000520E10022003E00B9
:10ED50003F29AE001E0037000100200001007800AE
:10ED600048280200000000008100E800811F7800B0
:10ED70002322AF00FEFF370020118800CF0078006B
:10ED8000A00020000008E600F4FF370030F6800005
:10ED9000040020004A71020000000000D1002000A1
:10EDA0000100780048280200000000008100E8000F
:10EDB000811F78002322AF00FEFF3700201188005A
:10EDC000CF007800300120000008E600F4FF370093
:10EDD0000060EF00D6003700200320001059020029
:10EDE00000000000C83EEC00967604000000000021
:10EDF00011F6800002002000C4DEBF000160EF00B9
:10EE00000000E900008009008058EB003F29AE00B7
:10EE10000C0037002322AF00FEFF37000402200061
:10EE2000241188002322AF00FEFF3700D402200007
:10EE3000241188002322AF00FEFF370004022000C7
:10EE4000241188004168AE009800370024F6800045
:10EE50004822DE0004007800C21EB4008002780060
:10EE60007E6F020000000000804A7800CA1EAF00DA
:10EE70002A00370024F680004822DE0004007800D3
:10EE8000C21EB40010427800E4CFB20021003A0064
:10EE900000002000C21EB4008002780024F680002A
:10EEA0004822DE0004007800C21EB400904A7800B8
:10EEB00010C0B300C5FEB7003F29AE0014003700F4
:10EEC00000002000C21EB400904278002322AF0050
:10EED000FEFF3700B4052000241188002322AF0074
:10EEE000FEFF37000402200024118800054078004E
:10EEF0000160EF0021702000566902000000000050
:10EF00002322AF00FEFF37000402200024118800F6
:10EF1000CA1EA800F0770400000000003F29AE00E0
:10EF20000E00370024F680004822DE00040078003E
:10EF3000C21EB40090427800054078000160EF00E6
:10EF40002170200056690200000000002322AF005B
:10EF5000FEFF3700040220002411880024F6800000
:10EF60004822DE0004007800C21EB400104278007F
:10EF7000F4CEB20012003A003F29AE000D00370077
:10EF80000100200001007800F029020000000000CC
:10EF90008100E800811F78002322AF00FEFF3700C8
:10EFA00020118800CF007800300020000008E60023
:10EFB000F4FF370010C0B30000E0B7005C0037007A
:10EFC000C57EEC00C4DEBF0024F680004822DE00CF
:10EFD0000024E1000200390000E0EF005400370097
:10EFE0004168AF002F00370044F680002303200063
:10EFF0000320B8008002780034F680000520E1008C
:10F0000022003E003F29AE001E0037000100200014
:10F010000100780048280200000000008100E8009C
:10F02000811F78002322AF00FEFF370020118800E7
:10F03000CF007800A00020000008E600F4FF3700B1
:10F0400030F68000040020004A7102000000000039
:10F05000D1002000010078004828020000000000D4
:10F060008100E800811F78002322AF00FEFF3700F7
:10F0700020118800CF007800300120000008E60051
:10F08000F4FF37000060EF00290037002003200064
:10F090001059020000000000C83EEC00F0770400A8
:10F0A0000000000022770400000000003F29AE00AD
:10F0B0001E003700010020000100780048280200EF
:10F0C000000000008100E800811F78002322AF00CB
:10F0D000FEFF370020118800CF007800A00020003C
:10F0E0000008E600F4FF370030F68000040020003E
:10F0F0004A71020000000000D100200001007800E9
:10F1000048280200000000008100E800811F78000C
:10F110002322AF00FEFF370020118800CF007800C7
:10F12000300120000008E600F4FF37000060EF0027
:10F13000CF02780000000600851F78003F29AE004E
:10F140000D0037000100200001007800022A0200B3
:10F15000000000008100E800811F78002322AF003A
:10F16000FEFF370020118800CF007800B00020009B
:10F170000008E600F4FF3700D0C0B300C4FEB700BB
:10F1800024EB210014F68800B01EF800C61EF9001A
:10F190008E760200000000000004E0002200320031
:10F1A000B5DEBF000160EF000083B200090032004D
:10F1B0003080B2000C0032006080B2000F003200DC
:10F1C000C080B2000D0032008080B2000F0032001B
:10F1D0000A00370010C0B30000E0B700130037008A
:10F1E00010790400000000002849E20003003A0002
:10F1F00010C0B30000E0B7000C00370000E0EF00E3
:10F200000A003700107904000000000010C0B300AD
:10F2100000E0B7000500370010790400000000008E
:10F22000BC780400000000000060EF00CF0278000E
:10F2300000000600117FEF0084F880006A24E100DE
:10F24000060031000403200083F8800004C0410060
:10F2500011FFB7003679040000000000740320009D
:10F2600083F8800004C0410011FFB70011DFBF0028
:10F2700000000600851F7800963EEF00E4F02F00A6
:10F28000C4F4880004032300D4F488001410280078
:10F29000E4F4880044032300F4F4880044032300CA
:10F2A00004F588004403230014F588004403230078
:10F2B00024F58800F0CEB300A6FEB70064F4800009
:10F2C000F447B200044078008FFEB70064F4800079
:10F2D0004822DE00F447B20004407800A7FEB700E1
:10F2E0008EDEBF0067406000A8FEB7008F5EE200C0
:10F2F00020003A00A75EE2001E003A00A85EE2008D
:10F300001C003A00F44880004822DE0004C3B2002A
:10F3100007003A000449800004C3B20004003A0028
:10F32000044980004822DE0004C3B200110032000C
:10F33000B86F02000000000084E92100A4F98800F1
:10F34000D070020000000000843E200084F5880098
:10F350009C7802000000000000C3B3001FE9B70062
:10F3600000C3B30020E9B70000C3B30021E9B70030
:10F370008C88A9008F5EE20005003A00A75EE200DB
:10F3800003003A00A85EE20001003A001A013700CB
:10F3900074F480004822DE006124E1001800360089
:10F3A00074F480004822DE007824E1000600390071
:10F3B00080C1B3008FFEB700F4032000B4F48800CE
:10F3C000FC790400000000008FDEBF0096FEB7004D
:10F3D000977EEF00B4F48000F30320000320B80010
:10F3E00080027800050278008301200011000900E6
:10F3F0000382D800B0F4880096DEBF008FFEB7000D
:10F4000034F580004822DE006124E1001800360057
:10F4100034F580004822DE007424E1000600390043
:10F4200040C1B300A7FEB700F4032000B4F4880085
:10F43000347A040000000000A7DEBF0096FEB7008B
:10F44000977EEF00B4F48000F30320000320B8009F
:10F4500080027800050278004301200011000900B5
:10F460000382D800B0F4880096DEBF00A7FEB70084
:10F4700044F580006124E1001700360044F5800067
:10F480006724E1000600390070C0B300A8FEB70091
:10F49000F4032000B4F48800687A0400000000003F
:10F4A000A8DEBF0096FEB700977EEF00B4F48000A0
:10F4B000F30320000320B8008002780005027800E2
:10F4C00073002000110009000382D800B0F4880006
:10F4D00096DEBF00A8FEB7008F5EE20004003A008F
:10F4E00000C3B300A9FEB7008E7A0400000000003C
:10F4F0008CDEBF000048B200040820000024E100B8
:10F5000004003A0020C3B300A9FEB7008E7A0400BD
:10F510000000000010C3B300A9FEB700A75EE20020
:10F5200004003A0000C3B300AAFEB700B07A04009A
:10F53000000000008DDEBF000048B200040820007B
:10F540000024E10004003A0010C3B300AAFEB70093
:10F55000B07A04000000000020C3B300AAFEB70088
:10F56000A85EE20004003A0000C3B300ABFEB7009F
:10F57000D27A0400000000008EDEBF000048B20016
:10F58000040820000024E10004003A0010C3B30086
:10F59000ABFEB700D27A04000000000020C3B30025
:10F5A000ABFEB70044F580004822DE0014C3B20071
:10F5B00008003A00F403200073F48000C819DE004C
:10F5C0000340520092FEB700937EEF00027B0400DE
:10F5D0000000000044F580004822DE0024C3B20091
:10F5E00006003A00000420008F5EB40092FEB700CF
:10F5F000937EEF00027B0400000000000404200062
:10F6000094F4880054F5800014C3B20008003A0056
:10F61000F403200033F58000C819DE0003405200D7
:10F6200090FEB700917EEF002E7B040000000000EA
:10F6300054F5800024C3B20006003A000004200004
:10F64000A75EB40090FEB700917EEF002E7B040011
:10F65000000000000404200084F4880054F58000B9
:10F660004822DE0024C3B20007003A00F403200061
:10F6700043F580000340520094FEB700957EEF00F2
:10F680005C7B04000000000054F580004822DE008E
:10F6900014C3B20006003A0000042000A85EB400C3
:10F6A00094FEB700957EEF005C7B04000000000034
:10F6B00004042000A4F4880094DEBF000160EF0081
:10F6C0004400DE00EF426000101FF800E5FF9F00DD
:10F6D000101FF9001A790200000000009EFEB7001A
:10F6E00094DEBF00EF426000101FF800E5FF9F00AE
:10F6F000101FF9001A790200000000009FFEB700F9
:10F7000090DEBF000160EF004400DE00EF426000C9
:10F71000101FF800E5FF9F00101FF9001A79020082
:10F7200000000000A2FEB70090DEBF00EF426000C4
:10F73000101FF800E5FF9F00101FF9001A79020062
:10F7400000000000A3FEB70092DEBF000160EF00E2
:10F750004400DE00EF426000101FF800E5FF9F004C
:10F76000101FF9001A79020000000000A4FEB70083
:10F7700092DEBF00EF426000101FF800E5FF9F001F
:10F78000101FF9001A79020000000000A5FEB70062
:10F790008FDEBF001CE9B700A9DEBF001FE9B7007C
:10F7A000A7DEBF001DE9B700AADEBF0020E9B70051
:10F7B000A8DEBF001EE9B700ABDEBF0021E9B7003D
:10F7C000B86F02000000000084E92100A4F988005D
:10F7D000D070020000000000047D200084F5880045
:10F7E0009C780200000000008C88A800E001200046
:10F7F0001059020000000000CF027800000006004F
:10F80000851F780084F02F00D4F2880004032300C1
:10F81000E4F2880004002600F4F2880004032300C8
:10F8200004F38800F0CEB30062FEB70074F02F003E
:10F8300024F388000403230034F3880004202A0002
:10F8400044F3880004F32E0054F3880094F02F0052
:10F8500064F388000403230074F388000400250087
:10F8600084F38800723EEF0004F02E00A4F38800B9
:10F8700094F02F00B4F3880004032300C4F388003D
:10F8800004102500D4F388007C3EEF0004F02E0025
:10F89000F4F3880084F02F0004F4880004032300AC
:10F8A00014F4880004402B0024F488001403200082
:10F8B00034F48800F0CEB30088FEB70044498000DD
:10F8C0007024E10003003200444980007124E1000B
:10F8D00009003A0052DEBF008CFEB70053DEBF00C5
:10F8E0008DFEB70054DEBF008EFEB7003A790200ED
:10F8F000000000001001370094F28000F447B200CD
:10F900000440780055FEB70094F280004822DE00E3
:10F91000F447B2000440780063FEB700A4F2800010
:10F92000F447B2000440780089FEB700895EE20027
:10F930000D003A00044980004822DE0004C3B200F2
:10F9400009003200B86F02000000000044E6210008
:10F95000A4F98800D0700200000000006ADEBF0039
:10F9600021E9B7008CA8A900555EE20014003A0016
:10F97000635EE20012003A00F44880004822DE0094
:10F9800004C3B20003003A000449800004C3B2007B
:10F990000B003200B86F020000000000A4E5210057
:10F9A000A4F98800D07002000000000060DEBF00F3
:10F9B0001FE9B70061DEBF0020E9B7008C88A9000D
:10F9C000555EE20005003A00635EE20003003A0083
:10F9D000895EE20001003A00D7003700555EE20080
:10F9E00004003A0000C3B30060FEB700107D0400BD
:10F9F0000000000052DEBF000048B20004082000F2
:10FA00000024E10004003A0020C3B30060FEB70008
:10FA1000107D04000000000010C3B30060FEB700BA
:10FA2000635EE20004003A0000C3B30061FEB70069
:10FA3000327D04000000000053DEBF000048B20029
:10FA4000040820000024E10004003A0010C3B300C1
:10FA500061FEB700327D04000000000020C3B30047
:10FA600061FEB70063DEBF000160EF0000027800B6
:10FA70007E20B80080027800E8824200B5F288005B
:10FA800055DEBF000160EF00140220000020B80026
:10FA900080027800E8824200C5F28800C4F280004B
:10FAA0006A20E10002003100A4002000C4F28800B6
:10FAB000C4F28000033220000418E100020031008B
:10FAC00004322000C4F28800B4F280006A20E10011
:10FAD00002003100A4002000B4F28800B4F28000DB
:10FAE000E32620000418E10002003100E426200093
:10FAF000B4F2880059DEBF00EF426000101FF8002A
:10FB0000E5FF9F00101FF9001A79020000000000B5
:10FB100072FEB70058DEBF000160EF004400DE0057
:10FB2000EF426000101FF800E5FF9F00101FF90072
:10FB30001A7902000000000073FEB70058DEBF0013
:10FB4000EF426000101FF800E5FF9F00101FF90052
:10FB50001A7902000000000074FEB70057DEBF00F3
:10FB6000EF426000101FF800E5FF9F00101FF90032
:10FB70001A790200000000007CFEB70056DEBF00CC
:10FB80000160EF004400DE00EF426000101FF8004B
:10FB9000E5FF9F00101FF9001A7902000000000025
:10FBA0007DFEB70056DEBF00EF426000101FF80078
:10FBB000E5FF9F00101FF9001A7902000000000005
:10FBC0007EFEB700555EE2000F00320004F38000B5
:10FBD00004C3B2000C0032008C88A8001CC9BF000E
:10FBE000555EE3000800320055DEBF001CE9B70097
:10FBF000B86F020000000000C4E62100A4F98800EC
:10FC0000D070020000000000635EE20010003200CD
:10FC100004F380004822DE0004C3B2000C0032006E
:10FC20008C88A8001DC9BF00635EE3000800320095
:10FC300063DEBF001DE9B700B86F020000000000DE
:10FC400064E72100A4F98800D070020000000000E1
:10FC500020C9BF00615EE30003003A001FC9BF0076
:10FC6000605EE3000A00320060DEBF001FE9B700FB
:10FC700061DEBF0020E9B700B86F0200000000009D
:10FC8000A4E52100A4F98800D07002000000000063
:10FC9000895EE2002800320054DEBF000048B20056
:10FCA000040820000024E10004003A0020C3B3004F
:10FCB0006AFEB700627E04000000000010C3B300BB
:10FCC0006AFEB7008CA8A8001EC9BF00895EE300C9
:10FCD0000E00320089DEBF001EE9B70089DEBF00DA
:10FCE00067406000004278000443B300044078009D
:10FCF00087FEB700B86F02000000000004E8210092
:10FD0000A4F98800D07002000000000021C9BF00E3
:10FD10006A5EE300080032006ADEBF0021E9B70036
:10FD2000B86F02000000000044E62100A4F988003A
:10FD3000D070020000000000CF0278000000060032
:10FD4000851F7800C500200003000900B51F78005A
:10FD50000202B80003F0A600020037000383B900D6
:10FD6000010037000303B8004200A90085024300E8
:10FD700060844B0001F0A60002003700028BB9003E
:10FD800001003700020BB80085024B0008844B00CD
:10FD90000980B000038BB90008044B0087834C0036
:10FDA0008701780008017800850078000400780059
:10FDB0002501200003000900CF127800CF0278004F
:10FDC00000000600851F7800C50020000300090020
:10FDD000B51F7800090020004300AF001900200083
:10FDE000891F78008384680001F0A60006003700B0
:10FDF0000000EA000100320002003A008100EA003F
:10FE0000010037008180EA0003F0A60006003700F9
:10FE10000201EA000100320002003A008301EA0018
:10FE2000010037008381EA000302690015003200F7
:10FE30000002EB008002EB000003EB008003EB000C
:10FE4000080220004200A9000080D2008180D20078
:10FE50000482D2008582D2000328E10001003A002A
:10FE600002A0E100030039000202520083825A001E
:10FE70004200A8000683D2008783D2000804E9006C
:10FE8000F0FF3A0009F0A600070037000600EA007C
:10FE90000100320002003A008700EA000500370046
:10FEA0008780EA00030037008700780006007800AA
:10FEB00000003700CF0478000900E00001003200A4
:10FEC0000400BE002501200003000900CF127800C5
:10FED000CF02780000000600851F7800861F78009A
:10FEE000871F780014002000E4F988003E3FEF00EF
:10FEF000417FEF00427FEF00B4F980006020E10015
:10FF00000E003C0003003500A4F980006020E100F1
:10FF10000A00310010C0B30041FFB700A0F9800013
:10FF2000B1F98000F2FF2F00F3FF2F00A07E020046
:10FF300000000000A0F98800B1F988003C1FE20031
:10FF400002003A003E1FE200310032004300A900E7
:10FF5000A0F98000B1F98000C2F980000300200000
:10FF6000E27E020000000000E0F98800F1F988005C
:10FF700014FA80000960EF00040078003A1FB40012
:10FF8000800278004300A800A0F98000B1F9800049
:10FF9000C2F9800003002000E27E020000000000A1
:10FFA0000003BE000403200004004300E0834B0074
:10FFB00087007800804A780014FA80000960EF001A
:10FFC000040078003A1FB400940320001024E100DC
:10FFD0000800310014FA80000960EF000400780086
:10FFE0003A1FB40080027800154278006742420050
:10FFF00084429800427FEC003C1FF800341FF90057
:020000040001F9
:100000003E1FF800361FF9009E7F0400000000002C
:1000100004FA80004822DE006124E10008003A0072
:1000200014FA80000960EF00040078003A1FB40061
:1000300080027800D0C2B300804A7800427FEC0092
:10004000407FEF0042DFBF000160EF004100DE00B3
:1000500004FA80000024E1001F003D0004FA800043
:100060000960EF00040078003A1FB40010407800E7
:1000700043FFB70004FA80000960EF000400780035
:100080003A1FB4008002780014FA800003FA80005E
:1000900003405200614050000080FB00D4F9800012
:1000A00004004000904A780014FA800003FA8000AF
:1000B00003405200614050000080FB00D4F98000F2
:1000C0008402400043DFBF00804A7800407FEC009C
:1000D000228004000000000014FA80000960EF0094
:1000E000040078003A1FB40080027800804AEB00D8
:1000F0003A1FF8000000F900CF0378004F037800A2
:10010000CF02780000000600851F7800341FF80039
:10011000361FF900B0F980001004E000030032003F
:10012000363FEC008A80040000000000B4F9800033
:10013000A3F9800003005200CF02780000000600FF
:10014000851F7800163FEF0054302200C4F8880065
:1001500004052300D4F8880004D02000E4F88800C7
:1001600054302200F4F888004405230004F9880084
:1001700004D0200014F988005430220024F98800AB
:10018000A405230034F9880004D0200044F9880035
:1001900094F88000F447B2000440780015FFB700DF
:1001A000A4F880004822DE006124E100140036003B
:1001B000A4F880004822DE007824E1000200360026
:1001C00080C1B30015FFB70015DFBF0016FFB700F1
:1001D000177FEF00B4F88000130320000320B8005D
:1001E00080027800050278008301200011000900D8
:1001F0000382D800B0F8880016DFBF0015FFB700F3
:1002000094F880004822DE00F447B20004407800F1
:100210002AFFB70054F980006124E1001300360082
:1002200054F980007424E1000200360040C1B3009C
:100230002AFFB7002ADFBF0016FFB700177FEF00C5
:10024000B4F88000130320000320B8008002780077
:100250000502780043012000110009000382D80044
:10026000B0F8880016DFBF002AFFB700A4F88000AE
:100270007447B200044078002BFFB7002BDFBF00AB
:10028000674060006104E1000F0036002BDFBF0013
:100290000160EF0067006000B0F88800B4F88000EB
:1002A000130320000320B8008002780005027800C4
:1002B00073002000110009000382D800B0F8880004
:1002C00016DFBF002BFFB700C1F2210002002000A3
:1002D000030009008058EB00155FE20006003A00B9
:1002E00050C3B3001BFFB70000C3B3001CFFB7002F
:1002F0001C8204000000000012DFBF000048B200B2
:10030000040820000024E10028003A002403200013
:10031000A3F88000C819DE000340520015FFB700A3
:1003200015DFBF0034FFB700357FEF00363FEF0029
:10033000A4002000C4F98800C4F22100D4F9880088
:100340006C7F020000000000800278000500E000E1
:1003500010003200C4F22100A4F988008480020059
:10036000000000006104E100060036002CDFBF0041
:100370001BFFB7002DDFBF001CFFB700C6810400C4
:10038000000000002CDFBF001CFFB700D28104007A
:100390000000000050C3B3001BFFB70000C3B30050
:1003A0001CFFB7001C820400000000002003200096
:1003B000157FB40015DFBF0034FFB700357FEF00B5
:1003C000363FEF00A4002000C4F98800C4F22100E9
:1003D000D4F988006C7F02000000000080027800E1
:1003E0000500E00010003200C4F22100A4F98800EA
:1003F00084800200000000006104E1000600360075
:100400002CDFBF001BFFB7002DDFBF001CFFB700B4
:1004100010820400000000002CDFBF001CFFB700AA
:100420001C8204000000000050C3B3001BFFB70093
:1004300000C3B3001CFFB70084F12100A4F98800B9
:10044000D070020000000000B86F02000000000041
:100450002A5FE20006003A0050C3B30021FFB70054
:1004600000C3B30022FFB700D682040000000000E2
:1004700013DFBF000048B200040820000024E100A0
:1004800025003A00200320002A7FB4002ADFBF00A5
:1004900034FFB700357FEF00363FEF00A4002000A7
:1004A000C4F98800C4F22100D4F988006C7F0200EE
:1004B00000000000800278000500E000100032001B
:1004C000C4F22100A4F9880084800200000000002A
:1004D0006104E100060036002CDFBF0021FFB700F9
:1004E0002DDFBF0022FFB7007C8204000000000067
:1004F0002CDFBF0022FFB70088820400000000004C
:1005000050C3B30021FFB70000C3B30022FFB70000
:10051000D6820400000000002403200053F980006C
:10052000034052002AFFB7002ADFBF0034FFB700A4
:10053000357FEF00363FEF00A4002000C4F98800AB
:10054000C4F22100D4F988006C7F02000000000092
:10055000800278000500E00010003200C4F22100A3
:10056000A4F9880084800200000000006104E1001A
:10057000060036002CDFBF0021FFB7002DDFBF00D3
:1005800022FFB700CA820400000000002CDFBF0079
:1005900022FFB700D68204000000000050C3B30061
:1005A00021FFB70000C3B30022FFB700E4F1210030
:1005B000A4F98800D070020000000000B86F0200AB
:1005C000000000002B5FE20006003A0050C3B300B9
:1005D00027FFB70000C3B30028FFB70092830400D1
:1005E0000000000014DFBF000048B2000408200033
:1005F0000024E10025003A00200320002B7FB400F6
:100600002BDFBF0034FFB700357FEF00363FEF0030
:10061000A4002000C4F98800C4F22100D4F98800A5
:100620006C7F020000000000800278000500E000FE
:1006300010003200C4F22100A4F988008480020076
:10064000000000006104E100060036002CDFBF005E
:1006500027FFB7002DDFBF0028FFB7003683040057
:10066000000000002CDFBF0028FFB7004283040019
:100670000000000050C3B30027FFB70000C3B30061
:1006800028FFB7009283040000000000240320002C
:1006900053F98000C819DE00034052002BFFB70059
:1006A0002BDFBF0034FFB700357FEF00363FEF0090
:1006B000A4002000C4F98800C4F22100D4F9880005
:1006C0006C7F020000000000800278000500E0005E
:1006D00010003200C4F22100A4F9880084800200D6
:1006E000000000006104E100060036002CDFBF00BE
:1006F00027FFB7002DDFBF0028FFB7008683040067
:10070000000000002CDFBF0028FFB7009283040028
:100710000000000050C3B30027FFB70000C3B300C0
:1007200028FFB70044F22100A4F98800D07002002D
:1007300000000000B86F020000000000CF02780047
:1007400000000600851F78008C28A9008C08A900ED
:100750008C48A9009048E2008A003200844480005E
:100760000960EF007300200004804100C48820006D
:1007700004004000104078002849E30081003A005E
:1007800028C9BF000160EF001080B2001F003200D6
:100790007080B2001D0032004080B2001B003200A9
:1007A0001080B200190032006080B20017003200E1
:1007B000D080B200150032001080B2001300320069
:1007C0006080B200110032008080B2000F00320061
:1007D0003080B2000D003200A080B2000B00320069
:1007E0004080B20009003200A081B2000E00320049
:1007F0001080B2000C003200D081B2001100320033
:100800001080B200160032001C0037003A7EEF0064
:100810003B7EEF003C7EEF00B4740200000000005D
:100820003E840400000000008C7EEF008D7EEF000F
:100830008E7EEF003A790200000000003E84040042
:1008400000000000527EEF00537EEF00547EEF0068
:10085000007C0200000000003E8404000000000054
:10086000127FEF00137FEF00147FEF00A0800200E3
:10087000000000003E84040000000000844480006A
:100880000960EF00F300200004804100C4882000CC
:100890008402400029C9BF00804A780090C8BF0088
:1008A0000160EF004100DD000004B000C4882000BA
:1008B00084024000944980008402980084448000AF
:1008C0000960EF00F30D200004804100C48820007F
:1008D0000400400010407800704060000004E00018
:1008E00028003A0090C8BF000160EF004100DD0021
:1008F0000003B000C488200084024000A4498000A6
:100900008402980090C8BF000160EF004100DD0044
:100910000006B000C488200084024000C449800062
:100920008402980090C8BF000160EF004100DD0024
:100930000007B000C488200084024000D449800031
:100940008402980090C8BF000160EF004100DD0004
:100950000005B000C488200084024000B449800033
:100960008402980090C8BF000160EF004100DD00E4
:100970000008B000C488200084024000E4498000E0
:1009800084029800A000200010590200000000001E
:10099000CF02780000000600820020001E0009003F
:1009A00000000000E2C2A900DEC2A9001F00090089
:1009B0000000000081C0D200C422A9004200AF00A4
:1009C000C022A8004200AE00C022A900DEC2A800DA
:1009D000E0C2AE00FEFF37000201E900EFFF3A007F
:1009E0001E00090000000000E2C2A900DEC2A9004A
:1009F00000000000C022A8001F0009000000000045
:100A00001F00090000000000DEC2A800E0C2AE0026
:100A1000FEFF37001F00090000000000000020005A
:100A2000C222AF000000A000E2C2A900DEC2A900FD
:100A3000C422A900C022A90000000600851F78007A
:100A4000F83DEF00C022A8001E00090000000000D1
:100A5000DEC2A8001F00090000000000E0C2AE00D6
:100A6000FEFF3700C422A900C022A9001E00090011
:100A700000000000E2C2A900DEC2A900A1C9B300C3
:100A8000CC84020000000000A1EF8000CC840200B2
:100A900000000000F83DEF00F5DDBF000160EF0051
:100AA000C4EF80000020E10009003100C0EF8000A9
:100AB000F61DB4009042780085407800CC84020096
:100AC00000000000F83DEC004C8504000000000030
:100AD000C022A90000000000DEC2A800E0C2AE00F3
:100AE000FEFF37001E0009000000000001000900A1
:100AF00000000000C022A8001E0009000000000045
:100B0000BE00090000000000CF02780000000600CF
:100B1000851F7800861F7800EE7DEF00EF1DA9008D
:100B2000DAC2AF0001003700560137008D48AE0031
:100B3000030037008C68AE00010037005101370018
:100B40008CE8AE0003003700EF1DA800D485040038
:100B5000000000008C68AE0003003700EF1DA90004
:100B6000D4850400000000003F09AE000D003700EE
:100B70000100200001007800AE1302000000000018
:100B80008100E800811F78002322AF00FEFF3700BC
:100B900020118800CF007800700020000008E600D7
:100BA000F4FF37003701370034EF8000E4CEB200A5
:100BB0000700320034EF8000F4CFB20004003200AE
:100BC000E6DDBF006F4060006204E100BE003A0055
:100BD000E6DDBF006F4060006204E10058003A00AB
:100BE0008D88AE00040037008DA8AF0001003700EB
:100BF0008DA8A800230137007008E20004003A0025
:100C000064092000844388001C8604000000000062
:100C10002209E20004003A002409E20002003A003E
:100C20002609E200040032008DA8AF000100370061
:100C30008DA8A80013013700254FE20009003200FB
:100C4000256FED0025CFBF00347980000024E1003E
:100C50000200360025CFBF0026EFB70094860400BF
:100C6000000000008D88AF002E0037008D88A8009E
:100C70008DA8AF00010037008DA8A8003F09AE0085
:100C8000280037000100200001007800C413020092
:100C9000000000008100E800811F78002322AF00DF
:100CA000FEFF370020118800CF007800600120008F
:100CB0000008E600F4FF370024CFBF000160EF001A
:100CC000040020004A710200000000009101200091
:100CD00001007800C4130200000000008100E80059
:100CE000811F78002322AF00FEFF3700201188000B
:100CF000CF007800200220000008E600F4FF370053
:100D000025CFBF000160EF00040020004A710200FF
:100D1000000000002322AF00FEFF370094022000F5
:100D200024118800D700370022C9BF00E7FDB700B3
:100D300024C9BF00E8FDB70026C9BF00E9FDB70020
:100D40003F09AE00410037008042EB00EF1DAF00CD
:100D50008502E8002322AF00FEFF3700A400200038
:100D6000241188002322AF00FEFF3700D4002000AA
:100D7000241188002322AF00FEFF370084022000E8
:100D800024118800054078000160EF000400200075
:100D90004A710200000000005100200001007800AC
:100DA000F8130200000000008100E800811F7800B5
:100DB0002322AF00FEFF370020118800CF0078000B
:100DC000400120000008E600F4FF3700E6DDBF0028
:100DD0000160EF002170220056690200000000004F
:100DE0002322AF00FEFF37000402200024118800F8
:100DF000E7DDBF000160EF002170220056690200AC
:100E0000000000002322AF00FEFF37000402200094
:100E100024118800E8DDBF000160EF00217022008E
:100E200056690200000000002322AF00FEFF3700D9
:100E30000402200024118800E9DDBF000160EF00FA
:100E4000217022005669020000000000E6DDBF00AC
:100E5000EAFDB700E7DDBF00EBFDB700E8DDBF004E
:100E6000ECFDB700E9DDBF00EDFDB7008CE8AE009A
:100E700009003700F47DEF0040C0B300F5FDB70076
:100E8000A4DE2100B4EF88001E85020000000000EF
:100E900060870400000000008C68AE000800370086
:100EA00020C0B300F4FDB70040C0B300F5FDB700AB
:100EB000A4DE2100B4EF88001E85020000000000BF
:100EC0004288040000000000F4788000F30F200046
:100ED0000418E100340031003F09AE003100370052
:100EE00001002000010078002A1402000000000028
:100EF0008100E800811F78002322AF00FEFF370049
:100F000020118800CF007800D00120000008E60002
:100F1000F4FF3700E6DDBF000160EF002170220022
:100F200056690200000000002322AF00FEFF3700D8
:100F30000402200024118800E7DDBF000160EF00FB
:100F40002170220056690200000000002322AF0039
:100F5000FEFF37000402200024118800E8DDBF00F6
:100F60000160EF00217022005669020000000000BD
:100F70002322AF00FEFF3700040220002411880066
:100F8000E9DDBF000160EF00217022005669020018
:100F9000000000002322AF00FEFF37009402200073
:100FA0002411880037003700E6DDBF006F40600085
:100FB000EEFDB700254FE20010003A00EEDDBF0065
:100FC0000160EF00C080B200050032001080B20066
:100FD00003003200C080B200030032000600370078
:100FE000FE87040000000000E85DE200020032001D
:100FF000FE870400000000002200370074EF80002C
:101000006224E1000A00360074EF80006C24E100E5
:10101000070031007008E20004003A006409200073
:101020008443880018880400000000001500370081
:101030001DCBBF000160EF004200DD00E4B12000E5
:1010400084024000E6DDBF00B0429800E7DDBF004B
:10105000A0429800E8DDBF0090429800E9DDBF00A3
:10106000804A78001E2FEC0000798000F478800020
:101070000020E100020036001E0FF800200FF900EA
:101080001D6BEC004F037800CF02780000000600D3
:10109000851F78008C68AE000C003700D0C8B30004
:1010A000E6FDB700F4DBBF00E7FDB700F5DBBF00EE
:1010B000E8FDB700F6DBBF00E9FDB7008885020058
:1010C0000000000082880400000000008CE8AE00F0
:1010D0000C0037008D28AE000A003700D0CCB300DA
:1010E000E6FDB700F4DBBF00E7FDB700F5DBBF00AE
:1010F000E8FDB700F6DBBF00E9FDB7008885020018
:1011000000000000CF02780000000600851F780074
:10111000861F7800871F7800A2830200000000006D
:10112000EC1BAF0002003700CB02A9000100370022
:10113000CB02A800EC3BAF0002003700CB22A90095
:1011400001003700CB22A800EC5BAF0002003700A3
:10115000CB42A90001003700CB42A800500020007C
:101160001059020000000000B86F020000000000EB
:101170002A29EF002C29EF002E29EF003029EF005B
:10118000ECDBBF0090E8B700ECDBBF000000FB0029
:101190006F004000C4882000040040001040780028
:1011A00029E9B700ECDBBF000000FB00670040004E
:1011B000C4882000040040004449800000429000A0
:1011C00044498800ECDBBF000000FB00000278000F
:1011D0006220B8000004B000C48820000400400071
:1011E000901F78003209F900844480000960EF0004
:1011F000F30D200004804100C4882000040040005A
:1012000010407800704060000004E0002D003A00BB
:10121000ECDBBF000000FB00000278006220B80099
:101220000003B000C488200004004000901F780034
:101230003409F900ECDBBF000000FB00000278007D
:101240006220B8000006B000C488200004004000FE
:10125000901F78003809F900ECDBBF000000FB00AC
:10126000000278006220B8000007B000C4882000A7
:1012700004004000901F78003A09F900ECDBBF0041
:101280000000FB00000278006220B8000005B000FA
:10129000C488200004004000901F78003609F9003F
:1012A000ECDBBF000000FB00000278006220B80009
:1012B0000008B000C488200004004000901F78009F
:1012C0003C09F900844480000960EF00430C2000D1
:1012D00004804100C488200004004000904278004F
:1012E000844480000960EF00C30C200004804100AA
:1012F000C48820000400400010437800844480002B
:101300000960EF00430D200004804100C4882000E4
:101310000400400090437800F41BF800E5FF9F00B4
:10132000F41BF90006407800F5FBB700F61BF80047
:10133000E7FF9F00F61BF90048880200000000004C
:10134000CF0378004F037800CF027800000006003A
:10135000851F7800861F7800FA3DEF0064F02F00AB
:10136000E4EF880004032300F4EF88000430260033
:1013700004F08800F0CEB30002FEB70074F02F0036
:1013800024F088000403230034F08800046028005F
:1013900044F0880004F02E0054F0880064F02F0020
:1013A00064F088000403230074F0880004702500B2
:1013B00084F08800F0CEB30012FEB70074F02F0066
:1013C000A4F0880004032300B4F08800040029007E
:1013D000C4F0880004F32E00D4F0880084F02F00BD
:1013E000E4F0880004032300F4F0880004502A008D
:1013F00004F188004403230014F18800F0CEB30008
:1014000024FEB70094F02F0034F188000403230079
:1014100044F1880004002B0054F188002C3EEF00BA
:1014200004F02E0074F18800A4F02F0084F18800ED
:101430000403230094F1880004002B00A4F1880029
:10144000363EEF00383EEF00F0CEB3003AFEB70074
:10145000E4F02F00E4F1880004032300F4F1880095
:101460000420260004F288008403230014F288007C
:101470000403230024F288008403230034F288004C
:101480000403230044F28800F0CEB3004AFEB70004
:10149000F8DDBF000160EF00F085B200830032008C
:1014A000C085B2008B0032005080B200890032004B
:1014B000B080B200870032001080B2008500320098
:1014C0004081B2008D0032001080B2009B003200DB
:1014D000D081B200AB0032001080B200B100320007
:1014E000A080B200B9003200F081B200C100320029
:1014F0001080B200D9003200F081B200E700320063
:101500006080B200EF003200F080B20005013200CE
:101510008082B20005013200F081B2001501320074
:101520006085B200250132001080B2003501320022
:101530006085B200450132003080B2004D013200BA
:101540008082B200550132001080B2006501320085
:101550007080B20075013200F084B2007D0132006B
:101560001080B200A70132004080B200CD013200ED
:101570005086B200D90132007080B200D70132002B
:10158000A082B200DF0132001080B200F50132000B
:10159000E087B2000B0232001080B2000902320074
:1015A0008085B200250232004080B2003502320050
:1015B0005080B200530232002080B2006302320039
:1015C0001080B200990232007080B200CF02320067
:1015D0008081B200F7023200F080B2004F03320087
:1015E0001080B200750332002080B2009B033200ED
:1015F0006086B200B5033200F080B2000904320008
:101600001080B200130432003080B2001C0432009B
:101610001080B200210432007080B2004404320015
:101620001080B200A60432003080B200C80432003C
:101630001080B200D1043200F080B200D704320032
:101640001080B200E00432003080B200E6043200C4
:101650001080B200F30432007080B200FD0432004A
:101660001080B200070532003080B2000E05320053
:10167000E081B200130532001080B200270532006D
:101680009080B2002F0532001080B2008105320038
:10169000D083B200D30532001080B200DD053200E5
:1016A000E086B200E7053200E605370000C9B30066
:1016B00019FEB70000C3B3001AFEB70044E12100D1
:1016C000A4F98800D0700200000000002A970400EE
:1016D0000000000000C9B30009FEB70000C3B3005A
:1016E0000AFEB70044E02100A4F98800D07002008F
:1016F000000000002A970400000000004449800018
:101700007024E10003003200444980007124E100AC
:1017100002003A0010C0B30000FEB70060C8B3007A
:1017200001FEB700C4DF2100A4F98800D0700200D8
:10173000000000002A9704000000000044498000D7
:101740007024E10003003200444980007124E1006C
:1017500002003A0010C0B30008FEB70060C8B30032
:1017600009FEB70000C3B3000AFEB70044E0210041
:10177000A4F98800D0700200000000002A9704003D
:101780000000000070C8B30001FEB700C4DF2100F4
:10179000A4F98800D0700200000000002A9704001D
:1017A0000000000010C0B30000FEB70070C8B30016
:1017B00001FEB700C4DF2100A4F98800D070020048
:1017C000000000002A9704000000000050CAB30087
:1017D00009FEB700C0C3B3000AFEB70044E0210011
:1017E000A4F98800D0700200000000002A970400CD
:1017F00000000000444980007024E1000300320032
:10180000444980007124E1000A003A0010C0B3008E
:1018100000FEB70040CAB30001FEB700C4DF2100DC
:10182000A4F98800D0700200000000002A8C040097
:101830000000000040CBB30009FEB70000C3B300B6
:101840000AFEB70044E02100A4F98800D07002002D
:10185000000000002A9704000000000044498000B6
:101860007024E10003003200444980007124E1004B
:1018700002003A0010C0B30000FEB70030C6B3004B
:1018800001FEB700C4DF2100A4F98800D070020077
:10189000000000002A9704000000000010CBB300F5
:1018A00009FEB70000C3B3000AFEB70044E0210000
:1018B000A4F98800D0700200000000002A970400FC
:1018C00000000000444980007024E1000300320061
:1018D000444980007124E10008003A0010C0B300C0
:1018E00008FEB70030CCB30009FEB70020C3B30038
:1018F0000AFEB700868C04000000000050CAB30046
:1019000009FEB700A0C3B3000AFEB70044E02100FF
:10191000A4F98800D0700200000000002A9704009B
:10192000000000002A9704000000000044498000E5
:101930007024E10003003200444980007124E1007A
:1019400002003A0010C0B30018FEB70000CAB3008E
:1019500019FEB70010C3B3001AFEB70044E121001E
:10196000A4F98800D0700200000000002A9704004B
:1019700000000000444980007024E10003003200B0
:10198000444980007124E10002003A0010C0B30015
:1019900018FEB70000CAB30019FEB70000C3B300B9
:1019A0001AFEB70044E12100A4F98800D0700200BB
:1019B000000000002A970400000000004449800055
:1019C0007024E10003003200444980007124E100EA
:1019D00002003A0010C0B30018FEB70050CBB300AD
:1019E00019FEB70010C3B3001AFEB70044E121008E
:1019F000A4F98800D0700200000000002A970400BB
:101A000000000000444980007024E100030032001F
:101A1000444980007124E10002003A0010C0B30084
:101A200018FEB70050CBB30019FEB70000C3B300D7
:101A30001AFEB70044E12100A4F98800D07002002A
:101A4000000000002A9704000000000050CAB30004
:101A500019FEB70010C3B3001AFEB70044E121001D
:101A6000A4F98800D0700200000000002A9704004A
:101A70000000000050CAB30019FEB70000C3B30055
:101A80001AFEB70044E12100A4F98800D0700200DA
:101A9000000000002A970400000000004449800074
:101AA0007024E10003003200444980007124E10009
:101AB00002003A0010C0B30018FEB70070CAB300AD
:101AC00019FEB70000C3B3001AFEB70044E12100BD
:101AD000A4F98800D0700200000000002A970400DA
:101AE00000000000444980007024E100030032003F
:101AF000444980007124E10002003A0010C0B300A4
:101B000018FEB70070CAB30019FEB70010C3B300C7
:101B10001AFEB70044E12100A4F98800D070020049
:101B2000000000002A9704000000000020C3B3005A
:101B30001AFEB70070CAB30019FEB70044E12100D5
:101B4000A4F98800D0700200000000002A97040069
:101B500000000000444980007024E10003003200CE
:101B6000444980007124E10018003A0010C0B3001D
:101B700034FEB70030C8B30035FEB70000C3B30071
:101B800036FEB70091C8BF00EF426000101FF8009A
:101B9000E5FF9F00101FF9001A7902000000000005
:101BA00037FEB70000C3B30038FEB70020C3B30050
:101BB00039FEB70004E32100A4F98800D0700200C8
:101BC00000000000FE8D040000000000A0C8B3006B
:101BD00019FEB70091C8BF006F4060000042780056
:101BE0000443B300044078001AFEB70044E121002A
:101BF000A4F98800D0700200000000002A970400B9
:101C000000000000444980007024E100030032001D
:101C1000444980007124E10014003A0010C0B30070
:101C200020FEB70020C8B30021FEB70000C3B300F8
:101C300022FEB70091C8BF00EF426000101FF800FD
:101C4000E5FF9F00101FF9001A7902000000000054
:101C500023FEB700C4E12100A4F98800D07002007F
:101C6000000000004E8E04000000000090C8B30089
:101C700019FEB70091C8BF006F40600000427800B5
:101C80000443B300044078001AFEB70044E1210089
:101C9000A4F98800D0700200000000002A97040018
:101CA00000000000B0C8B30019FEB70091C8BF0023
:101CB0006F406000004278000443B30004407800A5
:101CC0001AFEB70044E12100A4F98800D070020098
:101CD000000000002A9704000000000050CAB30072
:101CE00019FEB70020C3B3001AFEB70044E121007B
:101CF000A4F98800D0700200000000002A970400B8
:101D000000000000444980007024E100030032001C
:101D1000444980007124E10008003A0010C0B3007B
:101D200018FEB70040C8B30019FEB70000C3B300E7
:101D30001AFEB700A68E04000000000050CAB300CF
:101D400019FEB70020C3B3001AFEB70044E121001A
:101D5000A4F98800D0700200000000002A97040057
:101D600000000000444980007024E10003003200BC
:101D7000444980007124E10008003A0010C0B3001B
:101D800018FEB70040C8B30019FEB70010C3B30077
:101D90001AFEB700D68E04000000000050CAB3003F
:101DA00019FEB70030C3B3001AFEB70044E12100AA
:101DB000A4F98800D0700200000000002A970400F7
:101DC00000000000444980007024E100030032005C
:101DD000444980007124E1000C003A0010C0B300B7
:101DE00018FEB70040C8B30019FEB70000C3B30027
:101DF0001AFEB70044E12100A4F98800D070020067
:101E0000000000001A8F04000000000050CAB30058
